:020000040000FA
:040000006FD00400B9
:101000006F00907E00000000000000009020002093
:10101000AA220020A9BDF9F56C23002000000000E1
:10102000000000006C230020902000200000000041
:101030000000000090200020000000009020002010
:101040000000000090200020902000209020002030
:101050009020002090200020582F00209424002071
:101060000000000090200020902000201E2400207E
:1010700090200020D22300209020002090200020EB
:101080009020002090200020902000209020002020
:101090009020002001A04111B7170040985F3AC688
:1010A000945F3247E39CE6FE3245410182800111A4
:1010B00013078008F337078093F787083EC20100C3
:1010C0000100B7170040930570052380B70413068D
:1010D00080FA2380C7040100010083C6B70493F699
:1010E000F60DA385D704238007049246F3A6068055
:1010F0000100010093760502D5CEF336078093F602
:10110000860836C4010001002380B7042380C70489
:1011100001000100B70614007D89558D88C70100C4
:1011200001000100010023800704A246F3A6068007
:101130000100010073370780137787083AC6010062
:1011400001002380B7042380C704010001000100CF
:1011500001003727004093061005A303D7802380A2
:101160000704B247F3A70780010001009307800836
:10117000F3B7078093F787083ECE01000100B71749
:101180000040130770052380E704130780FA2380CB
:10119000E7040100010003C7B70413670708A3852C
:1011A000E70423800704F247F3A70780010001004A
:1011B0000561828093760504BDC6F336078093F6F9
:1011C000860836C8010001002380B7042380C704C5
:1011D00001000100B7061400938606047D89558D31
:1011E00088C7010001000100010023800704C246F6
:1011F000F3A6068001000100733707801377870884
:101200003ACA010001002380B7042380C70401000B
:1012100001003727004093062005A303D7802380D1
:101220000704D24781B773370780137787083ACC12
:10123000010001002380B7042380C70401000100DE
:1012400098471367070C98C723800704E24719BF24
:101250000111814601468145114506CE97000000E7
:10126000E780605893078008F3B7078093F78708F3
:101270003EC601000100B717004013077005238028
:10128000E704130780FA2380E7040100010003C785
:101290006704136717002383E70423800704B2471A
:1012A000F3A7078001000100F2400561828041112F
:1012B000814601468145114597000000E780A05214
:1012C00013078008F337078093F787083EC40100AF
:1012D0000100B7170040130670052380C70493066A
:1012E00080FA2380D70401000100FD552396B70240
:1012F00023800704A245F3A5058001000100733790
:101300000780137787083AC6010001002380C704CD
:101310002380D7040100010003C767041367170087
:101320002383E70423800704B247F3A70780010063
:10133000010001A0B1473305F50201007D1575FDDF
:101340008280411122C426C206C6AA8401446317C2
:101350009400B24022449244410182800504130566
:10136000803E420497000000E78000FD4180C5B741
:101370009305000273A04580824573901534924016
:101380002242B2424243D2436244F2440255925551
:101390002256B2564257D2576258F25806499649D9
:1013A000264AB64A464BD64B664CF64C065D965DD1
:1013B000265EB65E465FD65F09617300203041113C
:1013C000B7170040985F3AC6945F3247E39CE6FE49
:1013D000324541018280B71700401307000323887C
:1013E000E7028547171700002322F75673002030C5
:1013F000411122C42D6426C24AC006C637190040D6
:101400001304A4AAB704002023208900976000E0F9
:10141000E78000319C408297976000E0E780403091
:10142000E5B737370040834747009146BD8B639E41
:10143000D702B73600401306F00F973500009385AA
:10144000E52D9737000083D7673D03C7A6001377C4
:10145000F70F1DE3B7E70400BC4F09468945171590
:1014600000000345A5F7829731A099466394D70001
:10147000834757007300203003C786001377F70FA8
:10148000E365F6FC13851700AE97173800002317A5
:10149000A8382380E70075B7B787004003C7670007
:1014A000098B6309071003C77700930600031377BE
:1014B0000703630DD708174800000348F88517464F
:1014C0000000130666820547B30606012380E60086
:1014D00083C577001747000013070783429793F5EA
:1014E000F50F2300B70003C58700974500009385DB
:1014F000A580C2951375F50F2380A500034707004B
:1015000089451377F703630CB70C63E7E50A6306B5
:10151000071A8545630CB7129737000083C7D77F3A
:101520003307F600034707001377F70F19CB85073A
:1015300093F7F70F3D476363F71A17370000A30DC2
:10154000F77CB787004009472383E700B78700404F
:1015500083C77700E207E18763DE0704973700005F
:1015600083C7977B17370000130707783E97854698
:101570002300D70017370000130707793E9793061B
:1015800000032300D700173700001307E7763E97C4
:10159000A14685072300D70093F7F70F3D47636403
:1015A000F71417370000A309F776B78700400947FB
:1015B0002383E70073002030930610026300D70EE8
:1015C000930620026305D70693060002E316D7F4BC
:1015D00003C727021377C70F13672700D5A803C7D0
:1015E00067001377070465CB03C7A702173800000D
:1015F000130808511735000013054548134707081D
:101600002385E70203C7A7021377370F1367870005
:101610002385E702814713070004B305F5008C41D9
:10162000B306F80091078CC2E399E7FEF5B503C74E
:10163000A702134707042385E70203C7A70213770E
:10164000C70F136727002385E702F9B503C76700B3
:101650001377070449C303C767021738000013084C
:10166000E83D173500001305253513470708238388
:10167000E70203C767021377370F136787002383D7
:10168000E702814713070004B305F5008C41B30658
:10169000F80091078CC2E399E7FEBDBD03C767025E
:1016A000134707042383E70203C767021377C70FB3
:1016B000136727002383E70285B503C76700137705
:1016C000070411CB03C727021377370F136787006F
:1016D0002381E70291B5238006003DBD97370000C6
:1016E000A38C0762B9BD97370000A387076275BD59
:1016F0002303048015472303E48001002302A48010
:10170000828083076480E3CE07FE23030480828007
:1017100083076480E3CE07FE03454480828083070D
:101720006480E3CE07FE2302A4808280411126C498
:101730004AC24EC006C61377F50BAD47AA892E895B
:101740009544630CF700194597000000E78080FA84
:1017500097000000E78020FB8D444E859700000035
:10176000E78040F9FD59FD1463983401B240A2446A
:101770001249824941018280135509011375F50F01
:1017800097000000E780E0F92209F1BF011126CCA3
:1017900006CEB704080097000000E780C0F61545A4
:1017A00097000000E78000F597000000E78080F6D2
:1017B00097000000E78000F62AC697000000E78047
:1017C00080F432459377150089EB13651500137586
:1017D000F50FF240E24405618280FD14E9F0014515
:1017E000CDBF397126DC4ADA4ED852D656D45AD2F9
:1017F0005ED006DE62CE66CCB7E700E07D5783AAF6
:10180000070022C603AA470023A0E71823A2E7186F
:10181000B7170040130770052380E704130780FA09
:101820002380E70483C74704930B75FFB684E20760
:1018300093FBFB0F8546AA892E8B32893724004003
:10184000E187015763FA76016308D50089461307DB
:1018500000026313D5000157D98F93F7F70FB71C18
:1018600000402382FC0411472303E4801305F00F9A
:1018700097000000E78000E8094C97000000E7802F
:1018800080E863657C15B7050700DA9537870700A0
:10189000795563FEE504B3879500636AF704370B57
:1018A0000800A94733EB65016395F90881E8814495
:1018B00097000000E78020E5268515A8DA85094510
:1018C00097000000E780C0E605090345F9FFFD1415
:1018D000050B97000000E780C0E481C49377FB0FFD
:1018E000E5F797000000E780A0EA69F17D55B7179A
:1018F0000040130770052380E704130780FA238054
:10190000E70403C74704418B2382E704F250B7E79B
:1019100000E023A0571123A24711E2543244525948
:10192000C259325AA25A125B825B724CE24C21615C
:101930008280A547639BF90685691309F00FB306FA
:101940009900B3742B01B6941349F9FFB37499004D
:10195000856B33796901416B9387F9FFB3F72701F1
:1019600099E363FC340193D94900C147E3E637FFAB
:101970003DBF0569C1697D19D9B71305800D63881D
:101980006901130500026384790113051008CA85F3
:1019900097000000E780C0D997000000E78040DF93
:1019A00031D54E99B38434416DBFDA852D4597000A
:1019B0000000E780E0D7CA94E30B99EE0509970091
:1019C0000000E78020D5A30FA9FEFDB79387F9FF9C
:1019D00093F7F70F636DFC0C83C71C0413073008E3
:1019E0006315F706370708006361EB06B3079B0032
:1019F000B706100063FBD704334BEB0089476399AC
:101A0000F9068980D549E38404EADA850945970017
:101A10000000E780E0D111090327C9FF9147232087
:101A2000E48003076480E34E07FE23033481FD173F
:101A3000EDFBFD14110B81C49377FB0FE9FF9700B9
:101A40000000E780E0D461F155B5B717004003C747
:101A50005704B70708001377070219E3B787070091
:101A60007955E376FBE833079B00E3F9E7F841B5E6
:101A70008547E380F9F0DA852D4597000000E7807F
:101A800020CB9389F4FFE38404E297000000E78011
:101A900060C893F7390091EB83260480032709007F
:101AA00093074900E396E6E03E89CE84D9BFB54767
:101AB0006399F9001305900B97000000E78080C33D
:101AC000FDB3B1471305B00AE388F9FE9947639760
:101AD000F904B7050800B365BB002D459700000069
:101AE000E78000C581448D4BA14997000000E78045
:101AF00060C263967401832704802320F900850463
:101B0000E39534FF8327048013172B0163550700E7
:101B10002312F90069BB2322F90051BB9D47639F43
:101B2000F90281451305B00497000000E78040C02A
:101B3000BD442320090023220900FD59970000001D
:101B4000E78040BD93F77400CA9703C70700FD14F0
:101B5000398D2380A700E39334FF91BBA14763979E
:101B6000F90697000000E780A0C28144630D0B00D6
:101B70008D479304C0036308FB00930400056304CE
:101B80008B01930440041375C507E30295D21945F0
:101B900097000000E78000B697000000E780A0B63D
:101BA000054597000000E780E0B426859700000017
:101BB000E78020B7094597000000E78080B69700CE
:101BC0000000E780E0BCE31405CE0DB39147639FAE
:101BD000F9001305600697000000E780A0B19700A8
:101BE0000000E78040B213059009F9B5E38109CC04
:101BF000F1547DB9BD660147173600001306462F24
:101C0000938606A685458347060093F7F70F91C391
:101C100082800507E3F9E6FE97370000238AB72C98
:101C2000DDB77D166206618693178601E18763D46E
:101C3000070001458280931726003307F500AE9711
:101C400018439C4363E7E7007D16E37FF7FC7D556F
:101C5000828005458280FD15E205E18513978501A7
:101C6000618793F7F50F63480700FD15139725006B
:101C70002A97584365D713851700620561858280CE
:101C80003308B5021C4283A80600B335B502C297DB
:101C900033B50701AE98469585486367B5006394F0
:101CA000A50063E3070181480C43C6950CC388C2B5
:101CB0001CC2828081471397870161876343B70005
:101CC0008280139727002A97232007008507E5B70E
:101CD0008147014793968701E18663C5B6001335B6
:101CE0001700828093962700AA9694428507558F05
:101CF000D5B793D755408A07AA979C430545331516
:101D0000B5007D8D828017F3FFDFE702833D2A84D3
:101D100097000000E78060F405C5931725003E9406
:101D20000327C4FF814711EB7D1516053E9542053B
:101D3000418517F3FFDF6700033D05838507E5B79E
:101D40000145C5BF81471397870161876343C7007A
:101D5000828013972700B386E50094422A9785076F
:101D600014C3D5B77D1662066186014793178601B5
:101D7000E18763D50700133517008280931726008B
:101D8000B306F500AE9794429C437D16B58F5D8FE8
:101D9000F1BF8A05AA9501476363B500828083A6D7
:101DA000C5FFF11593D71600D98F9CC11397F60183
:101DB000E5B72A830148014701456343D700828084
:101DC000B387050183A80700B30706019C43C697A4
:101DD000AA976384F80033B517010507B308030118
:101DE000620723A0F80061871108C1BF2A83014759
:101DF0008147014563C3D70082803388E50083288B
:101E00000800330EE600032E0E003388A840330886
:101E1000C8416384080133B508018507B308E300AE
:101E2000E20723A00801E1871107E9B717F3FFDFF5
:101E3000E702232B0111B286B2842E86AA850A8579
:101E400097000000E780C0FA2A84A6850A859700DB
:101E50000000E78020E833348000060413351500C5
:101E6000018D056117F3FFDF6700E32917F3FFDF3B
:101E7000E702A3244111AA89AE8A328BB68402C23A
:101E800002C402C60144131C8401135C8C416349E3
:101E90009C02939B1400FD1B0549138CF4FFF15C1D
:101EA00033048901620461846340740792478E049D
:101EB000CE9423AEF4FE410117F3FFDF67006323E6
:101EC00013192400B30B2B01014A93172A00D6974C
:101ED00083A50B0088437800340050009700000071
:101EE000E78040DA050A93178A01E187F11BE35E78
:101EF000FCFC92474E9905042320F900A2473EC2FC
:101F0000B24702C63EC441B7131A8901135A8A4127
:101F1000131D240093178A01E18763CF970092472E
:101F20000A044E941CC0A24705091379F90F3EC25A
:101F3000B24702C63EC4ADB7B3079A0313152A00D1
:101F400056950841780034005000050AEA97DA9760
:101F50008C4397000000E780E0D26DBF197106C284
:101F600012C416C61AC81ECA22CC26CE2AD02ED219
:101F700032D436D63AD83EDA42DC46DECAC0CEC2C9
:101F8000D2C4D6C6DAC8DECAE2CCE6CEEAD0EED2F9
:101F9000F2D4F6D6FAD8FEDA971500009385859A22
:101FA0008841E700050092402242B2424243D243B8
:101FB0006244F244025592552256B2564257D257C5
:101FC0006258F25806499649264AB64A464BD64BBD
:101FD000664CF64C065D965D265EB65E465FD65F45
:101FE0000961730020300000972100209381810156
:101FF000175100201301018117F5FFFF1305C500DC
:102000009705002093850500171600201306C6FDCE
:1020100063FAC5008322050023A055001105910530
:10202000E3EAC5FE17E50100130585FF97150020BB
:102030009385C5FB171600201306466463FAC50096
:102040008322050023A0550011059105E3EAC5FE92
:1020500017150020130585629745002093850531EB
:102060006377B500232005001105E36DB5FEFD4241
:10207000739002BC8D4273904280B722000093821D
:10208000828873900230970200209382A2F793E235
:1020900032007390523097520000938242827390C4
:1020A00012346FB0F47573002030397101436EC67D
:1020B00019A0397141536AC866CA62CC5ECE19A0B4
:1020C000397101535AD056D252D44ED64AD826DA54
:1020D00022DC06DE33016140828241114AC026C201
:1020E00022C406C68282B24D4101024D924C224C5E
:1020F000B24B4101024B924A224AB2494101024984
:1021000092442244B240410182803D432A87637356
:10211000C3029377F700BDEFADE5937606FF3D8AE6
:10212000BA960CC34CC30CC74CC74107E36BD7FE30
:1021300011E28280B306C3408A0697020000969699
:102140006780A6002307B700A306B7002306B700E1
:10215000A305B7002305B700A304B7002304B70005
:10216000A303B7002303B700A302B7002302B700FD
:10217000A301B7002301B700A300B7002300B700F5
:10218000828093F5F50F93968500D58D9396050182
:10219000D58D61B7939627009702000096968682A8
:1021A000E78086FA9680C1171D8F3E96E374C3F8C8
:1021B000A5B7B717004003C777051377E70FA38BC1
:1021C000E704130700F8A38DE7043D47238CE704D9
:1021D00013075003A38CE70403C7A7051377D70F92
:1021E000238DE7048280B717004003C7E7020D89FB
:1021F00041111377C70F498F93068008F3B6068005
:1022000093F6860836C60100010093067005238008
:10221000D704930680FA2380D704010001002387A6
:10222000E70223800704B247F3A7078001000100FB
:102230004101828041112A83014E930E407E130F8B
:102240000019930F400663E56E12930800191303FB
:102250004006B3781503854E0D4FA14F33736502C9
:102260000D891335150063EFBE121308F6FF79468A
:1022700072984208135808013307C70213D6170093
:10228000BE0732976146B3F6C60213068070B38666
:10229000C6023697A166F58F42075D8FB7160040DC
:1022A00083C7F60293F70708A303F1000346710002
:1022B00083C7F60293F70708E394C7FE83477100CC
:1022C000B716004093F7F70F63880712930780084B
:1022D000F3B7078093F787083EC401000100B717E2
:1022E0000040930670052380D704930680FA23806C
:1022F000D7040100010023AA070383C6170393E64E
:102300000608A388D70223800704A247F3A7078003
:10231000010001001166B71700407D16D45BC85F4D
:1023200093854703A98EF18EF5FA93068008F3B6DC
:10233000068093F6860836C60100010093067005F4
:102340002380D704930680FA2380D704010001007C
:1023500098C103C7170313670704A388E702238004
:102360000704B247F3A70780010001004101828002
:102370007D133368E3039308E016630E08003368A7
:10238000F3039308D016630808009378330093B8DA
:1023900018009388D81633081E01131E0801135E17
:1023A0000E0155B56393E5030548638608000148AF
:1023B000630303002A8871087298FD15131E080133
:1023C000C205135E0E01C18179BD13F8150063F4D7
:1023D000BF007908D5B713381800E5BF83C7F602E8
:1023E00093F70708A303F1000346710083C7F602C1
:1023F00093F70708E394C7FE8347710093F7F70F3D
:10240000F1DFE9B531714AD966CB06DF22DD26DB83
:102410004ED752D556D35AD15ECF62CD6AC96EC758
:10242000AA8C02D897100000E78020B12A89930770
:102430008008F3B7078093F787083EDA01000100B0
:10244000B7170040130770052380E704130780FACD
:102450002380E7040100010003C7F7021377770F19
:10246000A387E70203C7F70213678700A387E70282
:1024700023800704D257F3A7078001000100054518
:1024800097000000E78060D6130780C13347E90258
:10249000116A93070AE893065002BD69930BA004E2
:1024A000814A014B13048008930470057D1AB347D9
:1024B000F9023307D7023EC0FD873ECC938709A6B9
:1024C0009309803E3347F7023AC27D873AC43347C7
:1024D00039038549B399990193D93940B306D70295
:1024E000B30B7703B3C6F602B3CBFB0236C6FD8649
:1024F00036C893D6FB4136CEB7460F0093860624E6
:102500003349D9028566938606FAB3969601B38954
:10251000E902130760553309D90293060010B38905
:10252000E9023349D902B3C9F9029316390036CA10
:1025300037190040FD8636D0930D090493D7F94131
:102540003ED2F336048093F6860836DC01000100A3
:10255000930770052380FD00930680FA2380DD0039
:10256000010001008346390593F6860FA309D904BB
:102570008346390593E61600A309D90423800D008C
:10258000E256F3A6068001000100130C80FA116DDB
:10259000F336048093F6860836DE010001009307C7
:1025A00070052380FD0023808D010100010083461A
:1025B0003905216693E60602A309D9048356090565
:1025C000B3E6A6012318D90483560905D18E231832
:1025D000D90423800D00F256F3A606800100010005
:1025E0008346390593F606026381061A03463905C8
:1025F000218A6DDE081897100000E7800098733676
:10260000048013768608B2C20100010023809D0079
:1026100023808D0101000100B717004003C6370574
:102620001376F60DA389C70403C6370513660602A1
:10263000A389C704835609052166B3E6A6012318BA
:10264000D90483560905D18E2318D90423800D009F
:102650009646F3A60680010001008346390593F6ED
:102660000602638B061483463905A18AEDFE9700A6
:102670000020E78040A2AA8636D497000020E78099
:1026800080A1A256E30AD5FE835609054255B3E65A
:10269000A6012318D90497100000E780C08F834655
:1026A0003905A18AEDDE03560905834629058247CF
:1026B0003376CA00B306DA0293D5F641B296B388F0
:1026C000F640E24733B8C6002E983308F840A247D8
:1026D000B3B616013308D84063C70701631DF8007D
:1026E000924763FA1701C247634FF80E63950701DB
:1026F000B24763EAF80E894663E9660FF24693151E
:10270000180013D3F8015E8613951800B365B30063
:1027100042D646D497A00100E78040063258050B08
:10272000137BFB0F63470001631A0838A2586387C5
:10273000083813081500B336A800B69513D6F5016E
:102740003298B336C800AE9613581800FE06B3E6AA
:1027500006017336048013768608B2C601000100B4
:1027600023809D0023808D01010001000356C902D2
:10277000B296C206C1822316D90223800D00B64646
:10278000F3A606800100010021B5F336048093F61C
:102790008608B6C00100010023809D0023808D01C2
:1027A000010001008346390593E60602A309D90416
:1027B00023800D0086460DB5F336048093F6860817
:1027C000B6C40100010023809D0023808D0101001B
:1027D00001008346390593E60602A309D904238044
:1027E0000D00A646BDB5E30B0BF0F336048093F65F
:1027F0008608B6C801000100930680FA23809D0078
:102800002380DD00010001008346390593F5FC0FAC
:1028100093F6860FA309D90483463905CD8EA30903
:10282000D90423800D00C646F3A6068001000100EE
:10283000130580FA03463905930639051D8A631C82
:1028400096297336048013768608B2CC0100010005
:10285000130680FA23809D002380CD000100010033
:1028600003C606001376F60D2380C60003C60600D5
:10287000136606022380C600835609051166D18EB1
:102880002318D904835609052166D18E2318D9044B
:1028900023800D00E646F3A6068001000100130622
:1028A00080FA8346390593F606026380062683463E
:1028B0003905130C3905A18AFDDA081897000000C4
:1028C000E780A06BF336048093F68608B6D001004B
:1028D0000100930680FA23809D002380DD00010023
:1028E000010083460C00116693F6F60D2300DC0010
:1028F00083460C0093E606022300DC00835609059C
:10290000D18E2318D904835609052166D18E231848
:10291000D90423800D008656F3A60680010001002D
:10292000130680FA8346390593F60602638A062069
:1029300083463905A18AEDFE97F0FF1FE780A07559
:102940002A8C97F0FF1FE7800075E30C85FF835604
:10295000090511664255D18E2318D904970000004D
:10296000E78060638346390513063905A18AFDDADD
:10297000F336048093F68608B6D40100010093066E
:1029800080FA23809D002380DD0001000100834642
:10299000060093F6F60D2300D60023800D00A65600
:1029A000F3A60680010001008356090503462905A8
:1029B000D247B376DA003306CA021305800C93556A
:1029C000F6413696330DF6408257333CD6002E9CA6
:1029D0003336A601330CFC40330CCC40330885035E
:1029E00092564E86B335A5033305A503C29597A02D
:1029F0000100E780A0D863468001631E0C16630CBB
:102A00000D16130615003335A6002E959356F501C5
:102A10003696B335D600AA959396F501058285853D
:102A2000D18E6346B000639D051A638B061A035668
:102A3000C90215823305D6003336C500B295634806
:102A4000B000639105241306F00F637DA62289462A
:102A500063F3561593078008F3B7078093F7870849
:102A6000BED6010001003717004093077005230010
:102A7000F704930780FA2300F7040100010083564E
:102A8000C70289678117D58FC207C1832316F70252
:102A900023000704B657F3A7078001000100FA508E
:102AA0006A54DA544A59BA592A5A9A5A0A5BFA4B62
:102AB0006A4CDA4C4A4DBA4D296182801308F5FF01
:102AC0003335A800FD152E951356F5013298B3360F
:102AD000C800AA9695B9F336048093F68608B6CA5C
:102AE0000100010023809D002380AD000100010052
:102AF00083463905CD8EA309D90423800D00D6461F
:102B0000F3A606800100010035B3F336048093F686
:102B10008608B6CE0100010023809D002380CD00F1
:102B2000010001008346390593E60602A309D90492
:102B300023800D00F646F3A606800100010095B340
:102B4000F336048093F68608B6D201000100238094
:102B50009D002380CD00010001008346390593E6E6
:102B60000602A309D90423800D009656F3A6068019
:102B70000100010045BB9306F5FF33B5A600FD1526
:102B80002E959355F501AE96B3B5B600AA9513965A
:102B9000F501858269B5F336048093F68608B6D8C8
:102BA00001000100930680FA23809D002380DD0050
:102BB000010001008356C9020566011693F6F60F5F
:102BC000D18EC206C1822316D90223800D00C656BB
:102BD000F3A6068001000100850A93FAFA0F95B268
:102BE00033E6B60045C20356C9023305D040333838
:102BF000A000B305B040B385054115826345B00020
:102C0000D1E16371A608894663F0560593078008F1
:102C1000F3B7078093F78708BEDA01000100B71702
:102C20000040130770052380E704130780FA238010
:102C3000E7040100010003D7C7027D8B2396E7025A
:102C400023800704D65781BDF336048093F68608A7
:102C5000B6DC01000100930680FA23809D002380EA
:102C6000DD00010001008356C9020566011693F6D6
:102C7000F60FD18EC206C1822316D90223800D0021
:102C8000E656B9B793078008F3B7078093F787082C
:102C9000BEDE0100010037170040930770052300D6
:102CA000F704930780FA2300F7040100010003569C
:102CB000C70293975600B297C207C1832316F70243
:102CC00023000704F657C1BB914763EEB70217B75D
:102CD0000100130727458A05BA959C41BA97828758
:102CE000B717004003A7470B1345F5FF698F23AAC9
:102CF000E70A03A7070B698F23A8E70A03A7070AB8
:102D0000798D23A0A70A8280B717004083A6470BBE
:102D10001347F5FFF98E23AAD70A83A6070B558D13
:102D200023A8A70A83A6070A758F23A0E70A828033
:102D3000B717004003A7470B498F23AAE70A03A749
:102D4000070B1345F5FF45BFB717004083A6470B98
:102D50001347F5FF758F23AAE70A03A7070A598DC2
:102D60004DB7B717004003A7470B498FEDB7914701
:102D700063EEB70217B701001307073C8A05BA953F
:102D80009C41BA978287B717004003A7470D1345A8
:102D9000F5FF698F23AAE70C03A7070D698F23A806
:102DA000E70C03A7070C798D23A0A70C8280B71727
:102DB000004083A6470D1347F5FFF98E23AAD70CD1
:102DC00083A6070D558D23A8A70C83A6070C758F26
:102DD00023A0E70C8280B717004003A7470D498F57
:102DE00023AAE70C03A7070D1345F5FF45BFB71747
:102DF000004083A6470D1347F5FF758F23AAE70C04
:102E000003A7070C598D4DB7B717004003A7470D0F
:102E1000498FEDB7797122D43714004026D24AD0B9
:102E2000035924028354040206D64209C2044ECE3A
:102E300052CC56CA13590901C1802DE11379F9F713
:102E400093F4F49F4209C20413590901C180930706
:102E50008008F3B7078093F787083EC4010001009C
:102E6000930770052300F404930780FA2300F40409
:102E70000100010023112403231094022300040401
:102E8000A247F3A7078001000100B25022549254D8
:102E90000259F249624AD24A45618280B7F5070079
:102EA00081463000B105194597000020E780609306
:102EB000A24713972701E34A07FC1369090893E423
:102EC000044093098008F3B7098093F787083EC050
:102ED00001000100930A700523005405130A80FACB
:102EE0002300440501000100231124032310940250
:102EF000230004048247F3A707800100010029454D
:102F000097F0FF1FE7800043F3B9098093F9890820
:102F10004EC20100010023005405230044050100B6
:102F200001008357040293E707202310F4022300D3
:102F300004049247B9B7B71700408847420541815A
:102F40009377050491EB9377F5013755E801130565
:102F500005803345F50282809377050C1307000442
:102F60006397E7009377F50137459C1CCDB7216542
:102F7000130505D0828037E700E01C435443A1834A
:102F8000E206D58F1CC1FD572320F7182322F7181E
:102F9000828013178500B7E700E023A0E710618166
:102FA00023A2A7108280B7F700E08847CC47828031
:102FB000814737370040A14663C4C700328582800D
:102FC0000345B740E38EA6FE3385F50003450500B3
:102FD00085072304A740CDB79707002093870701F3
:102FE0009C4317370020130767383E95636EE50052
:102FF00017370020130707616368A7001707002031
:103000002326A7FE3E858280FD57EDBF82804111B9
:1030100022C406C62A8497000000E78000F22947F0
:10302000B307E502B2408D83B3D7870222449507E8
:10303000B3D7E70237370040C207C1832316F70032
:1030400041018280411137150E0006C6970000002D
:10305000E78020FCB7370040130770F82381E700B2
:103060000D47A381E70013070004A380E70005478D
:103070002387E700B2404101828037370040834711
:1030800027001A0593F7F703C98F93F7F70F23016A
:10309000F7008280B737004003C7170019C9D98DE0
:1030A000A380B70003C70700136787002380E700EA
:1030B000828093C5F5FFF98DA380B7008280AE872B
:1030C0002A87B736004021463738004089E7170382
:1030D00000006700E3F383C8B600E30916FF0507A5
:1030E0008348F7FFFD17C20723041801C183F9BF06
:1030F000411122C406C62A8497000000E780E0E35D
:103100002947B307E502B2408D83B3D78702224433
:103110009507B3D7E70237370040C207C1832316AC
:10312000F74041018280716541111305052006C6F3
:1031300097000000E78000FCB7370040130770F8E5
:103140002381E7400D47A381E74013070004A380D4
:10315000E74005472387E740B24041018280CC41E8
:10316000411106C6328503C6150083C50500220637
:103170004D8E42068D654186138875A2630C06113B
:10318000634BC804138845A26300060D634AC80058
:10319000938535A26301B6082390060029464DA009
:1031A000138855A26305060D938565A2E316B6FE46
:1031B0008D451D4663E6E5081146198E63F3C70089
:1031C0003E86B7E704002390C600FC4797B5010090
:1031D0009385C5F89DA0138895A263030611634EDD
:1031E000060D1388A5A263000613938505A5E315B4
:1031F000B6FA99451D4663E5E504198E63F3C700E9
:103200003E86B7E704002390C600FC4797050020E0
:10321000938505E81DA09D451D4663E3E502214613
:10322000198E63F3C7003E86B7E70400FC4723907E
:10323000C600970500209385E544BA95829701461C
:10324000B240328541018280AD451D46E3EAE5FE8C
:103250003146198E63F3C7003E86B7E7040023901A
:10326000C600FC4797B501009385C5F1F9B7B14594
:103270001D46E3E7E5FC3546198E63F3C7003E863D
:10328000B7E704002390C600FC4797B5010093857B
:1032900065F065B78D451D46E3E4E5FA1146198EE4
:1032A00063F3C7003E86B7E704002390C600FC47DF
:1032B00097B50100938545EB49B78D451D46E3E180
:1032C000E5F81146198E63F3C7003E86B7E70400A0
:1032D0002390C600FC4797B50100938565EDB1BF0B
:1032E000A5451D46E3EEE5F42946198E63F3C700B4
:1032F0003E86B7E704002390C600FC4797B501005F
:10330000938545E71DBFB5451D46E3EBE5F239461C
:10331000198E63F3C7003E86B7E704002390C6000A
:10332000FC4797B50100938565E201BFB7E704004C
:1033300003A3071397060020938686D44146A5452C
:10334000170500201305C5CA02832D455DE703C597
:1033500005000947631FE50803A84500411106C69B
:103360000347180032850346080022074168518F41
:10337000930828FE6307170563E9E800051863034F
:10338000070323900600294591A8130648FE630A07
:10339000C7041518E31707FF15463E87637BF60041
:1033A000154701A8130600023E876374F600130751
:1033B0000002B7E704002390E600FC47131607015C
:1033C00011A83E8691C30546B7E70400FC47239049
:1033D000C6004206CC45418282970145B240410178
:1033E0008280130600083E87E375F6FC1307000889
:1033F000C9B723900600054582808280416779170E
:103400006304E504411122C406C685472A84639FEC
:10341000F500B7E7040022852244B24003A38713D6
:1034200097050020938545404101028389476399B0
:10343000F500B7E7040083A7070B8545829771D98C
:10344000B2402244410182808280797126D252CCDE
:10345000AE842A8A97B50100938585D717B50100F8
:10346000130585D906D63AC622D44AD03684328985
:103470004ECE97900100E780A07BA28517B5010092
:10348000130585D897900100E780807A29459790A9
:103490000100E780C07E83C7840093F70702F9E349
:1034A00083C904008947054532476396F908D4402B
:1034B00083C7160083C60600A207D58FC166138690
:1034C00016FE638CC7028D16638FD7068D669386B2
:1034D000269029456391D706B7E70400A2862254B7
:1034E00003A34714B250F2494A86A6850259925462
:1034F0005285624A8547456102832D450DEF93074A
:103500000002354563E98702B7E70400FC47C84479
:1035100013060002CA858297814997070020938786
:1035200067319C43014581CB9C4391C74E852286E0
:10353000CA8582970145B250225492540259F249E9
:10354000624A456182802D457DF79307700F3545AE
:10355000E3E387FEB7E70400FC47C8442286CA8538
:10356000829765BF2145C1BF411122C437E40400E1
:103570008327841326C2AA84416506C697050020C6
:103580009385852A7D1582978327C40A1705000035
:10359000130505E78588829795C003230413224409
:1035A000B240924497060020938606C04146C54526
:1035B00017050020130545AE41010283B2402244A5
:1035C000924401454101828019C59707002023A339
:1035D000A72601458280454582801147636AA70A74
:1035E00097B60100938686BD0A05369518414111AC
:1035F00006C63697AE87B28502871307000261457B
:10360000639DE700B7E70400FC47130600021705B7
:1036100000201305A50782970145B2404101828031
:1036200005476145E39BE7FEB7E70400FC47054615
:103630001705002013058507F9BF1307700F6145B3
:10364000E39DE7FCB7E70400FC471306700F17057E
:1036500000201305E505C1B7130700086145E39E87
:10366000E7FAB7E70400FC47130600081705002037
:10367000130585134DB715476145E390E7FAB7E7A2
:103680000400FC471546170500201305251A61B7ED
:1036900009458280411126C2B7E4040083A7C41300
:1036A00022C44AC006C62E84970500209385C517FC
:1036B0002A898297058905C5970700209387C79DAA
:1036C00083D7A70BA28503A3440D2310F400224443
:1036D000B24092444A850249014641010283B24008
:1036E00022449244024949454101828097070020C3
:1036F000238407149707002023A20714B71700405C
:1037000003A7070CB706C0FFFD16758F23A0E70CB3
:1037100003A7070DB7064000558F23A8E70C03A7A2
:10372000070C3D9B23A0E70C03A7070D13670701B8
:1037300023A8E70C8280B717004003A5470C83A796
:10374000470C598113451500C18B058999E3136511
:1037500025009707002083C7270E6380A7029707DD
:103760000020238BA70C11C9970700209387070D12
:1037700003A307006303030002838280114517F34C
:10378000FFFF670063C8411193962500AA852D4568
:1037900006C697F0FF1FE780C004B2400145410113
:1037A0008280011122CC06CE3714004026CA4AC8B6
:1037B0004EC652C483447405034AB4058349840544
:1037C0000349940597F0FFFFE780E09E8347A40537
:1037D00093F4F40F137AFA0F93E71700230DF40410
:1037E00093F9F90F1379F90FB717004003C7A7052D
:1037F000058B6DFF03D5C705A38D4705238C3705C2
:10380000A38C2705A38B9704F2406244D24442491B
:10381000B249224A0561828041119397050122C471
:1038200006C626C2C1872E8463DC0700B7E4040005
:10383000FC54829719C1BC5482972165218D15A82B
:1038400093F7150013C515008DE793F725009DC765
:1038500097000000E78060EEB7E70400BC4F130656
:10386000000A8945170500200345C50D82971345B9
:103870002400B24022449244410182809397250162
:1038800063D80702B7E4040083A7C41E8297970099
:103890000000E780E0EEBC4C375607001306063008
:1038A0008965170500200345E5098297096579B701
:1038B000939715010145E3DE07FA17B501001305DB
:1038C000A59C97900100E780804EB7E70400BC4FAD
:1038D000130600649165170500200345A50682972D
:1038E0001165A9BF011126CA9314450152C4D180A4
:1038F000139A250006CE22CC4AC84EC6338744010F
:103900009307001063E5E7067D74698C17090020B2
:10391000130909F3B289930600104A86A2852D4542
:1039200097F0FF1FE780E0EBB7E70400FC47CE8588
:10393000330599005286B7E400E0B709400082974A
:1039400023A034190100010085660146A2852545A2
:1039500097F0FF1FE780E0E8930600104A86A285F3
:10396000294597F0FF1FE780C0E723A03411F240FC
:103970006244D2444249B249224A05618280B7F783
:10398000070003C70701411106C622C426C24AC068
:10399000A547631DF70097000000E780E0F4B24000
:1039A000224492440249014541018280139425003A
:1039B000AA843289A286AA850146254597F0FF1F71
:1039C000E78020E2A2864A86A685294597F0FF1F58
:1039D000E78020E1E9B71D71A2CC37E404005C5C0C
:1039E000485886CE494697B50100938565858297EC
:1039F00011E917B501001305E58597900100E780EF
:103A0000003B01A0B7F600E0795798CAFD57DCCA21
:103A10000567B7E700E023A0E7101306F00290C2A5
:103A200023A0E718010001003707002018471306FC
:103A3000000481459706002023A4E6F04157A38A9D
:103A4000E7403C4408088297971700209387878CAB
:103A50003EC8856713870740231AE1001D673ACCEB
:103A600037070105130707103ACE938757D113077D
:103A7000B00F2310E1022312F102054797F7FFFF71
:103A80009387A7522301E1023ED8170700001307CE
:103A9000C7CF97070000938707D1B7F50700BAC2D1
:103AA0003EDC170700001307C7ED97070000938758
:103AB00027CD81463000E1051945BAC43EDE97F0B6
:103AC000FF1FE78000D218088147994630003E96D4
:103AD0000346060085070507A30BC700E398D7FE3A
:103AE000C24791C70357410185676373F70001A07F
:103AF000B7E7040083A7470A08088297AA8511C977
:103B000017A501001305457697900100E780401244
:103B100001A0F640664425618280411126C2B7E4C7
:103B2000040083A7040806C622C417050000130575
:103B3000E5CE8297170400201304C4E02300A400FC
:103B400097000000E780800297000000E78040BAFD
:103B500003450400224403A38405B24092441306A3
:103B60000032896541010283797106D622D4130798
:103B70008008F337078093F787083EC201000100F1
:103B8000B7170040930570052380B704130680FA29
:103B90002380C7040100010083C6F70293F6A60F35
:103BA000A387D702238007049246F3A6068001006C
:103BB000010073370780137787083AC401000100BA
:103BC0002380B7042380C7040100010003C7F70264
:103BD00013672700A387E70223800704A247F3A700
:103BE000078001000100054597E0FFFFE780E05FE7
:103BF00097000000E780C0B801478146814705462D
:103C000085451305407E97E0FFFFE780E06237E4DB
:103C100004003C446800514681458297B707C0A81C
:103C20003EC8B787E803938707D03ECA97E7FF1FD0
:103C30009387E7783EC67C5868008297B25022543A
:103C400045618280411197B50100938525CA17A56A
:103C500001001305655A06C697900100E78040FDF4
:103C600017B50100130545E197900100E78040FC7E
:103C7000B2402945410117930100670043004111FB
:103C800097B501009385C5C717A501001305C55653
:103C900006C697900100E780A0F917B5010013054B
:103CA00065DC97900100E780A0F8B240294541010A
:103CB000179301006700A3FC411122C406C6834785
:103CC00005002A849DC797B50100938525C917A5CE
:103CD00001001305655297900100E78060F54C40A4
:103CE00017B50100130585E797900100E78040F4C0
:103CF0003DA058410DEF97B50100938525C617A546
:103D000001001305654F97900100E78060F217B539
:103D10000100130525E697900100E78060F1224439
:103D2000B2402945410117930100670043F5A1679F
:103D30009386D7036313D70297B50100938505C215
:103D400017A501001305454B97900100E78040EE51
:103D500017B50100130505E37DBFED0797B5010019
:103D60009385C5BF17A5010013050549631BF7001F
:103D700097900100E780C0EB17B501001305C5E17E
:103D800059BF97900100E780A0EA4C4017B50100A9
:103D9000130585E291BF411197B50100938585B761
:103DA00017A501001305454506C697900100E78059
:103DB00020E8B2402945410117930100670023EC38
:103DC000797122D426D24AD02E842A898145B284A0
:103DD0004800714606D697E0FFFFE780403397F72B
:103DE000FF1F9387675DDC4783D7070023142101FA
:103DF0002313F10097500000E78040E08547A305BA
:103E0000F1009307401F3EC6FD572305A100230A7A
:103E1000F10097500000E780A0F22686A2854800B6
:103E200097500000E78060E0B2502254925402594B
:103E300045618280972700202391079E97270020C5
:103E4000238A078CB7E70400BC47411106C64146E8
:103E50008145170500201305653A82971707002052
:103E60000347C73B9307F00A6315F7029307F0F87F
:103E70008945170500201305653A17070020230F11
:103E8000F73897070020A38B073897600000E7807A
:103E9000409997600000E780A0C481453705040081
:103EA0009707002023AA073497070020239407349C
:103EB0009707002023810734970700202390072CC1
:103EC00097070020239E0728970700202393073297
:103ED00097070020239C073297300000E780402599
:103EE000014597600000E780C09C97B5010093856D
:103EF000E5A417A501001305253097900100E78080
:103F000020D317B50100130565D197900100E78014
:103F100020D2B2402945410117930100670023D602
:103F2000411122C497B50100938585A42A8417A561
:103F300001001305652C06C697900100E78040CF6D
:103F40004C4017B501001305E5BE97900100E780CE
:103F500020CE294597900100E78060D203470400F6
:103F60009307F00F631FF70297B50100938545A0F3
:103F700017A501001305452897900100E78040CB65
:103F80004C4017B501001305E5BB97900100E78091
:103F900020CA2244B240294541011793010067001D
:103FA00003CEB240224441018280411122C426C284
:103FB0002A84AE8417A501001305052497B50100D6
:103FC0009385C59606C697900100E78060C617B531
:103FD0000100130525C397900100E78060C52945BE
:103FE00097900100E780A0C997B5010093850594DB
:103FF000970700202394871617A501001305C51FF6
:1040000005449707002023999714970700202396CB
:104010008714972700202392978097900100E780CC
:1040200020C19715002083D5457F17B501001305E2
:10403000E5BD97900100E780A0BF2945979001005A
:10404000E780E0C3971700202386876C97F7FF1F50
:1040500093878736DC4703D70700C167FD176312D4
:10406000F7022244B7E70400B240924403A3870555
:10407000170500200345858D1306000A854541017B
:104080000283B2402244924441018280B1C1411175
:1040900022C417A50100130525162E8497B501002B
:1040A0009385058806C697900100E78060B8A285D1
:1040B00017B50100130545B497900100E78040B79C
:1040C0002244B2402945410117930100670023BBF8
:1040D0008280011122CC06CE26CA4AC84EC693F76A
:1040E00015002E84638D0710814617F6FF1F1306F7
:1040F000E6298545170500200355450697C00000B1
:10410000E78000FE15C997B501009385E58317A5E3
:1041100001001305650E97900100E78060B117A5B7
:1041200001001305252597900100E78060B029451F
:1041300097900100E780A0B497B501009385C580F2
:1041400017A501001305450B97900100E78040AECD
:1041500017A501001305452397900100E78040ADA6
:10416000294597900100E78080B197F7FF1F93875B
:10417000A724DC47054797A501009385E57C23909C
:10418000E70017A501001305250797900100E780B8
:1041900020AA17A501001305652097900100E7806C
:1041A00020A9294597900100E78060AD930710F89A
:1041B000170700202304F7069707002083D7C7F9C5
:1041C00017070020A30CF7041705002013050505A9
:1041D000A1839145170700202303F70497070020C8
:1041E000A38F070297500000E780A06313451400D7
:1041F000F2406244D2444249B2490561828093F759
:1042000005108DC7054597500000E780806A171597
:1042100000200355856097500000E780E035972027
:104220000000E780E00613450410D9B793F7250096
:10423000E9CF170700200357E7FB69C7AD64B7193B
:1042400000409384A4AA23A0990097060020938697
:10425000A6FA944297B701009387479E170600205D
:10426000034666F9814517050020130525F9977067
:104270000000E780400623A0990097F7FF1F2391D5
:10428000A7042A8941C197A501009385A57217A5A6
:104290000100130565F697900100E7806099CA85D3
:1042A00017A501001305051197900100E7804098BC
:1042B000294597900100E780809C97070020239B69
:1042C00007F2930710F8170700202309F7F4970760
:1042D000002083D767E817070020A301F7F4A18324
:1042E00017070020230DF7F291458D471705002091
:1042F0001305C5F217070020A303F7F2975000003B
:10430000E780205213452400E5B593F74500D1C35B
:1043100097A501009385056A17A501001305C5ED52
:1043200097900100E780C09017A501001305450A8A
:1043300097900100E780C08F294597900100E780A2
:104340000094930720F8170700202309F7EC97073C
:10435000002083D7A7E217070020A301F7ECA18371
:1043600017070020230DF7EA854717070020A30849
:10437000F7EA97500000E780A09C1705002013057E
:10438000E5E9914597500000E780A04913454400B6
:1043900085B593F78500A9C797A501009385856129
:1043A00017A50100130545E597900100E7804088B7
:1043B00017A501001305050397900100E7804087CA
:1043C000294597900100E780808B97070020239371
:1043D00007E297700000E780E0FF1345840009BD05
:1043E00093F70501D1C3854517050020035505D96D
:1043F00097400100E780C0D897A501009385855BB1
:1044000017A50100130545DF97900100E780408262
:1044100017A50100130545FE97900100E780408134
:10442000294597900100E7808085930730F81707AA
:1044300000202305F7DE9707002083D727D417072E
:104440000020A30DF7DC17050020130525DDA1834F
:104450008D45170700202304F7DC97500000E78004
:10446000403C1345040169B393F70502D1C797A5F2
:1044700001009385255417A501001305E5D7978002
:104480000100E780E07A17A50100130525F9978060
:104490000100E780E079294597800100E780207ED0
:1044A000930740F817070020230AF7D69707002044
:1044B00083D707CB17070020A302F7D6A1831707DE
:1044C0000020230EF7D4854717070020A309F7D44F
:1044D00097070020239607C897500000E780408682
:1044E00017050020130585D3914597500000E780FC
:1044F000403313450402EDB993F70504FDC397A5B6
:1045000001009385254B17A501001305E5CE978083
:104510000100E780E07117A501001305A5F1978060
:104520000100E780E070294597800100E780207551
:104530009707002083C787CE1307700A6386E706B4
:104540001307800A638CE7081307600A6393E70484
:10455000930760F8170700202302F7CC9707002085
:1045600083D727C917070020A30AF7CAA183170713
:1045700000202306F7CA854717070020A305F7CABE
:10458000B14517050020130565C997500000E78065
:10459000402997400000E780A07A1345040497075C
:1045A0000020239807C4A9B1930770F817070020CB
:1045B0002306F7C69707002083D7A7C31707002055
:1045C000A30EF7C4A18317070020230AF7C4854769
:1045D00017070020A306F7C4994565B7930780F82D
:1045E000F1B793F705080145E38407C097A50100DB
:1045F0009385453C17A50100130505C09780010070
:10460000E780006317A50100130545E497800100CA
:10461000E7800062294597800100E78040669307A4
:10462000A0F817070020230BF7BE9707002083D7B9
:10463000E7BD17070020A303F7BEA18317070020DB
:10464000230FF7BC854717070020A30AF7BC97077D
:104650000020239D07BA97400000E780606E170591
:1046600000201305A5BB914597500000E780601B13
:1046700013450408B5BE011122CC37E404005C5C8C
:1046800006CE354697A501009385454017B5010034
:104690001305C50A829711E917A50100130585BB0B
:1046A00097800100E780A07001A097F7FF1F938714
:1046B000A72A3EC4B7F50700856793870780814620
:1046C00017F6FF1F1306C628E10519453EC697E0F9
:1046D000FF1FE78000117C44194697F5FF1F938563
:1046E0002527170500201305A5A98297340017F682
:1046F000FF1F1306E62597B501009385A58617B51C
:1047000001001305A58797700000E780C0912A84F7
:104710001DCD97A501009385E52817A50100130578
:10472000A5AD97800100E780A050A28517A50100E4
:104730001305C53697800100E780804F2945978093
:104740000100E780C053F24062440561828097E037
:104750000000E78020F417A501001305252B9760C2
:104760000000E780008B97A00000E780604897403A
:104770000100E780A0D317F5FF1F130565C0974020
:104780000100E78040BC17A50100130525299740CB
:104790000100E78020D42A8497600000E78000EDC4
:1047A00097100100E780C08497600100E780A04473
:1047B00097700000E780804497600000E780006306
:1047C00097A501009385051E17A501001305C5A235
:1047D00019C897800100E780A045A28517A50100B0
:1047E0001305052E81BF97800100E780604417A55F
:1047F00001001305252F97800100E78060432945BC
:1048000097800100E780A04797F00000E780C04153
:1048100055C985453705040097300000E780409171
:1048200097A501009385051817A501001305C59CE0
:1048300097800100E780C03F17A501001305052CF4
:1048400097800100E780C03E294597800100E780FE
:10485000004397F7FF1F9387A7A583D70700171774
:104860000020231CF7FA8547171700202304F7EAD6
:1048700097200000E78080B597200000E78040A1E6
:1048800017150020035565F997500000E780C0CE4A
:10489000054597500000E780C00197A5010093856A
:1048A000651017A501001305259597800100E78085
:1048B000203817A501001305A52697800100E78081
:1048C0002037ADBD97A501009385C50D17A5010043
:1048D0001305859297800100E780803517A50100B8
:1048E0001305C53397800100E78080342945978000
:1048F0000100E780C038014569BF411122C437E497
:1049000004008327041A06C6829797500000E780A8
:1049100060CA8327040817F5FFFF1305C57B82973C
:1049200097F7FF1F2384A70217F5FF1F1305C5A8DC
:1049300097400000E78060732244B24041011703B2
:104940000000670083D3B7E70400FC471171A2DDC4
:10495000CAD986DFA6DBCED72E8432892E86AA85D9
:10496000170500201305858B829717070020130772
:10497000E78A83470700930680029387E70793F748
:10498000F70FE3ECF610BA898A0717A7010013079F
:10499000E78FBA979C43BA9782878D4797A5010006
:1049A0009385850217A5010013050585630FF400A3
:1049B00097800100E780C02717A50100130585BF78
:1049C00097800100E780C026BDA497800100E780A2
:1049D000202617A50100130565BF97800100E78019
:1049E0002025294597800100E7806029930720F85A
:1049F000114697050020938565824A851707002098
:104A0000230EF78097070020A38B078097F0FFFF06
:104A1000E780403B2A841DC997A501009385C5FA0C
:104A2000179501001305457D97800100E780402020
:104A3000A28517A50100130525BD97800100E78019
:104A4000201F294597800100E780602397A501007A
:104A5000938585F7179501001305057A9780010066
:104A6000E780001D17A50100130545BB97800100D5
:104A7000E780001C294597800100E78040204165C0
:104A8000930730FA054697F5FF1F938525797D1525
:104A900017F7FF1F2304F77897F0FFFFE7808032B6
:104AA0002A841DC997A50100938505F21795010079
:104AB0001305857497800100E7808017A28517A5EC
:104AC0000100130565B497800100E7806016294551
:104AD00097800100E780A01AB7E70400BC4F056685
:104AE000130606C8A14517F5FF1F034525E6829763
:104AF000FE506E54DE544E59BE591161828091476A
:104B00006303F40297A50100938505EC1795010056
:104B10001305856E97800100E780801117A50100BD
:104B2000130505B371BDB7E70400FC4F914517F5B8
:104B3000FF1F0345A5E1829797A501009385C5E86E
:104B4000179501001305456B97800100E780400E23
:104B500017A50100130585B197800100E780400D7E
:104B6000294597800100E780801197400000E78089
:104B7000201D914535A485476303F40297A50100E4
:104B8000938585E41795010013050567978001005B
:104B9000E780000A17A501001305C5AE15B597F704
:104BA000FF1F239D275DB7E704000566BC4F130672
:104BB00006C8C1450DBF8D476303F40297A50100E8
:104BC000938585E017950100130505639780010023
:104BD000E780000617A50100130585ACD5B3930740
:104BE00040F8114697F5FF1F938545634A8517F7EF
:104BF000FF1F2305F76297F7FF1FA382076297F055
:104C0000FFFFE780201C2A84E30405EE97A501003E
:104C1000938585DB179501001305055E97800100DC
:104C2000E7800001A28517A501001305E59D978087
:104C30000100E780E0FF294597800100E78020041C
:104C400045BD9147E31CF4F6B7E70400FC4F93051C
:104C5000000217F5FF1F034565CF829797A5010056
:104C6000938585D617950100130505599780010096
:104C7000E78000FC17A50100130505A4F1BD8947D5
:104C800063E3870297A50100938505D4179501007A
:104C90001305855697800100E78080F917A501006C
:104CA0001305C5A231BB97F4FF1F83C4445797F780
:104CB000FF1F83C7B75697A501009385E5D0A204CF
:104CC0001795010013054553DD8C97800100E7809F
:104CD00020F6A28517A50100130585A09780010085
:104CE000E78000F5C204294597800100E78020F99C
:104CF000C1849305D4FF93960401C1824A8693F53B
:104D0000F50F17F5FF1F1305955197200000E78059
:104D1000E045E35F90DC930750F817F7FF1F230F80
:104D2000F74E83C73900228697F5FF1F9385054FFD
:104D300085074A8517F7FF1FA303F74E97F0FFFF7C
:104D4000E78040082A84E30505DA97A501009385EA
:104D5000A5C7179501001305254A97800100E78034
:104D600020EDA28517A50100130505E8C9B58947FF
:104D700063E3870297A50100938505C51795010098
:104D80001305854797800100E78080EA17A5010099
:104D90001305C59635B197400000E78060FAA285FB
:104DA00017F5FF1F1305854797500000E78060A7A0
:104DB00081B38D476303F40297A501009385C5C0B5
:104DC000179501001305454397800100E78040E6F1
:104DD00017A5010013054594E5B6B7660200014624
:104DE000B7750200054597E0FF1FE780809F930796
:104DF00060F817F7FF1F2303F74297F7FF1FA38001
:104E000007429307000617F7FF1F230BF740894758
:104E100017F7FF1FA306F74097F7FF1F23830740ED
:104E200097F7FF1FA38F073EC14717F7FF1F230BFD
:104E3000F73E930720F917F7FF1FA305F73E31460A
:104E400097F7FF1FA381A73E97F5FF1F9385053DA9
:104E50004A8597F7FF1F2388073C97F0FFFFE780FD
:104E600060F62A84E30605C897A501009385C5B5B9
:104E7000179501001305453897800100E78040DB56
:104E8000A28517A501001305A58A55B3B147630391
:104E9000F40297A50100938525B31795010013052A
:104EA000A53597800100E780A0D817A5010013055C
:104EB000E58939B6B7E70400FC4F9305000417F500
:104EC000FF1F0345A5A8829797400000E78040E7B1
:104ED000B145F9B5914763E3870297A50100938532
:104EE000A5AE179501001305253197800100E780D5
:104EF00020D417A5010013052587D9B497F4FF1F07
:104F000083C4043297F7FF1F83C77731A204DD8C77
:104F10008E04B77702006D14BE942286A68517A56D
:104F200001001305A58597800100E78060D0B7E7F1
:104F30000400FC47228697F5FF1F9385752E2800F5
:104F4000829793160401C1823000A685094597E037
:104F5000FF1FE78000892A8409C917A501001305EE
:104F6000A58397800100E78080E4930770F81946D5
:104F700097F5FF1F9385852A4A8517F7FF1F230F93
:104F8000F72897F7FF1FA38D872897F0FFFFE7808B
:104F900060E32A84E30E05B497A501009385C5A2BA
:104FA000179501001305452597800100E78040C84B
:104FB000A285179501001305257F95B99947630BC5
:104FC000F41297A50100938525A0179501001305FC
:104FD000A52297800100E780A0C517950100130561
:104FE000257EF9BA914763E3870297A5010093856F
:104FF000A59D179501001305252097800100E780E6
:1050000020C3179501001305257D5DBA97F4FF1F96
:1050100083C4042197F7FF1F83C77720A204DD8C88
:105020008E04B77702006D14BE942286A68517956C
:1050300001001305A57B97800100E78060BFB7E7FB
:105040000400FC47228697F5FF1F9385751D2800F5
:10505000829793160401C1823000A6850D4597D032
:10506000FF1FE78000782A8409C9179501001305FE
:10507000A57997800100E78080D3930780F81946CF
:1050800097F5FF1F938585194A8517F7FF1F23079B
:10509000F71897F7FF1FA385871897F0FFFFE780A2
:1050A00060D22A84E30605A497A501009385C591E3
:1050B000179501001305451497800100E78040B75C
:1050C000A285179501001305657595B69947630389
:1050D000F40297A501009385258F1795010013050C
:1050E000A51197800100E780A0B417950100130572
:1050F0006574F9B0B7E70400FC4F9305000417F599
:10510000FF1F0345A584829797400000E78040C3B6
:10511000994579B18D476303F40297A50100938502
:10512000A58A179501001305250D97800100E780DA
:1051300020B0179501001305657159B0179501004E
:105140001305C57197800100E78060C61305C01282
:1051500097D0FF1FE780E01E014597E0FFFFE78043
:10516000C0E10D4597100000E780E09F294597D0EA
:10517000FF1FE780001D97D0FF1FE780600D8DBAED
:1051800099476303F40297A501009385E58317957A
:1051900001001305650697800100E78060A9179557
:1051A00001001305656C29B817F7FF1F0347570760
:1051B00097F7FF1F83C7C70622075D8F9166BA96D0
:1051C000C2061166C1821306F6EF8D476365D602EB
:1051D00097E7FF1F9387471E9C4B17F6FF1F034659
:1051E00016049386C7002DC203D6070069CA890733
:1051F000E39CD7FE89471307A0F8114697F5FF1FD8
:105200009385C5014A8597F6FF1F2389E60017F7A6
:10521000FF1FA306F70097F0FFFFE780A0BA2A84DC
:10522000E308058C979501009385057A1795010091
:10523000130585FC97800100E780809FA285179564
:1052400001001305A563E5B203D60700630EE60A65
:105250008907E39BF6FE8D4779BF91476304F4020B
:105260009795010093854576179501001305C5F8BC
:1052700097800100E780C09B1795010013058561A9
:105280006FF00FF4B7E70400FC4F9305000817E533
:10529000FF1F0345A56B8297C9B8979501009385B9
:1052A000A57217950100130525F597800100E78089
:1052B0002098179501001305655F6FF06FF023903C
:1052C000E70017E5FF1F1305250F97100100E78082
:1052D000A0C2979501009385256F179501001305CE
:1052E000A5F197800100E780A094179501001305B0
:1052F000E55C97800100E780A09329459780010035
:10530000E780E0978147C5BD2390070017E5FF1FA1
:105310001305850A97100100E78000BE97950100EC
:105320009385856A17950100130505ED97800100A7
:10533000E7800090179501001305C5595DBF411125
:1053400022C406C6834705002A849DC7979501009D
:105350009385456317950100130505EA97800100C1
:10536000E780008D4C4017A501001305258E97801E
:105370000100E780E08BE1A05841B707CF00938799
:10538000777D631DF706979501009385A55F1795B7
:105390000100130565E697800100E78060891C44E1
:1053A0008356E4008355C40003C6070017A5010017
:1053B0001305458B97800100E780808729459780FA
:1053C0000100E780C08B0357E4009707002083D7D4
:1053D000C7446309F7008355C400084497E0FFFF02
:1053E000E78020CE0356E4008355C40008442244DD
:1053F000B240410117F3FFFF67002355B707CC0008
:105400009387777D6315F7049795010093858557FA
:1054100017950100130545DE97800100E780408164
:105420001C448356E4008355C40003C6070017A537
:1054300001001305258397700100E780607F2244F7
:10544000B240294541011783010067004383B70734
:10545000CE009387777D6304F702979501009385CB
:10546000655217950100130525D997700100E78053
:10547000207C4C401795010013050574CDBDB2404A
:10548000224441018280B7E70400FC4741112E8687
:1054900006C622C426C24AC02E842A89AA8517F5C8
:1054A000FF1F1305A5D78297979501009385855314
:1054B00017950100130545D497700100E7804077E8
:1054C00097F5FF1F83C585D517950100130585F94D
:1054D00097700100E780C075294597700100E7804B
:1054E000007A97F4FF1F938464D383C70400414775
:1054F0009387070693F7F70F636EF75A1797010024
:10550000130707E38A07BA979C43BA9782879D4798
:105510006307F402979501009385C54C1795010028
:10552000130585CD97700100E78080701795010005
:105530001305C5F397700100E780806F8DA497F77E
:10554000FF1F83C7B7CDDDCB17F7FF1F034737CD4D
:1055500097F7FF1F83C7A7CC22075D8F97F7FF1F21
:1055600083C707CCC2075D8F97F7FF1F83C757CB51
:10557000E207D98F17F7FF1F2320F7C883C76400FE
:105580009795010093850546179501001305C5C63B
:1055900017F7FF1F2301F7C697700100E7804069E6
:1055A00097F7FF1F938747C58C4317F6FF1F0346E6
:1055B00086C417950100130525ED97700100E7805B
:1055C0002067294597700100E780606B97F7FF1F00
:1055D000A38607C42244B24092440249930700F8CC
:1055E00017F7FF1F230CF7C29D4517F5FF1F130583
:1055F000E5C24101174300006700A3229760000045
:10560000E780C0EC97F7FF1F238BA7C09357850057
:1056100017F7FF1FA305F7C0935705012A8417F753
:10562000FF1F230FF7BE93578501014517F7FF1F93
:10563000A308F7BE97600000E78000EA97F7FF1F16
:105640002381A7BE979501009385C5391795010061
:10565000130585BA97700100E780805D17F6FF1F7C
:10566000034626BCA28517950100130565E3B1B773
:10567000CD476303F402979501009385A5361795EE
:105680000100130565B797700100E780605A179510
:105690000100130565E279BD37E404007C4441460E
:1056A00097F5FF1F938595B717F5FF1F130505B5F0
:1056B000829797F7FF1F83C787B717F7FF1F034727
:1056C000F7B6A20703238405D98F17F7FF1F23130B
:1056D000F7B21306000A89452244B24092440249B7
:1056E00017E5FF1F03458526410102838D476303AC
:1056F000F402979501009385E52E17950100130597
:10570000A5AF97700100E780A0521795010013051F
:1057100065EA0DB517F4FF1F034464B097F7FF1F48
:1057200083C7D7AF979501009385C52B22041795A2
:105730000100130565AC5D8C97700100E780404F58
:10574000A285179501001305A5D897700100E78081
:10575000204E294597700100E78060520D4697F56D
:10576000FF1F9385A5AB228597E0FFFFE78080654B
:10577000AA8421C1979501009385C526179501003C
:10578000130585A797700100E780804AA6851795C5
:105790000100130525D597700100E7806049224478
:1057A000B240924402492945410117730100670044
:1057B000034D97F7FF1F2393879CB7E704001166FB
:1057C00003A38705130606E8914539B78D476303A0
:1057D000F402979501009385E520179501001305C4
:1057E000A5A197700100E780A0441795010013055B
:1057F00025EB89B317F4FF1F034464A297F7FF1F3B
:1058000083C7D7A1979501009385C51D22041795DD
:1058100001001305659E5D8C97700100E780404193
:10582000A28517950100130525CD97700100E7802B
:105830002040294597700100E78060440D4697F5A8
:10584000FF1F9385A59D228597E0FFFFE780805786
:10585000AA841DC1979501009385C518179501006D
:105860001305859997700100E780803CA685179500
:1058700001001305A5C905B797F7FF1F2392878E6F
:10588000B7E70400116603A38705130606E893052E
:10589000000299B5894763E38702979501009385D4
:1058A0006514179501001305259597700100E78091
:1058B000203817950100130565E1ADB997F4FF1F76
:1058C00083C4E49597F7FF1F83C757959795010009
:1058D00093854511A204179501001305E591DD8C10
:1058E00097700100E780C034A68517950100130565
:1058F00065C397700100E780A033294597700100C8
:10590000E780E037228697F5FF1F9385259126854E
:1059100097E0FFFFE780004B2A84630E051A9795F6
:1059200001009385250C179501001305E58C9770F0
:105930000100E780E02FA285179501001305C5BF80
:1059400099BD854763F98718834519002244B24001
:1059500092440249B335B00097F7FF1F238AB782FC
:1059600017950100130585BE4101177301006700FB
:10597000232CA2852244B24092444A850249410127
:10598000170300006700632499476303F4029795A7
:10599000010093852505179501001305E58597708E
:1059A0000100E780E028179501001305E5EB59B6E3
:1059B00017F4FF1F0344A48697F7FF1F83C71786BA
:1059C00097950100938505022204179501001305A0
:1059D000A5825D8C97700100E7808025A2851795D0
:1059E0000100130525B897700100E7806024294560
:1059F00097700100E780A028194697F5FF1F93854F
:105A0000E581228597E0FFFFE780C03BAA841DC1A6
:105A100097950100938505FD178501001305C57D48
:105A200097700100E780C020A68517950100130537
:105A300065B495B397E7FF1F239A877CB7E7040007
:105A4000116603A38705130606E89305000869B1EC
:105A50008547979501009385E5F8178501001305A3
:105A6000A579630BF40097700100E780601C17951F
:105A70000100130565B17DBC97700100E780401BF4
:105A8000179501001305C5B197700100E780401A12
:105A9000294597700100E780801E2244B24092445D
:105AA000024997E7FF1F239707744101176300001E
:105AB00067004392979501009385C5F21785010011
:105AC0001305857397700100E78080161795010014
:105AD0001305C5DD85B4B240224492440249410118
:105AE0008280411106C622C497E0FFFFE780802D27
:105AF00021CD97E7FF1F83D7C76985072A8417E75A
:105B0000FF1F2318F76897950100938525EF97E706
:105B1000FF1F2391A768178501001305E56D977096
:105B20000100E780E010A285179501001305C50B61
:105B300097700100E780C00F2244B240294541011F
:105B4000177301006700A31397E7FF1F83D7A764AC
:105B5000B2402244850717E7FF1F231EF762410169
:105B60008280411122C491462A8417E6FF1F130642
:105B7000E6789D652D4506C697D0FF1FE78060C675
:105B8000B7F7070003C70701A5476313F70001A094
:105B90009306001001469D65254597D0FF1FE780BD
:105BA00040C497E7FF1F238B87742244B24091467D
:105BB00017E6FF1F130686749D652945410117D31B
:105BC000FF1F670003C21171CED7B7E9040083A796
:105BD000C904CAD917E9FF1F13094964A2DD2E863B
:105BE00086DFA6DB2E84AA854A85829797E7FF1F6A
:105BF00083C7C7621307700A6385E710636DF700F8
:105C00001307600A6385E704FE506E54DE544E5954
:105C1000BE59116182801307800A6385E716130756
:105C2000900AE393E7FE8D476306F41C9795010005
:105C30009385C50E178501001305055C977001005B
:105C4000E78000FF179501001305850A25A08D4701
:105C5000630CF402979501009385450C17850100AC
:105C60001305855997700100E78080FC17950100A6
:105C70001305450197700100E78080FB2945977067
:105C80000100E780C0FF49B785471795010013055C
:105C9000250117E7FF1F230DF74E97700100E780DE
:105CA0000011B7750200B76602000146054597D09E
:105CB000FF1FE78000B3930760F817E7FF1F230F6C
:105CC000F75497E7FF1FA38C07549307002617E7A5
:105CD000FF1F2327F754E5779387072117E7FF1F57
:105CE0002312F754B14597E7FF1F238E075297E71A
:105CF000FF1FA38AA7524A8597000000E780E0169D
:105D000021B7914763E387029795010093850501C9
:105D1000178501001305454E97700100E78040F19B
:105D2000179501001305C5F9B1B797E4FF1F83C4A8
:105D3000244F97E7FF1F83C7974EA204DD8C83A7EC
:105D4000C9046D14228697E5FF1F9385754D2800C1
:105D500082978E0493160401B7750200C182300049
:105D6000A695094597D0FF1FE780A0A7930770F875
:105D700017E7FF1F2304F74A994597E7FF1FA38101
:105D8000A74A95BF914763E38702979501009385E2
:105D9000E5F8178501001305254697700100E78097
:105DA00020E917950100130525F3E9B597E4FF1FD6
:105DB00083C4044797E7FF1F83C77746A204DD8C9F
:105DC00083A7C9046D14228697E5FF1F9385554567
:105DD000280082978E0493160401B7750200C182D1
:105DE0003000A6950D4597D0FF1FE780809F930751
:105DF00080F8BDBF179501001305C5F0977001002D
:105E0000E780E0FA930790F82304F1008347190034
:105E10008D452800A304F100834729002305F100E4
:105E200097000000E78060041305C01297C0FF1FB1
:105E3000E7802051014597D0FFFFE78000140D4512
:105E400097000000E78020D2294597C0FF1FE78018
:105E5000404F97C0FF1FE780A03F7DB397E7FF1F2C
:105E600023A6A74A828097E7FF1F9387274A03A3A9
:105E70000700630303000283174300006700639A6F
:105E800041114AC09706002083D62699328917D639
:105E9000FF1F0356865422C426C206C62A84AE8437
:105EA00097000000E780C05D35C12DC0994763FFB2
:105EB00097048347140003470400A207D98F139760
:105EC0008700A183D98FC2073167C1831307C755E4
:105ED000639EE70297D7FF1F83D72750A301F400E3
:105EE000A1832302F4009707002083D7079391C76B
:105EF000A302F400A1832303F400A68517950100F3
:105F00001305C5E597700100E78080D29707002050
:105F100083C74780A5C797D5FF1F83D5054C179525
:105F20000100130565E597700100E78060D02686C3
:105F3000A28517D5FF1F0355454A97000000E7804B
:105F400080BA6306090497F7FF1F83C7A77CA1E304
:105F500097E7FF1F83C7C73B9DCB95C897E7FF1FF8
:105F600083C707238DE722852244B2400249A685D4
:105F700092444101174300006700A38A179501006E
:105F8000130585E097700100E78060E25DBFB240D5
:105F9000224492440249410182808347550083454F
:105FA000450017950100130525DAA207DD8D17734B
:105FB00001006700E3C7179501001305E5D71773C4
:105FC00001006700C3DE8D4763FBB70A011126CAD3
:105FD00006CE22CC0344350097E4FF1F83C454331C
:105FE00097950100938505DBB337800017E7FF1F06
:105FF000A300F73209C497950100938565DA1795D8
:106000000100130565DA97700100E78060C297E729
:10601000FF1F83C7F72F6386970097000000E78074
:10602000E02E97E7FF1F83C7B72E8DC7854723064E
:10603000F100B7E7040083A74717700085451305F3
:106040005030829717950100130505D7977001000E
:10605000E780E0D59967938757EE2316F100680033
:1060600085479145A30781002307F10097000000B1
:10607000E780A0DFF2406244D244056182808280E2
:10608000894763F7B708011122CC06CE26CA83449C
:10609000250085472A84639DF404914763F5B7047E
:1060A000034545008347340022055D8D97D7FF1FC8
:1060B0002395A73297000000E78060459967938792
:1060C00067EE2314F1008347340023059100A305F4
:1060D000F10083474400954528002306F10097000E
:1060E0000000E78080D8F2406244D244056182809B
:1060F000FDF89967938767EE2314F10097D7FF1F88
:1061000083D7A72DA305F10023050100A183E1B7E3
:1061100082800111996722CCD51717F4FF1F130451
:10612000645F2314F1008347040026CA97F4FF1F1D
:106130009384A46E2305F10083D7040028009545BD
:10614000A305F100A18306CE2306F100970000000D
:10615000E780A0D103D60400834504001795010011
:10616000130505C797700100E78080ACF2406244D8
:10617000D244056182809D677971D9172316F10099
:1061800097F7FF1F83C7075906D62307F100A9C356
:10619000B7E70400FC47414697E5FF1F93850506D6
:1061A0001305F10082976800CD4597000000E78055
:1061B000C0CB97F5FF1F83C5E55517950100130563
:1061C00025C497700100E780A0A6B2504561828087
:1061D000B7E70400BC47414681451305F1008297AB
:1061E000D9B745C5411106C622C4930750FA23000A
:1061F000F5009307A005A300F50089472301F500EA
:106200009147A301F50093077003A302F50097F7E8
:10621000FF1F9387275083C70700230205002A84A6
:106220002303F50097E7FF1F9387970E83C70700A7
:10623000414697E5FF1F938565FCA303F50097F79B
:10624000FF1F83D7875D2304F500A183A304F50016
:1062500097D7FF1F83D767182305F500A183A305F0
:10626000F500B7E70400FC47310582972285F14528
:1062700097000000E780C01C230EA4002181A30E1C
:10628000A400B24022444101828082805D710A856F
:1062900086C6A2C497000000E780E0F437E404005B
:1062A0007C448A850810794682973C441305E103B3
:1062B000094681458297101093050002014597D049
:1062C000FFFFE780C031B640264461618280411102
:1062D00022C426C24AC02A84AE843289AA85856631
:1062E0000146254506C697C0FF1FE780804FA2855F
:1062F0002244B240CA862686024992442945410179
:1063000017C3FF1F6700E34D0111B7C7A55A22CC81
:106310009387C73317E4FF1F130494FF3EC48347DA
:1063200004002C002146196506CE3EC697000000E9
:10633000E78020FA8345040017950100130545BB4B
:1063400097700100E780C08EF24062440561828050
:106350000111A146300099652D4522CC06CE97C08B
:10636000FF1FE7800048A24737C4A55A1304C4336F
:1063700063958702B245179501001305A5AAB335A9
:10638000B00097E7FF1FA385B7F897700100E7807B
:10639000208AF2406244056182809165A146300006
:1063A000938505F02D4597C0FF1FE7808043A247E6
:1063B000E38287FC97E7FF1FA38C07F481451795BD
:1063C0000100130565A8D1B77971D14670009165B8
:1063D0002D4522D406D697C0FF1FE7808040B247E4
:1063E00037C4A55A1304F43563988702B7E704004D
:1063F000FC4717E5FF1F130565E041460C0882972F
:1064000017950100130545AA97700100E780209AAF
:10641000B2502254456182809165D14670009385C7
:1064200005E82D4597C0FF1FE780A03BB247E38FEB
:1064300087FA17950100130525A9F9B7C167697691
:106440008146FD1705061397060141836364B70073
:106450003E8582803307D50003470700B98F214767
:1064600013F81700858363050800B18FC207C18345
:106470007D171377F70F6DF78506F1B741C5A5476F
:10648000054763F2B70883471500034705003168E5
:10649000A207D98F13978700A183D98FC207C18321
:1064A0001308C855054763900707411106C622C463
:1064B00026C203442500914763F0870493075400E4
:1064C00063ECF502A301C50021822302C5009304F9
:1064D000340091C6A302D500A1822303D5002A84EB
:1064E000A68597000000E780A0F526942300A4006D
:1064F0002181A300A4000147B240224492443A857E
:106500004101828005473A8582800111B7C7A55AAB
:1065100022CC9387E7342A842AC621462C001565AD
:1065200006CE3EC497000000E780A0DAA28517954A
:1065300001001305E59D97600100E780606F9700FB
:106540000000E780E0D4F2406244056182800111DE
:10655000A146300095652D4522CC06CE97C0FF1F81
:10656000E7802028A24737C4A55A1304E434639572
:106570008702B245179501001305058F97D7FF1FB6
:10658000239DB7E4C205C18197600100E780406A9E
:10659000F2406244056182809165A1463000938596
:1065A00005EE2D4597C0FF1FE780A023A247E38299
:1065B00087FCD14717D7FF1F2311F7E2D145179565
:1065C00001001305658CC9B721C1411126C206C659
:1065D00022C4AE848DC52A8497000000E7808066BF
:1065E00097E7FF1F83C7C7D299CB22852244B240C9
:1065F000A685924441011733000067008322B24010
:106600002244924441018280828001114AC806CE10
:1066100022CC26CA4EC693F715002E899DCBAD67B6
:10662000371700409387A7AA1CC3B7E70400BC4FE5
:1066300013060019854517D5FF1F0345E5D9829735
:1066400013451900F2406244D2444249B2490561FF
:10665000828093F72500638A071C17F7FF1F0357F3
:10666000A71B954763F9E70C014417F6FF1F1306B4
:10667000A60A930630051305500413081004930866
:10668000B00413039005930764006374F7043A841D
:10669000FD5997F4FF1F83C4240897F7FF1F83C792
:1066A000B707A204DD8CAD679387B755638BF414ED
:1066B00063E3970AA9679387A755638EF414A285AD
:1066C00017F5FF1F1305450597000000E78000F050
:1066D00031A2B307860083C50700639AD50483C53A
:1066E00017006396A50483C527006392050583C53B
:1066F0003700639ED50283C54700639A150383C79D
:10670000570063966702A2890DE897F5FF1F83D5AE
:10671000A510B3853541C20517F5FF1F1305C5FF49
:10672000C1814E9597000000E78040EAE1A0050492
:106730004204418089BF3A84FD598547E3EB87F4E1
:106740005DC4854517F5FF1F130505FD9700000083
:10675000E780C0E769A8B1679387C7556380F404F1
:10676000B5679387D755E39CF4F4A28517F5FF1F0F
:10677000130585FA97300000E780A00A8947630F68
:10678000F4049305E4FFC205C18117F5FF1F13054B
:10679000C5F897000000E780E04A89A09720000034
:1067A000E780C0F797000000E780204911C9A28563
:1067B00017F5FF1F130545F697000000E780804896
:1067C0000546A28517F5FF1F130505F597F0FFFF96
:1067D000E780406B97200000E78040F4A68517858E
:1067E00001001305A57497600100E7806044FD5720
:1067F000E39DF9F097F7FF1F239007021345290047
:1068000091B5A28517F5FF1F130505F197F0FFFF5E
:10681000E780E078E1B7A28517F5FF1F1305C5EF04
:1068200097F0FFFFE780607955BF93F7450001457A
:10683000E38A07E017850100130585709760010062
:10684000E780E05697300000E780402B1345490071
:10685000D5BB411122C437E404005C5C06C6354652
:10686000978501009385852217950100130505ED95
:10687000829711E9178501001305456D97600100A6
:10688000E780E05201A08327041C82972A840545F3
:1068900097C00000E78060DF97500100E780408BE1
:1068A00097400100E780406097B00000E780E0F08B
:1068B0002285B2402244410182804111054506C62D
:1068C00022C426C297C0FFFFE78000551305A0042D
:1068D00097B0FF1FE780A07D757585457D1597C032
:1068E000FFFFE780A03E7D7585451305F53697C00F
:1068F000FFFFE7800048371400408327840A8D4556
:106900001305002093E707202324F40A97C0FFFF14
:10691000E780C03BB7E4040097D0FFFFE780E0804A
:10692000C85897600100E78080481795010013055B
:10693000E5E097600100E78080478327840C854568
:10694000414593E707082324F40C97C0FFFFE78035
:1069500040428D451305000897C0FFFFE780604166
:1069600097C0FFFFE780406E37A5070013050512AB
:1069700097C0FFFFE780E069014597C0FFFFE78010
:10698000007095450545894717F7FF1F2308F7E86D
:1069900097C0FFFFE7804070B7E700E013070006ED
:1069A000238DE7403707000423A0E71097D0FFFFAF
:1069B000E780A00297D0FFFFE780601697000000F5
:1069C000E78060E997000000E780C098970000002A
:1069D000E78020B897E0FFFFE78060F297000000B3
:1069E000E780802797000000E780801083A70408D5
:1069F000170500001305A5C1829797D7FF1F238DA8
:106A0000A79CBC4C130600648545829797C0FF1F66
:106A1000E780009E01458280AD673717004093876D
:106A2000A7AA1CC3B7E700E03707400023A0E71878
:106A300001000100B7F7070003C70701A547631668
:106A4000F7009397450191C301A04111AE8601461D
:106A5000AA85254506C697C0FF1FE78080D8B240AB
:106A6000B7E700E03707400023A0E710410182802C
:106A70004111B2862E86AA852D4506C697C0FF1FF6
:106A8000E78020D6B240014541018280930700048F
:106A900063ECC7041D71A2CC2A840808A6CACAC820
:106AA00086CE32C697600100E780200DAD673717AC
:106AB00000409387A7AA1CC3B7E400E03709400051
:106AC00023A0241901000100B2461008A28529451F
:106AD00097C0FF1FE780E0D0F640664423A0241152
:106AE000D6444649256182803955828041110D6521
:106AF0008D4506C697C0FFFFE780401DB7170040D1
:106B00008D6623A6D70A17F5FF1F130565D11387D6
:106B1000C70A9387870A1CC15CC5856689675CC9FB
:106B200058C114C518C9B7E70400B24003A3871EB3
:106B3000410102838145B307B5008387070089E7D8
:106B400017230000670023C48505C205C181E5B78E
:106B500097870100938787591357C5003E970347CE
:106B60000700011106CE2304E100135785003D8B79
:106B70003E970347070023060100A304E1001357D3
:106B800045003D8B3D893E97AA970347070083C781
:106B9000070028002305E100A305F100970000008D
:106BA000E78080F9F24005618280411126C2E977D1
:106BB00097F4FF1F938444D722C49387A7552E844C
:106BC0002381B4002E86AA8517F5FF1F130505D66D
:106BD00006C62390F400A381040097600100E780BB
:106BE000C0F993052400C205C18117F5FF1F1305E5
:106BF000C5D397000000E780A084B3878400238278
:106C0000A7002181A382A700930564002244B2401B
:106C100026859244C205C181410117230000670007
:106C200083B609C99307800263E6B7001703000023
:106C30006700E3F7828017F5FF1F0345E5BF8280F9
:106C400097F7FF1F83C707CE89E717230000670068
:106C500083B3828097F7FF1F83C7E7CF99EF411176
:106C600006C697200000E780E0A9B240854717F7E5
:106C7000FF1F2302F7CE4101828082806307054A0D
:106C80006385054A5D71CAC04EDE86C6A2C4A6C22F
:106C900052DC56DA5AD85ED662D466D26AD0B94788
:106CA0002A89AE8963F9B70639469785010093852D
:106CB000A53197600100E780E0E931ED8347E90005
:106CC000130710036394E702854717F7FF1F230B91
:106CD000F7C4178501001305253097F7FF1F23928E
:106CE00007C497000000E78020E571A013070003A8
:106CF0001785010013054531E395E7FE97F7FF1F60
:106D0000238207C297F7FF1F239D07C01785010045
:106D10001305052EF9B797F7FF1F83C7A7C0638731
:106D20000722BD6AB96B938CFA55014A17FBFF1F06
:106D3000130BCBB0138CEB65938AFA6605A8B307E7
:106D4000490183C6070097F7FF1F83D787BDB1E3CB
:106D50009307A005639BF600854717F7FF1F2312D3
:106D6000F7BC97F7FF1F238BD7AC050A93170A01CF
:106D7000C183E3E637FDB640264496440649F259FE
:106D8000625AD25A425BB25B225C925C025D6161E4
:106D90008280054D639BA7039307500A639EF6000C
:106DA000894717F7FF1F231EF7B6930750FA17F707
:106DB000FF1FA305F7A855BF9307A005E387F6FAC1
:106DC00097F7FF1F239F07B44DB71387170042079C
:106DD000DA9741832380D70017F6FF1F2313E6B409
:106DE0008D47E3F4E7F817F4FF1F034454A597F722
:106DF000FF1F83C7C7A422045D8C9307F4FFC2075B
:106E0000C1839306F00DE3EDF6FA93076400C20721
:106E1000C183E31CF7F493052400C205C18117F573
:106E2000FF1F1305C5A197F0FFFFE78060613307DF
:106E30008B008347570003474700A207D98F17F7F6
:106E4000FF1F231007AE6318F50E8144630CA401E5
:106E500097F4FF1F83C4C49EA20497F7FF1F83C744
:106E6000379EDD8C170500001305E5DB97F0FFFF6B
:106E7000E78000FF63878407636D9C029387EB556F
:106E80006382F40497F7FF1F83C7879B05476389D5
:106E9000E70681CB1387A7051377F70F8D4663F2BB
:106EA000E6081307F0072300E100A300F10089457D
:106EB0009DA063829405E39754FD97F0FFFFE78060
:106EC000C02B11A8A28517F5FF1F1305659797F032
:106ED000FFFFE780800F014597F0FFFFE78040F854
:106EE00069B5A28517F5FF1F1305859597F0FFFF7C
:106EF000E7804019CDB797F0FFFFE780C021E1BFE1
:106F0000930710F8130511002300F10097F0FFFF1D
:106F1000E780602DFD450A8597000000E78020C9C5
:106F20005DBFA28517F5FF1F1305859197F0FFFF41
:106F3000E780A0C94DB79307F00789450A8523105C
:106F4000F10097000000E78080C605B5BD4763F8F3
:106F500037174146978501009385450D4A8597600F
:106F60000100E78020BF631C05141785010013058D
:106F7000250D97000000E78020BC17F5FF1F035583
:106F8000C58997000000E780E0BC97E7FF1F83C733
:106F90006778178501001305250289E71785010029
:106FA0001305050297000000E78000B9178501006E
:106FB0001305850A97000000E78000B817C5FF1F7A
:106FC0000355453F97000000E780C0B817850100D2
:106FD0001305C50897000000E78000B617C5FF1F1E
:106FE0000355A53F97000000E780C0B61785010054
:106FF0001305450797000000E78000B417D5FF1F71
:107000000355651997000000E780C0B4178501009B
:107010001305C50597000000E78000B217D5FF1FD4
:107020000355251797000000E780C0B217850100BF
:107030001305450497000000E78000B017D5FF1F37
:107040000355451597000000E780C0B01785010083
:107050001305850297000000E78000AE17C5FF1FEB
:107060000355052697000000E780C0AE1785010094
:107070001305050197000000E78000AC97D7FF1FBC
:1070800083C7C717A20717D5FF1F034535175D8DA7
:1070900097000000E78000AC97D7FF1F83C7271633
:1070A000A20717D5FF1F034595155D8D97000000BA
:1070B000E78040AA177501001305C5741DB1C147CB
:1070C00063FE37054146978501009385A5FB4A85F8
:1070D00097600100E78000A831E1834709011307A9
:1070E0001003639CE700854717E7FF1F2306F7742B
:1070F00017850100130545FAEDB613070003178540
:107100000100130565FCE39EE7BC97E7FF1F23859D
:107110000772178501001305A5F9E1B6CE854A85EA
:1071200097C0FFFFE780E0F9B9B18280411126C224
:10713000AE848D4522C406C62A8497C0FFFFE7802F
:1071400040C3B717004099C803A5C70C418D23A6BB
:10715000A70CB240224492444101828003A5870CCF
:10716000418D23A4A70CF5B78347050003471500FD
:10717000A207D98FC2076177C18713072720639AB7
:10718000E70083452500370504001703000067006A
:1071900023FA828017E6FF1F1306467C8147B286DA
:1071A0001303F00FA9483308F6000348080013F74B
:1071B000F70F6307A80C630668008507E39517FFC0
:1071C0002947B387E6002380A70097E7FF1F93872F
:1071D000A7795DA8411113D765001347170006C6AC
:1071E00093F63500058B954791CA05469947638705
:1071F000C60009469D476383C600A14713F64500B4
:107200003336C00093F68503050685C2A145638B1E
:10721000B604E145638AB604930580026388B60428
:10722000930580036393B600914697F5FF1F238271
:10723000F59A97F5FF1F238DC59897F5FF1FA38932
:10724000D598BE8517850100130545EE97600100AE
:10725000E780009EB240854717F7FF1FA30BF79604
:10726000410182808546D1B78946C1B78D4675BF39
:1072700017850100130505EE176301006700439BA6
:1072800017E7FF1F1307476EBA972380B700E14740
:10729000E302F5F493077002E30CF5FC82802A8781
:1072A00023800500814717E5FF1F1305256B130891
:1072B000F00F2946B306F50083C606006396E60282
:1072C00097E6FF1F9386466AB69783C70700054572
:1072D0002380F5009947636EF7029D4763FDE70041
:1072E000E147630DF7008280638506018507E3931C
:1072F000C7FC0145C5B7238005008280B737004031
:1073000003C7370083C7050093F70704D98F23808D
:10731000F50082805D7152DC56DA5ED6716A97FBA9
:10732000FF1F938B2B9C8D6AA6C24EDE62D486C64D
:10733000A2C4CAC05AD866D26AD06ECEC1495E8C89
:1073400097E4FF1F93840463130A0A20938A7ADC6C
:1073500017F9FF1F0349099CB3872B0183C7070057
:1073600093F7F70FC9EFB787004003C76700058B96
:10737000E310077C03C76700118BE30D077E83C70B
:107380005700918B99E36F10200317F7FF1F0347F6
:10739000879885476304F7006F10400197F7FF1F38
:1073A000A389E78297E7FF1F2386076897E7FF1FF8
:1073B0002384077497F7FF1F2382078097E7FF1F37
:1073C000238F077E97E7FF1FA386076697E7FF1FB8
:1073D000A384077297E7FF1FA382077E97E7FF1F2B
:1073E000A38F077C97E7FF1FA386077E97F7FF1FF2
:1073F000A3830792B787004011476F007077930708
:10740000190093F7F70F3D476364F70617F7FF1F5F
:107410002302F79097F7FF1F9387C78ECA9783C7FA
:1074200007001307100293F7F703638EE71E6366E6
:10743000F70405446385871CE38C07620947638E64
:10744000E71013070002E384E74EB7E700E03707D1
:10745000400023A0E7180100010062992300090001
:10746000FD1923A0E71093F9F90FE39309EEE5BDA9
:1074700097F7FF1F2380078A71BF130730026388C5
:10748000E70C63E8E71613074002638CE70A13076B
:107490000003E39CE7FA97F7FF1F9387A785CA9736
:1074A00003C70700A1471377F70FE31BF71483C740
:1074B000640097E6FF1F2385F67097E7FF1F83C7D9
:1074C000D74B91C7FD5797E6FF1F238BF66E97E5C5
:1074D000FF1F83C5354A97E7FF1FA383B76E97E762
:1074E000FF1F83C7274913FB07089306000493F780
:1074F0000706639FD74C9307A009638DF51663EACF
:10750000B7129307F0056386F54A93075009638421
:10751000F52A014497E7FF1F83C7976A1547E3924F
:10752000E736B7E700E03707400023A0E71801007F
:107530000100B786004023808602130680FC6F009E
:10754000500EFD5717E7FF1F230BF766FDBDFD57D4
:1075500017E7FF1F2304F766CDBD1785010013054C
:10756000E5D097600100E780808497E7FF1F93874D
:107570006778CA9703C40700014B97ECFF1F938CF1
:10758000EC571374F40F178D0100130DADCE634744
:107590008B04294597500100E780606E854717E707
:1075A000FF1FA30BF75417E7FF1F2308875417E7A4
:1075B000FF1F2301F76237E700E0B70640002320F2
:1075C000D71801000100378600408347A60293F7D1
:1075D000370F2305F6022320D71085BDB3876C0132
:1075E00083C507006A85050B97500100E78040645A
:1075F00079BF854717E7FF1F2300F750B9B517E795
:10760000FF1F1307276F4A970347070097E6FF1FDF
:10761000A382F64297E6FF1F238FE64017E7FF1F7E
:10762000230AF75A1DB5854717E7FF1F2304F740C4
:1076300029BD9307400A6389F5349307200B6384BF
:10764000F5369307100AE396F5EC8387240001448E
:10765000E3D207EC97E7FF1F83C7F73193F63700B4
:10766000638A061A0546638AC62209466395C61AC6
:107670001D4755A217E5FF1F0345E52FC94797ECA6
:10768000FF1F83CC5C2F97E5FF1F83C5E52E17E412
:10769000FF1F0344742E6315F510CD476392FC1051
:1076A00093077008639CF5021307300FB7170E009D
:1076B0006308E4001307900DB7B704006314E408EF
:1076C00017E7FF1F2324F750BE8517850100130518
:1076D000E5BA97500100E780A05525BD93078008C3
:1076E000639DF500B307804013F4F70FB7774600AA
:1076F000938787CDB3D78702E1B793079008639A42
:10770000F500B307804013F4F70F91679387C766BE
:10771000D5B79307A008639BF500B307804013F427
:10772000F70FB7173D0093870790E9B79307B008A5
:10773000639AF500B307804013F4F70F91679387BE
:1077400097D04DBF93F5F5078D47639BF500B307C1
:10775000804013F4F70FB7975B00938707D859BFA2
:107760008947639BF500B307804013F4F70FB777A1
:107770000B009387071BBDBF8547639AF500B307CE
:10778000804013F4F70FDD67938767E3A5B7D287CF
:1077900085F9B307804093F7F70FB3D7FA020DB717
:1077A00097000000E780409FA28566859700000053
:1077B000E780809EB9BB9305610017E5FF1F034575
:1077C000851B17E4FF1F0344141B97000000E7808C
:1077D00040AD93057100228597000000E78060AC02
:1077E0003C0017E7FF1F232DF74E8347610023045A
:1077F000F10083477100A304F100894717E7FF1FD9
:107800002300F73C8357810017E7FF1F2314F71667
:10781000094409B3154793F64700B336D00093F7F0
:107820008703850685C32146638BC7066146638A45
:10783000C706130680026388C70613068003639396
:10784000C700914717E6FF1F2304D63897E6FF1FAE
:10785000A380F63897E7FF1F238DE73617E7FF1F52
:10786000034787119376070497E7FF1F83C7D71055
:107870008DEE1377770C93067008630CD70213779D
:10788000F7078D466312D70CB307F040B7955B003E
:1078900093F7F70F938505D849A81947ADBF8547DA
:1078A00055B7894745B78D4771BF93067008631177
:1078B000D7021307300FB7150E006389E7021307CD
:1078C000900DB7B504006383E7021307700845BF46
:1078D0009306800C6311D702B307F040B7754600DA
:1078E00013F7F70F938785CDB3D5E70297E7FF1F0F
:1078F00023AEB72CD9BB9306900C631CD700B307FB
:10790000F04093F5F70F91679387C766B3D5B70239
:10791000F1BF9306A00C631DD700B307F040B71565
:107920003D0093F7F70F93850590B3D5F5027DBF22
:107930009306B00CE315D7F4B307F04093F5F70FB7
:107940009167938797D0D9B78946631BD700B30750
:10795000F040B7750B0093F7F70F9385051BF1B750
:107960008546631AD700B307F040DD6593F7F70F3C
:10797000938565E35DBFD28535FBB305F04093F594
:10798000F50FB3D5BA029DB783C72400C18B99C741
:10799000854717E7FF1F2308F722A5BE97E7FF1FBC
:1079A00023830722BDB6854717E7FF1FA303F722EE
:1079B0008DB63C0017E7FF1F2324F73209479307D2
:1079C00000032314F10097E6FF1F238BE61E2DBD55
:1079D00063940756A94763E5B74217770100130779
:1079E00027728A05BA959C41BA97828717E4FF1FD0
:1079F000034474F8894C6306940D63E68C0685474E
:107A00006303F4089307F00F17E7FF1F0347471BB3
:107A100063F6E70017E7FF1F2304F71A97ECFF1F31
:107A200083CC0C1A9307000413F4FC0F63F4970142
:107A30001304000497E7FF1F9387872A03AD07000D
:107A400022862685EA85B38C8C40229D97500100C2
:107A5000E780A01297E7FF1F2384971797E7FF1F80
:107A600023A0A72945BC8D47630CF40A9947E31B63
:107A7000F4F8977701009387276F17E7FF1F2321FB
:107A8000F726A94751B717E7FF1F0347C72897E70E
:107A9000FF1F9387E7144946977501009385C575C5
:107AA0006306870097750100938505713E859750A1
:107AB0000100E780800C17E7FF1F2323A722C94797
:107AC000A1B797E6FF1F83C60625054797E7FF1F67
:107AD000938707116394E6023E851306700297753B
:107AE00001009385E56E97500100E780000917E7D4
:107AF000FF1F2327A71E9307700239B73E85130681
:107B00003004977501009385E56697500100E78082
:107B1000C00617E7FF1F2325A71C93073004EDB508
:107B200097E5FF1F83C525E5177501001305457609
:107B300097500100E780C00F054D97EDFF1F83CDE3
:107B40008D1D97E5FF1F83C505E31775010013051C
:107B500025746398AD0B97500100E780600D97E79F
:107B6000FF1F83C747E1B5CBE36EF4E8177401004C
:107B70001304C46C638CB701177401001304846C84
:107B800063869701177401001304446D2285975092
:107B90000100E78000231375F50F93071500860792
:107BA00017E7FF1F230EF7028D4717E7FF1FA309F3
:107BB000F70297E7FF1F9387A7020147BE86137658
:107BC000F70F89076365A60297E7FF1F23AAD7105F
:107BD00097E7FF1F83C7C70005BD9777010093870D
:107BE000E75E17E7FF1F232DF70E914731BD3306E0
:107BF000E40003460600A380070005072380C700B2
:107C00007DBF97500100E780A00297E7FF1F83C761
:107C100087D6E1D7E368F4DE177401001304045F2C
:107C2000638CA701177401001304C45E6386970177
:107C3000177401001304845F228597500100E780C8
:107C400040181375F50F93071500860717E7FF1FF8
:107C50002308F7F88D4717E7FF1FA303F7F897E707
:107C6000FF1F9387E7F70147BE861376F70F890753
:107C7000E37CA6F43306E40003460600A380070075
:107C800005072380C700D5B797E5FF1F83C5A5CE9D
:107C9000177501001305856097500100E78040F9D2
:107CA00097E7FF1F83C797F393E7470017E7FF1F87
:107CB000A306F7F283C7240017E7FF1FA30EF7F010
:107CC00089B8177501001305A55E97500100E7807C
:107CD000000E97E7FF1F938727F083C7070017E77A
:107CE000FF1F2309F7C817E4FF1F034464ED333473
:107CF00080000DB0177501001305C55C9750010099
:107D0000E780E00A97E7FF1F83C757ED93E7070176
:107D100017E7FF1FA304F7EC83C7240017E7FF1F33
:107D2000230CF7EA6FF0EFFE177501001305C55A33
:107D300097500100E780A00703C704007D8B51EF37
:107D4000B787004003C767021377C70B1367270085
:107D50002383E70203C7A7021377C70B1367270024
:107D60002385E70203C7E7021377C70B13672700D2
:107D70002387E70203C727031377C70B136727007F
:107D80002389E702854717E7FF1F2305F7CA17E78F
:107D9000FF1F2303F7D617E7FF1F2301F7E217E7BB
:107DA000FF1F230EF7E097E7FF1FA38507C897E79C
:107DB000FF1FA38307D497E7FF1FA38107E097E77F
:107DC000FF1FA38E07DE97E7FF1FA38507E097E756
:107DD000FF1FA38207F46FF0CFF389476312F70206
:107DE00097E7FF1F83C747B99146638CD70863E0C5
:107DF000F604638EE70C6369F70A05476380E70EB4
:107E0000FD5717E7FF1FA30DF7DA37074000B7E765
:107E100000E023A0E71801000100B7860040130628
:107E2000F0FC2381C60223A0E7106FF00FE21307D6
:107E300020086382E7086362F70213071008E391E2
:107E4000E7FC378700408347670293F7C70B93E748
:107E500027002303F7026FF0CFEB13073008638985
:107E6000E70213074008E39DE7F8378700408347A0
:107E7000270393F7C70B93E727002309F7026FF057
:107E80004FE9378700408347270393F73707F5B754
:107E9000378700408347E70293F7C70B93E7270034
:107EA0002307F7026FF0EFE6378700408347E702CA
:107EB00093F73707F5B7378700408347A70293F753
:107EC000C70B93E727002305F7026FF08FE437878E
:107ED00000408347A70293F73707F5B7378700407D
:107EE0008347670293F73707ADB71775010013058E
:107EF000A53F97500100E78080EB97E7FF1F238B9A
:107F000007A6D5B3177501001305053F975001006B
:107F1000E780E0E997E7FF1F239E07A497E7FF1F8D
:107F2000938707CA03C40700894763F3870009449E
:107F30001374F40F6FF00FDE13070002E392E7EC07
:107F4000631B0B0A638FF500930720026383F50818
:107F5000177501001305C53D97500100E78040CD1E
:107F600045B5177501001305E53997500100E78005
:107F700000E40144177D0100130D0D3AA14CB387B5
:107F8000840083C507006A85050497500100E780D7
:107F900020CAE31694FF177501001305A58C9750AE
:107FA0000100E780C0E017E4FF1F0344E49C01E800
:107FB00097E7FF1F2382079A014B6FF0AFD58947E0
:107FC000E310F4E4854717E7FF1F2307F7986FF0E6
:107FD0004FD417E6FF1F0346169A97E5FF1F83C588
:107FE0008599177501001305A53397500100E780A7
:107FF00020C46FF00FD26380F50693071002E39957
:10800000F5F497E5FF1F83C5259717750100130544
:10801000253397500100E780A0C197E7FF1F23A1F8
:1080200097CC97E7FF1F938767BA944383D747009E
:1080300017E7FF1F0347E7B917E6FF1F232CD69268
:108040001D4497E6FF1F2399F69297E7FF1F2386AB
:10805000E7926FF02FCC97E5FF1F83C5E591177569
:1080600001001305652F97500100E78060BC97E77A
:10807000FF1F2383078E97E7FF1F239D078E6FF057
:108080002FF92547638FE7C89946378700406394E7
:10809000D70223008702B7E700E0B706400023A01D
:1080A000D71801000100130600FC2301C70223A01A
:1080B000D7106FF08FB99306100A639FD700230083
:1080C0008702B7E700E0B706400023A0D7180100F9
:1080D0000100130680FCD1BF9306A009E381D7FEFF
:1080E0009306400AE38DD7FC93062002639DD700D8
:1080F000B7E700E0B706400023A0D7180100010051
:1081000023008702F9B78546E384D7FE930700086A
:10811000E300FBFEB7E700E0B706400023A0D71856
:1081200001000100130620FC23008702BDBF17E7F2
:10813000FF1F0347F7A86302F71E63E7E7029547AF
:108140006300F7109947630AF704B786004023805D
:108150000602B7E700E03707400023A0E718010058
:1081600001001306A0FC75B99307F005630AF70038
:10817000930750096306F70093071002E317F7FC13
:10818000B7E700E03707400023A0E718010001002F
:10819000B7860040130620FC69B117EBFF1F034BA5
:1081A0002BA2930700045A8D63F46701130D00049A
:1081B00097E7FF1F9387C7B283AC07001374FD0FC7
:1081C0002286E685268597500100E780009BB3074D
:1081D0008B40669417E7FF1F2304F79E97E7FF1F66
:1081E00023A087B0B7870040630C0B022380A7034E
:1081F000B7E600E03706400023A0C61801000100E2
:1082000003C72702134707042381E70203C7270296
:108210001377C70F2381E70223A0C6106FF0EFA2E8
:108220002380070237E700E0B70640002320D71875
:1082300001000100130620FC2381C7026FF0AFB9D3
:10824000378700408347370097E6FF1F83C6D698DD
:1082500093F70708D58FA301F700B7064000B7E7EB
:1082600000E023A0D718010001001306A0FC35BDD3
:1082700097E7FF1F938707A8CA9783C7070093F75D
:10828000F70FC1CF97E7FF1F83C7E7A8D9E717E725
:10829000FF1F0347F792930700026310F70883ADAF
:1082A000040017DDFF1F034D2D6D97DCFF1F83CCEE
:1082B000BC6C17DBFF1F034B4B6CE6876A87DA86C3
:1082C0006E8697D5FF1F83C52569177501001305B5
:1082D000250A97500100E780A09597E7FF1F23A785
:1082E000B78F97E7FF1F2385A78F97E7FF1FA3810E
:1082F000978F97E7FF1F238E678D97D7FF1FA38C5C
:108300008764B7E700E03707400023A0E7180100C3
:108310000100B78600406FF04FA2B7E700E03707D3
:10832000400023A0E71801000100B786004015BDFA
:1083300097E6FF1F83C6269E0547639CE6042947F0
:108340002381E70209472383E7022385E70297E7B2
:10835000FF1FA381078897E7FF1FA38E079AB787A0
:108360000040A381070017E7FF1FA3070786054703
:108370002383E700B640264496440649F259625AE0
:10838000D25A425BB25B225C925C025DF24D61614B
:10839000828029472381E70209472383E702238557
:1083A000E7022387E7022389E70255B717D7FF1FA4
:1083B000A303F75A6FE01FFF854717D7FF1F230B53
:1083C000F76617D7FF1F2309F77217D7FF1F230779
:1083D000F77E17D7FF1F2304F77E6FE0BFFE8547A8
:1083E00017D7FF1F2308F76417D7FF1F2306F7705F
:1083F00017D7FF1F2304F77C17D7FF1F2301F77C34
:1084000017D7FF1FA308076217D7FF1FA306076E22
:1084100017D7FF1FA304077A97D7FF1FA381077AF7
:108420008280411106C697000000E78080FBB78775
:10843000004023800700130740FC2386E700130752
:10844000C004A386E70017D7FF1F1307A75223987E
:10845000E70017D7FF1F1307E755239AE70017D741
:10846000FF1F13076761239CE70017D7FF1F130740
:10847000E76C239EE70029472381E702094723830E
:10848000E7022385E7022387E7022389E702A38126
:108490000700930600F8A380D7009306900223807C
:1084A000D700FD562383D7002381E70093060005FC
:1084B00037E700E0230BD740B70640002320D71052
:1084C00003C7170013671700A380E700B24097D7D0
:1084D000FF1F2393077041018280411106C6970058
:1084E0000000E78000F0B7870040238007001307F3
:1084F00000FC2386E7003147A386E70017D7FF1F5C
:10850000130747472398E70017D7FF1F1307874A2A
:10851000239AE70017D7FF1F13070756239CE7008E
:1085200029472381E70209472383E7022385E702DE
:10853000A3810700930600F8A380D700930690025A
:108540002380D700FD562383D7002381E7009306BD
:10855000000537E700E0230BD740B7064000232093
:10856000D71003C7170013671700A380E700B240B6
:1085700097D7FF1F2392076641018280F167938797
:10858000072017D7FF1F2323F764854717D7FF1F3F
:108590002310F764A14717D7FF1F230CF76297D763
:1085A000FF1FA388076297D7FF1F2385076297D70E
:1085B000FF1F2383073A97D7FF1FA38E07388147F2
:1085C00017D5FF1F13058539FD5517D6FF1F130655
:1085D000A6392947B306F5002380B600B306F60096
:1085E000238006008507E397E7FE97D7FF1FA38A3E
:1085F000075C97D7FF1FA388075C97D7FF1F2383CC
:10860000075C97D7FF1F238E075A97D7FF1F238D2D
:10861000075A97D7FF1FA387075A97D7FF1F2384AF
:10862000075A814717D6FF1F1306C66B4147B3068B
:10863000F600238006008507E39BE7FE828017D7BC
:10864000FF1F0347476D85476316F70017030000B8
:108650006700E3E8170300006700E3DC411122C470
:1086600006C617D7FF1F0347076B85472E8613F4EF
:10867000F50FAA856317F70417D5FF1F1305C54328
:1086800097400100E780604F97D7FF1F238607467A
:10869000B787004023848702B7E600E03706400032
:1086A00023A0C6180100010003C7A7021377C70F54
:1086B0002385E702B240224423A0C61001454101B0
:1086C000828017D5FF1F1305E53297400100E78030
:1086D000C04A97D7FF1F238F0734B78700402382F4
:1086E0008702B7E600E03706400023A0C618010065
:1086F000010003C767021377C70F2383E7025DBF3B
:10870000411106C697000000E78080E7B2404101B2
:10871000170300006700E3F2411106C697F0FFFF60
:10872000E78080BF97D7FF1F83C7D730A1CB97D5EE
:10873000FF1F83C5453089C917D5FF1F1305C52FF6
:1087400097E0FFFFE780C05397D7FF1FA384072E52
:1087500097D7FF1F2380074837E700E0B7064000A0
:108760002320D718010001003786004083476602A6
:1087700093F7370F2303F6022320D710B2404101AD
:10878000828041C9D9C597D7FF1F83C7E744D1C3AA
:10879000011122CC4AC84EC656C25AC006CE26CABD
:1087A00052C42E89AA890144930A0004371B03008E
:1087B00063772403B3078940C207C183BE8463F48F
:1087C000FA0093040004C204C180130A1BD497D793
:1087D000FF1F83C727269DE37D1A631C0A00F24012
:1087E0006244D2444249B249224A924A024B05614C
:1087F000828097F0FFFFE78020B2D1BF33858900E8
:108800002694A685420497000000E78060E5418039
:1088100045B7828097D7FF1F9387875318429C43A1
:1088200083D645000345070083C5C70003564600AD
:108830006396A50083D5E700638DD502011106CEAE
:108840002386A7002397D700B705CF00DC4B93857D
:10885000757D05077D162EC2230001003AC423163C
:10886000C1002317D10099C30A858297F2400561A0
:1088700082808280DC4DDC4B81CFB7E704009045DD
:1088800003A38705914517D5FF1F0345A54C028318
:1088900082806D713C083EC6B707E5002322911027
:1088A0003EC8AA843C083285232611103ECA2324E0
:1088B0008110232021112E8997300000E780E05A93
:1088C0002A8497750100938525AE1765010013056D
:1088D000A59297400100E780A035A2851775010099
:1088E000130505BD97400100E78080342945974076
:1088F0000100E780C038B705CB009385757D68001F
:1089000097100000E7800069A2856800973000009A
:10891000E7800048014781467000CA852685972078
:108920000000E780808C05CD2A849775010093852F
:10893000A5A7176501001305258C97400100E78066
:10894000202FA28517750100130545B79740010038
:10895000E780002E294597400100E78040328320C0
:10896000C110032481108324411003290110516197
:10897000828097D7FF1F9387A73D18429C43797148
:1089800022D406D60348070083C807012A8483D669
:108990004500035546006396080183D82701638D7F
:1089A000D8022388070105072399D7003708CC0090
:1089B000DC4B1308787D3ACC1307F5FF42CA230835
:1089C0000100231EE100231FD10099C7080832C609
:1089D0002EC482973246A245228597000000E78088
:1089E00080EBB2502254456182806D713C083EC0DC
:1089F000B707E5003EC23C083EC4232611102324DD
:108A0000811023229110231701002318010023193C
:108A10000100231A0100231B010097B7FF1F83D712
:108A2000279E99E3C167FD172316F10097B7FF1F33
:108A300083D7279D91EB97D7FF1F938767319C437F
:108A40009C43DC4783D7070017B4FF1F1304449BE4
:108A5000584C2317F10083574400484B2318F1006A
:108A600031E1977501009385259B1755010013058A
:108A7000A57897400100E780A01B1775010013053A
:108A8000E59A97400100E780A01A29459740010028
:108A9000E780E01E8320C11003248110832441104D
:108AA0005161828097B7FF1F83C7F79589EBB7E7BE
:108AB0000400BC5782975C4C23AA0700E1BFFD1756
:108AC00097B6FF1FA381F69403560701834704015D
:108AD0004C470A85230BF10097300000E78060289F
:108AE00097D7FF1F9387C7269C430147814688433A
:108AF0000A866C0097100000E780206FAA8429C1C5
:108B00009775010093854591175501001305C56EB2
:108B100097400100E780C011A68517750100130575
:108B2000A59197400100E780A010294597400100DA
:108B3000E780E014584CB7E70400BC57484B9DBF92
:108B400097B7FF1F83C7378CF5D7B7E70400BC4F33
:108B50001044854517D5FF1F0345C51F82971DBFCC
:108B60005C4EDC4BB9CFB1CD411122C41755010089
:108B7000130585682E84977501009385258806C6A0
:108B800097400100E780C00AA28517750100130510
:108B9000658D97400100E780A009294597400100B5
:108BA000E780E00DB7E704002244B24003A3870545
:108BB00017D5FF1F0345051A1306400691454101CD
:108BC00002838280411122C417B4FF1F1304048161
:108BD0001C4C06C689C7DC4399C34C488297584C45
:108BE000B7E70400BC57484B82975C4CB240224424
:108BF00023AA07004101828017B7FF1F13070780D0
:108C0000834707009306F00B850793F7F70F63E997
:108C1000F60097A6FF1F2383F67E03450700828098
:108C2000930700F8FDB783574500638607100111CD
:108C30004AC817A9FF1F1309A97C52C4032AC901F6
:108C400006CE22CC03274A0126CA4EC656C2F15789
:108C500035E31307D00DFD57636EC704B7E9040071
:108C600083A709072A841305860042054181B2843F
:108C7000AE8A8297232AAA000325C9015C49A9E785
:108C80009765010093858575175501001305C55635
:108C900097400100E780C0F9177501001305C584EE
:108CA00097400100E780C0F8294597400100E78020
:108CB00000FDDD57F2406244D2444249B249224AA3
:108CC000924A3E850561828093874400B705CF00B4
:108CD0002319F5009385757D310597100000E78015
:108CE000602B0325C90183456400310597300000DE
:108CF000E780000A0325C9012686D685310597300D
:108D00000000E78000067146A2854A859740010071
:108D1000E780A0E6504419CA83A78905854517D581
:108D2000FF1F034525038297814769B7970000001D
:108D3000E780E0CBD5BFFD573E858280411126C23A
:108D400097A4FF1F9384C46BD84C22C437E404005B
:108D50003C54484B06C68297DC4C0323C40522448E
:108D6000B240924423AA070017D5FF1F034585FE92
:108D7000854541010283411126C297D4FF1F938488
:108D800024FD9C4006C622C44AC0D5C3DC43C5C3EB
:108D90005CC12300B5002A84976501009385455F77
:108DA000175501001305454597400100E78040E84D
:108DB000294597400100E78080EC9C4023A40700F0
:108DC00023A2070097A7FF1F93874761DC4FDC4B67
:108DD00091C7295597000000E78000DF97A7FF1F84
:108DE00093870762DC4FDC4B89C797000000E78060
:108DF00020F537E904008327C905894517D5FF1FEA
:108E0000034545F582978327C905914517D5FF1F6F
:108E1000034545F482979C4003A34701630903007F
:108E200022852244B2409244024941010283B24069
:108E3000224492440249410182800111328506CECA
:108E400022CC26CA2E8497300000E7800002AA8434
:108E50009765010093850557175501001305C5391E
:108E600097400100E780C0DC0307840003566400DC
:108E700083554400A686176501001305A560974039
:108E80000100E780E0DA294597400100E78020DF14
:108E900097A7FF1F83C7E754639D9700014597007D
:108EA0000000E78060D281450A8597000000E780D6
:108EB000C0ECF2406244D244056182806D7123248B
:108EC0008110232611102322911093F745002E8440
:108ED000638707143C083EC0B707E5003EC23C0864
:108EE0003EC4231701002318010023190100231A8F
:108EF0000100231B010097A7FF1F83D7274E99E38B
:108F0000C167FD172316F10097A7FF1F83D7274DD1
:108F100091EB97D7FF1F9387A7E39C439C43DC47C4
:108F200083D7070017A7FF1F1307474B2317F1002D
:108F3000544F835747002318F100DC4AA1E7976597
:108F400001009385654C175501001305E52A9740EC
:108F50000100E780E0CD176501001305254D97401E
:108F60000100E780E0CC294597400100E78020D14F
:108F7000134544008320C110032481108324411031
:108F80005161828097A7FF1F83C7B7452555D9C375
:108F9000FD1717A6FF1FA306F64403D60601834755
:108FA0000701CC460A85230BF10097300000E780CB
:108FB00040DB97D7FF1F9387A7D99C4317A7FF1FB5
:108FC0001307C741976601009386464988430A867E
:108FD0006C0097100000E7804021AA8451D9976562
:108FE000010093856542175501001305E520974060
:108FF0000100E780E0C3A685176501001305C5439E
:1090000097400100E780C0C2294597400100E780F2
:1090100000C7268597000000E78000BB91BF93F74B
:1090200025009DC7B7E70400BC4741468145280895
:109030008297255597000000E78000B9280893051E
:10904000F00F97000000E78040D3134524001DB7C0
:1090500093F71500014599DF97000000E7802099FC
:109060001345140001BF5C4D411106C688C317D7D4
:10907000FF1F232FF7CCB7E7040083A707081705C6
:1090800000001305E5E38297B24097D7FF1F2383C3
:10909000A7CC01454101828001113335A000A3070F
:1090A000A100B7E7040083A7471706CE1306F10017
:1090B0008545130550308297F24005618280828099
:1090C000411122C406C697D7FF1F83C727CA014490
:1090D00089EF97B7FF1F83C7B723054499E717C4E4
:1090E000FF1F0344246313441400228597000000EB
:1090F000E780C0FA176501001305054A09E4176502
:1091000001001305654A2244B240410117430100A2
:10911000670003B2797122D4A30F010037E4040081
:109120008327841726D24AD006D6AA842E8913050F
:1091300050309305F10132C6829732468347F101E0
:1091400093150601C18185CB01452EC6970000000D
:10915000E780C0F483274417B2454A862685829764
:10916000054597000000E78060F3B2502254925406
:10917000025945618280832744174A862685829753
:10918000EDB741119397050122C406C626C2C187D7
:109190002E8463D40702B7E40400FC5417A5FF1F14
:1091A00003450529829719C1BC5482972165218DF9
:1091B000B240224492444101828093F715008DC74A
:1091C000B7E7040083A7471A17A6FF1F1306462513
:1091D00097D5FF1F9385C5B817A5FF1F03454525E4
:1091E000829713451400E9B793F7250099CFB7E7A5
:1091F0000400BC4F13060064894517A5FF1F0345F3
:10920000252382971345240065B793F7850085CF02
:1092100097D7FF1F83C747B685E7B7E7040003A8C2
:10922000871A1307401F97A7FF1F83C76720814630
:1092300013064006994517D5FF1F035565B30298DD
:1092400013458400B5B793F745000145B5D3B7E49E
:10925000040083A7041817D5FF1F035565B1829733
:10926000BC4C13060064914517A5FF1F0345451C20
:109270008297134544002DBF97D7FF1F83D747AF71
:109280006398A70217D7FF1F2315B7AE17D7FF1F85
:109290002312C7AE17D7FF1F231FD7AC2E86176523
:1092A00001001305E536BE851743010067004398AA
:1092B000176501001305453717430100670023AF09
:1092C0000357450097D7FF1F83D787AA631EF7046C
:1092D000C1674111F91722C417D7FF1F232AF7A826
:1092E00037E4040097D7FF1F23A607A897D7FF1FCF
:1092F000A38E07A697D7FF1F238007A87C4C06C61E
:10930000894517A5FF1F0345A51282977C4C9145FF
:1093100017A5FF1F0345C51182972244B2404101A2
:1093200017030000670003DA176501001305C52F56
:10933000174301006700A3A77D15954763E2A71CAB
:10934000176701001307C7230A053A951C4101114D
:1093500022CC06CEBA972E848287176501001305AA
:10936000252D97400100E78080A4A1A203C7250016
:1093700099476311F7022E8597000000E78080F47B
:1093800083456400176501001305852B9740010094
:10939000E780008A97B7FF1F238C07F61765010047
:1093A0001305C52B7DBF03C7250095476319F70239
:1093B000C16717D7FF1F0357A79BF91703D5A50050
:1093C0006309F702B7E7040083A7C71782971765F9
:1093D00001001305A52997400100E780409D8547BE
:1093E00017B7FF1F2306F7F2176501001305852A3B
:1093F0008DBF97D7FF1F239DA79683D7E50097D6EC
:10940000FF1F2398F69683D7050197D6FF1F239356
:10941000F69683D7250197D6FF1F239EF69497D7FC
:10942000FF1FA3850794631BE502B7E70400BC4F49
:10943000096613060690A14517A5FF1F034545FFC2
:1094400082970356E4008355A400176501001305B5
:10945000252397300100E780A07D51B79307700F57
:109460002316F100B7E7040083A7870D17A6FF1F97
:10947000034606FC6C0082974DF9854717D7FF1FFE
:10948000A306F78E5DB71765010013056521D1BDF1
:1094900083C5250091476392F50217650100130506
:1094A000A52197400100E780809097000000E780A9
:1094B00060C1F24062440561828099476392F5027F
:1094C000228597000000E780E0DF83456400176590
:1094D00001001305E51697300100E7806075D1BFE4
:1094E0009547639AF50083471400E1F3176501007F
:1094F0001305C51EBDB5176501001305A51EE1BF07
:1095000082803757315F97A7FF1F9387A7F3130711
:1095100077D598C39356C500176701001307070C4A
:10952000BA9683C5060093568500BD8ABA9603C6CF
:10953000060093564500BD8A3D89BA962A9783C690
:10954000060003470700238407002383D700A38373
:10955000E7002382B700A382C70097A7FF1F938766
:1095600067EF2383B700A383C7002384D700A384B6
:10957000E7008280411106C697000000E780A0F84E
:10958000B7E7040083A7871417A6FF1F130686EB0F
:10959000D54501458297B2404D4697A5FF1F93855B
:1095A00065EB130570304101170300006700C3B677
:1095B00061712324811A37E40400832704082326D9
:1095C000111A2322911A2320211B232E311917054A
:1095D0000000130545BB829717A9FF1F130949E532
:1095E000994785442300A900231CF10097650100D9
:1095F0009385C5FD93074006175501001305C5BFA8
:10960000231CF1082308910097C9FF1F9389E920C3
:1096100097300100E780C06183D50900176501001C
:109620001305C5F997300100E78080602945973020
:109630000100E780C06403D5090089699700000034
:10964000E78060EC832744171008854513055030E8
:1096500082978327441717A6FF1F1306A6DFCD4561
:109660001305703082978327441717A6FF1F130630
:1096700066DCB545130560308297832744173008B0
:10968000894513051031829783274417300989458E
:1096900013052031829783274415938509900D4542
:1096A0008297832744159385099011458297A305D6
:1096B00091002306910002CD23080100230C010034
:1096C00083278416300991451305704082978327BC
:1096D00084161306B1008545130500408297832741
:1096E00084167000854513051040829783278416E1
:1096F000300885451305204082978327841610087B
:109700008545130550408297832704157D55829720
:10971000832744137D5582977D5597A0FFFFE780EF
:10972000E0E48327440C829797A0FFFFE78040C0C6
:109730008327841417A6FF1F1306C6D0D5450145FD
:10974000829789471306700F814528092306F10087
:109750009790FFFFE780A09B8D4713060008814587
:109760002808230CF1089790FFFFE780409A914763
:10977000230CF1009757010093878799984383C77B
:1097800047003AC8230AF10097D0FFFFE78040B0B6
:1097900070008545054597A0FFFFE78040E430094C
:1097A0009305700F094597A0FFFFE78040E330085D
:1097B000930500080D4597A0FFFFE78040E21008E1
:1097C0009545114597A0FFFFE78060E1C16717C786
:1097D000FF1F1307E759F9171CC32322070017A51A
:1097E000FF1F1305A5C497A0FFFFE78020DE832796
:1097F000C41D17C5FF1F1305255682973C48034516
:109800000900854582978320C11A0324811A832485
:10981000411A0329011A8329C1195D618280C16738
:1098200017C8FF1F0358C854F9176301F8083DCD46
:10983000B5CD011126CAB7E4040083A7841222CC57
:109840002E862315B10006CE2A8401478146ED45B8
:10985000428582972AC611ED17650100130545D987
:1098600097300100E780A054F2406244D244056181
:109870008280FC440356A100A28582972C0017C564
:10988000FF1F0355E54E97A0FFFFE780E0E069DD8D
:1098900017650100130505D797300100E7802051B7
:1098A00083A7C412ED45280082977DBF82800DC535
:1098B000854717A7FF1FA304F7B897A7FF1F2381AA
:1098C00007B8354697A5FF1F9385C5B613056030C9
:1098D000170300006700438497A7FF1FA38107B603
:1098E000E9BF97C7FF1F83C72749A9EFC16717C7FC
:1098F000FF1F0357E747F9176306F7044111854730
:1099000022C417C7FF1F2309F74637E404007C4C25
:1099100006C6A14517A5FF1F034585B182970323FE
:10992000841A2244B24097A7FF1F83C767B017C5A8
:10993000FF1F0355E5431307401F814631469945F4
:109940004101028382806D7123248110232611102E
:1099500023229110328401CD8947630AF5028320C6
:10996000C110032481108324411051618280176546
:1099700001001305E5D7AE8497300100E78020434E
:10998000A285268597C0FFFFE78020B0C9BFB7E753
:109990000400FC472800829717650100130505D6CF
:1099A00097300100E780A0408347810039C4130746
:1099B000000B6380E7021387A7051377F70F8D4627
:1099C00063EDE602A285280097C0FFFFE780E01F55
:1099D00079B78547E3F587F883459100175501006E
:1099E0001305C5B6B335B00097A7FF1F2382B77A1A
:1099F00097300100E780C0239DB703479100A2077D
:109A0000D98F35671307D7556385E7086368F70271
:109A10002D671307B7556387E70631671307C755E7
:109A2000638AE70429671307A7556394E702A285B1
:109A3000280097C0FFFFE780405815B739679306A5
:109A4000E7656381D70863E9F6001307E755638488
:109A5000E706A28528003DB73D679306F755638A60
:109A6000D7061307F766E396E7FE97C0FFFFE78088
:109A7000C070F5B50146A285280097C0FFFFE780BA
:109A80006040F1BDA285280097C0FFFFE78020510C
:109A9000F9B58947E3F587EC97000000E780A0E47B
:109AA0009305E4FFC205C1811305A1009790FFFF54
:109AB000E78020616DB5A285280097C0FFFFE78091
:109AC000C05071BDA285280097C0FFFFE780805B72
:109AD00079B597C0FFFFE780006451B5C16717C52E
:109AE000FF1F0355E528F9176307F500B7E70400E2
:109AF00003A3C71702838280854717C7FF1F230769
:109B0000F726014517F3FFFF670043591783FFFF4F
:109B1000E702435B2A8408452E89B28919C900C12E
:109B2000971500009385A586610597100100E780D1
:109B3000402381447D5A97100000E780A03563C719
:109B4000A404814497100000E780C03563C8A404D2
:109B500097C7FF1F938787229C43DC47B307F940D1
:109B600091872302F400638309048327C900B307A4
:109B7000F4409587A302F4001C4C89C79C4799C305
:109B8000228582971783FFFF670003575C44139772
:109B900014008504BA972390470171BF1C4813979E
:109BA00014008504BA972390070069BF83278900B2
:109BB0000547B307F4409587A302F40083570400D8
:109BC000638EE7028DC309476384E7040D47E3957D
:109BD000E7FA97670100938727051CCC9767010078
:109BE0009387870511A897670100938767CB1CCCE3
:109BF000976701009387C7CB5CC8BDBF976701001B
:109C0000938707B71CCC97670100938767B7EDB7B9
:109C100097670100938707061CCC9767010093871D
:109C20006706D9BF95E51783FFFFE702434B004660
:109C300018448347940075839D8B6317F700971032
:109C40000000E78020B048C41783FFFF6700634B24
:109C500082801783FFFFE702E34613893500C16462
:109C600042094111AA890144F11413590901054A15
:109C70002EC697100000E780E021B2456348A4009B
:109C8000014541011783FFFF6700034783A70900D0
:109C900013171400BA9783D707006388B70063943B
:109CA000970063742A010504E1B70545D9BF1783FE
:109CB000FFFFE7024340AA892E89328BB6843A8A95
:109CC000BE8A97A00000E78020F671C926859720FC
:109CD0000000E78020048D4763E7A7007D551783C8
:109CE000FFFF6700C34083DB440097100000E7805C
:109CF00060202A8497100000E780002193077400F9
:109D000031443305850263CDA70297100000E78038
:109D1000601E97100000E780E01D2A849710000065
:109D2000E780801E9307740031443305850263C3C6
:109D3000A70497100000E780E01B9307450029A8BF
:109D400097100000E780401C330585021307F017C9
:109D50009307C017E35FA7FA2D55E3C277F96304B1
:109D60000B02D6865286A6854A8597000100E780B9
:109D7000E0DBB5B797100000E780001933058502D6
:109D80009307C5FFD1BF832749001385C90083D539
:109D9000270097000000E78000EC61F581B7695566
:109DA0003DBF97C7FF1F239DA7FC97C7FF1F938742
:109DB000E7FC904381470C463307F5004207418397
:109DC0006393B70082805446139847008507C29674
:109DD0002390E600D5B797C7FF1F938727FA9C43C8
:109DE00003C58700828017C5FF1F035565F9828070
:109DF0001783FFFFE702A32EC1671387D7FF630B0B
:109E0000E502636AA700F1176300F50201451783B5
:109E1000FFFF6700032F1387E7FF6302E502FD17CB
:109E20001D8D13351500E5B797500000E780C02160
:109E30007D15C5BF97500000E78040F6D5BF97500D
:109E40000000E78060F4EDB71783FFFFE7022329E6
:109E50004111AA8401442EC697100000E7808004B7
:109E6000B2456348A400014541011783FFFF670025
:109E700043299C48131514003E9583570500E3853C
:109E8000B7FE0504C9BF03485500814693F7F60F96
:109E900063E5070181473E858280584593975600C8
:109EA000BA9703D727006316B70003D70700E30468
:109EB000C7FE8506E1BF8346450001479377F70F4C
:109EC00063E4D700814711A81C4513165700050706
:109ED000B29703D60700E313B6FE3E858280178350
:109EE000FFFFE702231E93170501C18797CAFF1FD3
:109EF000938ACAE8635BF00883A70A00C0479C47BF
:109F000003570400198D420541816368F50001443F
:109F100022851783FFFF6700231E12052A94CDBFF9
:109F2000DC4713944900014A3E948347440063414F
:109F3000FA02014A834754006349FA028509C209BB
:109F400093D9090183A70A009847E3EBE9FCC1B75D
:109F50001C4413195A00A6853E994A8597000000B3
:109F6000E780C0EE05E1050AC9B75C4413195A0041
:109F7000A6853E994A8597000000E78020ED19E10B
:109F8000050A4DBFE30C09FA61B7AA8481495DBF98
:109F90001783FFFFE702A3141C452A8481E7930778
:109FA000C5001CC51C44231204001CC09307F00FFD
:109FB00063EDB70093F5F50F228597200000E78049
:109FC00020DD1783FFFF6700C31393940501C1676A
:109FD000C18063F9F500A685228597200000E780FF
:109FE00040E0C5B7C18193F5F50F228597200000A9
:109FF000E78000DAA685228597200000E78040DB15
:10A00000C9B797C7FF1F938767D7884382801C45CE
:10A0100099C797C7FF1F23A3A7D6014582807D5507
:10A02000828097C7FF1F938767D598438347450072
:10A03000484792073E9582801783FFFFE702230A75
:10A04000617100451C183EC6B70780013EC81C1848
:10A050003ECA8357440002CE02D002CC231EF10038
:10A06000834784002A8902D22301F1023C083ED4AE
:10A0700002D697000000E78000FB835705002316F7
:10A08000F10297500000E78060BF2307A1025C4007
:10A0900003556400F18313F717008347F10252055B
:10A0A0005181F99BD98FA307F10297000100E78046
:10A0B000409739CDAA840355050097A00000E7809A
:10A0C00080B783D704002AD26800231CF10083D70D
:10A0D0002400231DF1001C4803D647008C43972021
:10A0E0000000E78000C88347B400CA861756010005
:10A0F000130686618117A305F4006C0048109700D1
:10A100000100E780A0A25D611783FFFF670063FF86
:10A110002155D5BF1C45B1CF03C5A70089461357AC
:10A120006500630BD7028D46630ED7028546630038
:10A13000D702130740063305E50203C7B700418B7A
:10A1400015CB83C7B700BD8B3355F540828013759F
:10A15000F5031307803EC5B709671375F5031307A9
:10A160000771D1BF372709001375F5031307077C63
:10A17000D9B7014582801783FFFFE70243F603A9A1
:10A180008500630C09048347B900AE8493F7070E7A
:10A1900085C303459900930520030D810505B3058B
:10A1A000B5028844610597100100E780A0CB35A077
:10A1B0002E8597000000E78020F62A8419CD9700AD
:10A1C0000000E78020588325C900B307B54063FA33
:10A1D00087002E94B305A440E9F51783FFFF6700BD
:10A1E00043F285457DBF1783FFFFE70243EF2A84D3
:10A1F00003D50500011132C636C43AC22EC002CAC8
:10A2000002CC02CE97A00000E780E0A282452ACAD5
:10A2100022852ECC97000000E780E0E00357050080
:10A22000231EE10097500000E78040A5A246324679
:10A230009247230FA10036874C08B286228501463B
:10A2400097000000E780E0A605611783FFFF670025
:10A2500043EB1783FFFFE70283E861711C183EC6DA
:10A26000B70780013EC81C183ECA3C0800453ED4D2
:10A27000AA8402CC02CE02D002D202D697000000FD
:10A28000E78060DA8357050035592316F1029750AD
:10A290000000E780A09E2307A10209C48357440061
:10A2A00081EB21594A855D611783FFFF670063E5F4
:10A2B000035564005205518197F00000E7806076F5
:10A2C0002A8965D18347B40093F7070E99C7130510
:10A2D000840197100100E78020BB83574400231EB0
:10A2E000F100834784002301F1025C40035509001B
:10A2F000D98313F7070883471102231CA10093F7A2
:10A30000F707D98FA300F10283572900231DF1001D
:10A310005C40F18313F717008347F102F99BD98F53
:10A32000A307F10297A00000E780E0902AD235D978
:10A33000834794006800139757008347B400FD8B50
:10A34000D98FA305F4001C4803D647008C439720FF
:10A350000000E78000A1A687175701001307C73A3E
:10A36000740005464C10268597000000E780609435
:10A370002A890DD98347B400A685FD8BA305F40077
:10A3800097000000E78060DF31BF1783FFFFE7021F
:10A3900003D5832485FE2A84411126859700000079
:10A3A000E78080D7834734FF93F7070E8DCB2AC60B
:10A3B000268597000000E78060C809CD834734FFF9
:10A3C000B245FD8BA309F4FE91C5228597100100CB
:10A3D000E78040A941011783FFFF670083D27DD941
:10A3E0008327C4FF2685829775F5834734FF93F74B
:10A3F000070E91C7228597100100E780E0A803258A
:10A4000084FE97000000E78000E5E9B71783FFFFAF
:10A41000E702E3C99C4141112A8903C70700894724
:10A420002E84935667006380F6040D466388C60445
:10A430009307F0076304F7022E8597200000E7805A
:10A44000C0A2AA848149C16B130C490097C7FF1FA2
:10A450009387C7929C43984763E4E90441011783BB
:10A46000FFFF670083C803D745008547E3F8E7FE91
:10A470002E8597200000E780A0A4E1B703D7450010
:10A48000E3FEE7FC2E8597200000E780009EAA846B
:10A49000228597200000E780609FC204C98C5DB7C9
:10A4A000DC470355A900139A49003E9A931705010A
:10A4B000C187635DF00083570A006397A70263E7D3
:10A4C00074038327CA00034D5A002DA0A16721679A
:10A4D000A98F1307F7EFE374F7FE6397090097005E
:10A4E0000000E780209161FD85098DB783278A00F0
:10A4F000034D4A00835DA90003576900216A138B4D
:10A50000C7003AC6814A33CA4D01631E5D0197C731
:10A51000FF1F938727879C43E1DBA28662868145E4
:10A5200026858297D1B7A1679387F7EF930C4BFFEE
:10A5300063F24703B2455A8597F0FFFFE780A071A9
:10A540000DC103278B00104709CE10436382C4025C
:10A550003107D5BFEE85668597000000E780008F44
:10A5600071F993861A0093FAF60F130B0B0271BF61
:10A57000835644005C43E3E9F6F622853AC6971019
:10A580000000E7808078A1679387D7042A8A035D5B
:10A590004400324763E897008347D90093E707F800
:10A5A000A306F9001C4766852286E2858297C1676B
:10A5B0000844FD17337AFA00529508C02312A4010B
:10A5C00025B71783FFFFE702E3AFAA892E8A8144EC
:10A5D00097BAFF1F938A8A7A83A70A00984763E68F
:10A5E000E4001783FFFF670023B1DC4713944400A6
:10A5F00001493E9413BB140083474400634BF900A8
:10A60000014913BB140083475400634FF9008504CC
:10A61000E1B70844931759005287DA860146A285AC
:10A620003E9582990509C9BF48449317590052873E
:10A63000DA860546A2853E9582990509E9B7178312
:10A64000FFFFE702C3A9814517F5FFFF1305454C3E
:10A6500097B7FF1F2396077297000000E780A0F6C8
:10A660001783FFFF6700E3A997B7FF1F9387077161
:10A670009C4395C31783FFFFE70263A6814517F547
:10A68000FFFF1305E54897000000E780C0F317833C
:10A69000FFFF670003A782801783FFFFE70283A203
:10A6A00037E404008327841241112315E100AE89A9
:10A6B0003289368A3A8681460147ED45AA848297D7
:10A6C0002AC621C90356A100D28597200100E78040
:10A6D000C04A8327C413CE8526858297058905C97C
:10A6E0008327440D2314210101462C0026858297DF
:10A6F0002A8401C9B7E7040083A7C712ED452800E3
:10A700008297228541011783FFFF6700E39E49443A
:10A71000D5B76554FDB75C41FD175CC182801783D6
:10A72000FFFFE702C39BB7E70400FC5F82979547F2
:10A730003305F50281450D811783FFFF6700639C98
:10A740001783FFFFE702A399B7E70400FC5F829736
:10A7500095473305F5020D811783FFFF6700639A64
:10A760001783FFFFE702A397B7E7040083A7870BD0
:10A770000355050082971783FFFF670083981783AF
:10A78000FFFFE702C395035505003287AE86179693
:10A79000FF1F035646D297B5FF1F9385E55E9700CE
:10A7A0000000E780A0EF1783FFFF67008395178302
:10A7B000FFFFE702C392B7E7040083A7C71782979A
:10A7C0001783FFFF6700E3931783FFFFE7022391DF
:10A7D000B7E7040083A7871397B5FF1F9385C55A72
:10A7E000829701451783FFFF6700A3911783FFFF3F
:10A7F000E702E38EB7E7040083A7C71F81451795DB
:10A80000FF1F035545C782971783FFFF6700638FBC
:10A810001783FFFFE702A38CB7E7040083A7871322
:10A8200097B5FF1F93854557829701451783FFFF13
:10A830006700238D1783FFFFE702638AB7E70400F1
:10A8400083A7C71F81451795FF1F0355C5C882976A
:10A850001783FFFF6700E38A1783FFFFE702238860
:10A860002E8597800000E78020AF97800000E7806A
:10A8700020EC1783FFFF6700C3881783FFFFE70201
:10A88000038697800000E78020F61783FFFF6700AC
:10A8900043875C49E1175CC95CC583572501A10763
:10A8A0002319F50083570501A1072318F5008280BD
:10A8B000F1473305F50297B7FF1F9387E74F9C4396
:10A8C0003E9582808D476315F60803D7460085477D
:10A8D00063F0E7081783FFFFE7026380368536845D
:10A8E0002E8997100000E780405829C983574400FB
:10A8F00093140501C18063E397042285971000003B
:10A90000E780A056FD14231294009307A002630071
:10A91000F5029307B0026307F50293079002631FE5
:10A92000F500228597E00000E780C0AB01A8014652
:10A93000CA85228597A00000E780A0AF1773FFFFAC
:10A940006700237C228597100000E7800003FDB795
:10A95000828097B6FF1F938666469C42014599CF39
:10A960009843D44217B6FF1F232AE6446396D700C4
:10A9700097B6FF1F23A6E6441385C7FE8280177390
:10A98000FFFFE702C37597000000E780A04B71440A
:10A9900033058502914597900000E78060E811E556
:10A9A00065551773FFFF6700C37597B7FF1F23A394
:10A9B000A74097000000E780E048330585029145F5
:10A9C00097900000E780C0E561DD97B7FF1F23A5E2
:10A9D000A73E97000000E780E04697B7FF1F23954A
:10A9E000A73C97000000E780E04597B7FF1F239E34
:10A9F000A73A97570100938767D617B7FF1F2329F8
:10AA0000F73A97070000938707E917B7FF1F232F2F
:10AA1000F738014579B71773FFFFE702436CAA8542
:10AA200017B5FF1F1305453897100000E780005B3E
:10AA30001773FFFF6700E36C1773FFFFE702236ADA
:10AA400097000000E78060FD97100000E780805AC3
:10AA500097B7FF1F938787369C4391CF1387C7FE15
:10AA600019CB83D5C7FF17B5FF1F1305A535970071
:10AA70000100E780203F1773FFFF670083681773AB
:10AA8000FFFFE702C36597000000E780C0EC09CD37
:10AA9000834785002A8493F7070499EB0355E50063
:10AAA00097000000E78080F91773FFFF6700636578
:10AAB0008347C5009304450117B9FF1F13090930E7
:10AAC00085E3832709005CC997B7FF1F23A8972E4A
:10AAD00083274900F1FB97B7FF1F23A3972EE9B700
:10AAE000FD172306F500610597800000E78000D67A
:10AAF0008307840063CB07048347840093E707F848
:10AB00002304F400B7E704009C5F82974205A9473D
:10AB100041813375F5028347840093F707FCC98FA1
:10AB20002304F4008347D4003E951C402318A4005E
:10AB300089CF984319CB8347C4005040814585078E
:10AB40003305F502420541810297832709005CC85D
:10AB500097B7FF1F23A497268327490089E797B754
:10AB6000FF1F23AF97248347C4009DDF8355040153
:10AB700017B5FF1F1305052597000100E780802EFC
:10AB800025B71773FFFFE702835597B7FF1F93871A
:10AB9000A7489C4701448583858B85E3AE84B285B5
:10ABA0003A8697100000E780C04A2A8419C597109A
:10ABB0000000E7800041829408CC22851773FFFFD4
:10ABC000670023541773FFFFE702C34F41112E891B
:10ABD00032C6AA8997000000E780C03132471306C9
:10ABE0000502CA86970500009385C5CC17B5FF1FDF
:10ABF0001305851B97000000E780E0F82A8425C92B
:10AC00009304C50097000000E78020411946AA85FB
:10AC1000268597100000E780C0148545268597108B
:10AC20000000E780A010175501001305E5B04E9510
:10AC300083450500268597100000E78060155C4875
:10AC400031468145A1075CC85CC483572401E117E4
:10AC50002319F40083570401E1172318F4001C4C56
:10AC60003E859770FFFFE780804AA3042501228577
:10AC700041011773FFFF670023481773FFFFE702C7
:10AC800003464111AA842EC632C497100000E78003
:10AC9000A035004DB2452246834784000CC050C009
:10ACA00093F7F70393E707042304F4002318040041
:10ACB000268597100000E780C03083479400A9469E
:10ACC0002317A40013D7370005073307D7029D8B3E
:10ACD00085072306F400A306E40083C70401D848CF
:10ACE0008507230FF7FE17B7FF1F1307270D5843DC
:10ACF000232A04009307440129E317B7FF1F2321E8
:10AD0000F70C17B7FF1F232BF70A17B4FF1F130405
:10AD1000640B228597000100E78000071C44858BA7
:10AD20005D8D19E58145228597000100E78080133C
:10AD300041011773FFFF6700C33C1CC317B7FF1F18
:10AD40002320F708D9B71773FFFFE70243399705A8
:10AD50000000938565B7014597000000E78000B0CB
:10AD600001451773FFFF6700C3391773FFFFE70241
:10AD7000033797000000E78080B01773FFFF67007C
:10AD800043388347C500A5E31773FFFFE702233568
:10AD90002A840355E50097000000E78000C821C120
:10ADA0008347840093F7F7FB2304F4001C4091C70A
:10ADB000DC4381C74C400145829797000000E78043
:10ADC00080B917B5FF1F1305E5FF97000100E78065
:10ADD000A00B0355E40097000000E78020C617731E
:10ADE000FFFF6700033282801773FFFFE702232F04
:10ADF00097B7FF1F938787FC97050000938565C869
:10AE000017B5FF1F130505FC23A0070023A20700A9
:10AE100097000100E780E0F41773FFFF6700632EDF
:10AE20001C4D91CFDC4381CF1773FFFFE702232B2B
:10AE30008345070082971773FFFF6700832C82808A
:10AE400097B7FF1F938747FA9C4303C5070082808B
:10AE500097B7FF1F938747F99C4303C5170082806C
:10AE600097B7FF1F938747F89C4303C5270082804D
:10AE700097B7FF1F938747F79C4303C5470082801E
:10AE800097B7FF1F938747F69C4303C5370082801F
:10AE900097B7FF1F938747F59C4303C557008280F0
:10AEA00097B7FF1F938747F49C4303C567008280D1
:10AEB00097B7FF1F938747F39C4303C577008280B2
:10AEC00097B7FF1F938747F29C4303C58700828093
:10AED00097B7FF1F938747F19C4303C59700828074
:10AEE00097B7FF1F938747F09C4303C5A700828055
:10AEF00097B7FF1F938747EF9C4303C5B70011E146
:10AF00001D45828097B7FF1F938707EE9C4303C5BB
:10AF1000C700828097B7FF1F938707ED9C4303C547
:10AF2000D700828097B7FF1F938707EC9C4303C528
:10AF3000E700828097B7FF1F938707EB9C4303D5F9
:10AF40000701828097B7FF1F938707EA9C4303C5D9
:10AF50002701828097B7FF1F938707E99C4303D59A
:10AF60004701828097B7FF1F938707E89C4303D56B
:10AF70006701828097B7FF1F938707E79C4303D53C
:10AF80008701828097B7FF1F938707E69C4303C51D
:10AF9000A701828097B7FF1F938707E59C4303C5EE
:10AFA000B701828097B7FF1F938707E49C4303C5CF
:10AFB000C701828097B7FF1F938707E39C4303C5B0
:10AFC000D701828097B7FF1F938707E29C4388577A
:10AFD000828097B7FF1F938727E19C4303D5C70261
:10AFE000828097B7FF1F938727E09C4303D5E70232
:10AFF00019E11305800C828097B7FF1F9387C7DE86
:10B000009C4303C50703828097B7FF1F9387C7DD63
:10B010009C43C85B828097B7FF1F9387A7DC884358
:10B02000828019E17D558280F5DE984265DFFDD989
:10B0300017B7FF1F130747FE1847AA877155058BDF
:10B04000631D072403C507001547E37DA7FC03C75D
:10B0500037001305F0057D171377F70FE364E5FC60
:10B0600003C35700E30003FC83C86700E38C08FABE
:10B0700003C77700494579171377F70FE364E5FABB
:10B0800003C7A70011481305F7FF1375F50FE36B0E
:10B09000A8F803CE97000D481305FEFF1375F50FB2
:10B0A000E362A8F803C8B7006309080065181378BD
:10B0B000F80F1305600DE36705F703C5C70079486E
:10B0C00079151375F50FE36FA8F403C8D7000D4584
:10B0D0007D181378F80FE36705F503D80701930E81
:10B0E00040175118420813580801E3ED0EF303C846
:10B0F000E7007D181378F80FE36605F303C827010E
:10B100007D181378F80FE36F05F103C88700C54E6B
:10B1100075181378F80FE3E70EF103D86701856E11
:10B12000938EBEE06D18420813580801E3EC0EEF51
:10B1300003D847016D18420813580801E3E40EEFE5
:10B1400003D887017918420813580801E36C05ED0C
:10B1500003C8A7017D181378F80FE36505ED03C553
:10B16000B7011D487D151375F50FE36DA8EA03C5FA
:10B17000D701714879151375F50FE365A8EA03D572
:10B18000E7011308E00F7D1542054181E36CA8E853
:10B1900003C50702494879151375F50FE364A8E85C
:10B1A000C85301C937C834005915130858BFE36B99
:10B1B000A8E603A8870237C53400130555BF591800
:10B1C000E36205E717B5FF1F232EC5C003C60501BF
:10B1D00017B5FF1F232AF5C00545E375C5E403D85D
:10B1E0002501D04933760603E31E06E203C61501A6
:10B1F000E30A06E217B6FF1F2324B6BE83C5270065
:10B2000001466387A50003C61700F1453306B60261
:10B2100083C707039305C00272971A071307C70570
:10B2200016031A9796084697B387B70241553E977B
:10B230003297420741836362E8061773FFFFE70214
:10B2400003EA368597800000E780A06897E0000059
:10B25000E780E06E2A8497A00000E78020092A9406
:10B2600097D00000E780204D2A9497900000E78057
:10B27000A0812A9497F0FFFFE780A0702A9497405E
:10B280000000E78060932A9497700000E780A09CFC
:10B2900022951773FFFF6700C3E682801773FFFFD5
:10B2A000E702E3E34111A307A10097A00000E780B4
:10B2B000A0C59305F100170500001305A5B697F08A
:10B2C000FFFFE7804030014541011773FFFF670032
:10B2D00043E31773FFFFE70203DE17B4FF1F1304F6
:10B2E000A4D30328840079599368180097B4FF1FEA
:10B2F00023A814D31378180063100802BA84BE89F7
:10B30000368B328A2E89AA8A97F0FFFFE780E0AC5D
:10B310007D15269519E531594A851773FFFF67009A
:10B3200003DD97F0FFFFE78040AB7D152695A16711
:10B33000E353F5FE97B7FF1F9387C70098433E8CF2
:10B34000814B01CB014597D00000E780E06A933B39
:10B3500015004A85DA865686D28597900000E780E8
:10B36000C04D2A8911CD1C44F99B17B7FF1F232913
:10B37000F7CA83270C00CDD3E3800BFA829769BF0D
:10B38000268597B7FF1F23AB07C897F0FFFFE7801D
:10B3900080A14146CE8517B5FF1F130565D19710D3
:10B3A0000100E780807D97B00000E78000C00325A2
:10B3B000040B97B00000E780C0C3054597B00000BC
:10B3C000E780C0CA054597000000E78060EDA9B797
:10B3D00097B7FF1F938747C49C47858BEDC71773AB
:10B3E000FFFFE702C3CF17B5FF1F1305A5CA97B725
:10B3F000FF1F23A307C297B7FF1F23A107C297B759
:10B40000FF1F23AF07C097000100E780E0A7975018
:10B410000000E780E0F597F00000E780607397F0A8
:10B420000000E780607997B7FF1F938767BD9C4353
:10B4300091C7054597800000E780402097B7FF1F20
:10B440009387C7A59C4399C741657D1597700000F8
:10B45000E78040A297D00000E780A06497B000008A
:10B46000E78040B697B7FF1F9387C7CB9C431397DE
:10B4700017016356070097D00000E780C0D397B745
:10B48000FF1F23A707C297B7FF1F23A507C297B7C0
:10B49000FF1F23A307C297B7FF1F23A107C297006F
:10B4A0000000E780C08C97000000E780007297F0F2
:10B4B000FFFFE780001997D00000E78000FD1773B9
:10B4C000FFFF670003C4828097B7FF1F9387C7B44D
:10B4D000884382801773FFFFE70263C097800000F4
:10B4E000E780607597800000E780C0771773FFFFE3
:10B4F000670023C11773FFFFE702C3BC2A849304CC
:10B50000140201112E85B289A685214636C63A89D4
:10B5100097100100E78000640DE9B24638082686DE
:10B52000CE851305940497500000E78060412146C2
:10B530002C084A8597100100E780C061133515007B
:10B5400005611773FFFF670023BB0145D5BF177364
:10B55000FFFFE702C3B89305450617B5FF1F1305A4
:10B56000E58897000100E780E08F1773FFFF670011
:10B5700043B91773FFFFE70283B641112EC697F058
:10B58000FFFFE780201CB24588C141011773FFFF10
:10B59000670023B71773FFFFE702C3B2AA842E84A4
:10B5A00097800000E780006CAA8985452285970076
:10B5B0000000E780E07D83C7E4011389940899E3E4
:10B5C00013890403CE85228597000000E780407C24
:10B5D000214693051902228597000000E7806078D4
:10B5E00097B7FF1F938747A38C43228597100000CE
:10B5F000E780C0822146938584022285970000005F
:10B60000E78020761773FFFF670003AF1773FFFF14
:10B61000E70263AA397197D00000E780A0DB9305A9
:10B62000400661E997800000E7800060630205142E
:10B6300097A7FF1F83C7477D13B7170097A6FF1F64
:10B640002384E67C014499CFC16417B9FF1F130915
:10B65000A99C9309400EFD1497000000E7808087A5
:10B660006342A40A97F0FFFFE780C00D4169B72944
:10B670000900096AFD7A2A8B81447D199389F97B37
:10B68000130A0A71938A8AC797000000E7808084B2
:10B6900063D7A4041304400EB387840217B7FF1FB7
:10B6A000130787970324070B3E948357C4016382D3
:10B6B000270B18403307EB4063EAE9008347440057
:10B6C0008507B3874703D6976365F7080146814529
:10B6D000094597F0FFFFE780204FAA8B29E59740A7
:10B6E0000000E780808385476317F50689659385A9
:10B6F000057117A5FF1F1305656F97F00000E78020
:10B70000607695A0B30734030327090BBA9703D7D4
:10B71000C7016308970003C75700A382070023826D
:10B72000E700050415BF9305C500228597000000BA
:10B73000E78080E65E8522869745010093850501B6
:10B7400097F0FFFFE780A0535E8597100000E78029
:10B75000608A850415BF97B7FF1F9387E78B9C47C7
:10B760008D83858BC1F721611773FFFF67002398D5
:10B7700001468545094502D002D202D402D697F08F
:10B78000FFFFE7806044AA8479DD97D00000E7805E
:10B79000A0C31389C4002A8481454A85970000000C
:10B7A000E780005F0C4041464A8597000000E78033
:10B7B000405B832944006385090C4E8502D802DA78
:10B7C00002DC02DE97100100E780A05F2ACE141091
:10B7D00005462C0808184ECC97500000E780E00A78
:10B7E0001375F50F51ED8355840093E525004A85C7
:10B7F00097000000E780E05E11460C104A85970034
:10B800000000E7800056014697450100938585F4C6
:10B81000268597F0FFFFE780804626859700000089
:10B82000E780407D5C40A1D3014685450D4597F0FA
:10B83000FFFFE7806039AA841DD548401389C40002
:10B8400097100100E780E0572AC64A85970000005C
:10B85000E780404C3246636FC5004C404A859700F4
:10B860000000E780005001468145268597F0FFFFE4
:10B87000E780E040268597000000E780A077E5B5E7
:10B8800083558400ADB71773FFFFE702438597A781
:10B89000FF1F938767789C471DC193E7870017A513
:10B8A000FF1F1305A55417A7FF1F232BF77697F04B
:10B8B0000000E78000591773FFFF67008384DD9B5A
:10B8C00017A7FF1F232EF77497300000E780E0646E
:10B8D0007DF117A5FF1F1305655197F00000E78064
:10B8E000A05AD1BF1763FFFFE702E37C4169AA8931
:10B8F0002E8AB28A368BBA8B814417ACFF1F130C89
:10B90000AC71930C400E7D1997F0FFFFE780805CCF
:10B9100063C4A40001443DA03384940383270C0B2B
:10B920003E948357C401638627055A87D68652867C
:10B93000CE851305040397000000E780E0BB01C932
:10B9400023800B0022851763FFFF6700437A83473C
:10B95000F40185C35A87D6865286CE85130594088E
:10B9600097000000E78040B909C585472380FB00A8
:10B97000D1BF850451BF835745006380071E1763FD
:10B98000FFFFE702237401112A8497000000E7807B
:10B99000C04D09C985476309F50605611763FFFFB7
:10B9A0006700837597D00000E780C0A27DF58357BC
:10B9B00044004947ED9BE392E7FEC145228597008D
:10B9C0000000E7804033AA84228597000000E780CA
:10B9D000204F0357440002CE91472A89631AF7008B
:10B9E000228597000000E780A0513C082ACC3ECE7B
:10B9F00097D00000E780409D5C55C5D374084A8607
:10BA0000A6850545829751BF03574400D147E3F609
:10BA1000E7F8032A0400C169014997AAFF1F938A26
:10BA2000AA5F130B400EFD1997F0FFFFE780804AD5
:10BA3000634FA90E2285032A040097000000E780C7
:10BA4000C042A1452A89228597000000E780A02AEC
:10BA5000AA84228597000000E780804A14402A8645
:10BA6000AA8978082685CA8597000000E780C0E784
:10BA7000AA8405D503C7F40189476315F7008347F6
:10BA8000C10181DF5546D2851385640097100100FE
:10BA9000E780A00E014597800000E780C01901C52E
:10BAA00083D7C401A5E797A7FF1F9387E7569C4755
:10BAB00093551900858913D73700058B01CF8983EA
:10BAC000858B6399B70001452EC697000000E7807B
:10BAD000C0DBB2454E8597800000E780601F0346BB
:10BAE000C1012A8493751900268597900000E7808C
:10BAF000E03935C1268597800000E780E01826856B
:10BB000011C0014597800000E780004C973000008D
:10BB1000E780A0408547E312F5E883C75400130788
:10BB2000F00FE38CE7E68507A382F400BDB5B3040C
:10BB3000690383A70A0BBE9483D7C401638B3701C3
:10BB40005546D2851385640097100100E780800078
:10BB500055DD0509D1BD5DD86DB782801763FFFF44
:10BB6000E702435697800000E780000C05C1C164DE
:10BB7000014417A9FF1F1309294A9309400EFD1418
:10BB800097F0FFFFE7800035634EA40017A5FF1F65
:10BB90001305C52597F00000E780A02A1763FFFF73
:10BBA00067008355330534038327090B3E9583577C
:10BBB000C501638897002312050097800000E78085
:10BBC000A00C050475BF97A7FF1F9387E7449C4708
:10BBD0008D83858B8DE31763FFFFE702435017A525
:10BBE000FF1F1305A52097F00000E780E0291763E9
:10BBF000FFFF6700035182801763FFFFE702234EB8
:10BC0000970500009385C5A017A5FF1F1305051E06
:10BC100097F00000E780E0141763FFFF6700634EB2
:10BC20001763FFFFE702A34B8841B7E70400BC5B43
:10BC3000050542054181829709C585472300F50026
:10BC400005051763FFFF6700C34B83C7F5FF2E850C
:10BC50008507A38FF5FE828083C7F5FFFD1793F755
:10BC6000F70FA38FF5FE99EF1763FFFFE702234756
:10BC7000B7E70400BC571385F5FF82971763FFFFF2
:10BC80006700234882801C41035745008D8FBA9579
:10BC90001CC12312B5003E85828093D78500A20582
:10BCA0001441DD8D835745001387E6FF18C18907CE
:10BCB0002312F50013D685004111238FB6FEA38F02
:10BCC000C6FE4101828018419307F7FF1CC18357CC
:10BCD000450085072312F500A30FB7FE8280835726
:10BCE00045008D8F2312F5001C41BE950CC12E8599
:10BCF0008280AA8703D7470008410D8FAA95239217
:10BD0000E7008CC38280184108453305A740828034
:10BD100083574500035765001D8F1C410845338537
:10BD2000A7403305A74082801763FFFFE702233B4C
:10BD300041112EC62A8497000000E780A0FDB2457D
:10BD40006373B50001A0835744000840BE952312D9
:10BD5000B4003E9541011763FFFF6700833A176304
:10BD6000FFFFE702C33741112E84B28532C6970028
:10BD70000000E780A0FB3246A28597100100E78013
:10BD8000C0DF41011763FFFF6700A3371763FFFFA1
:10BD9000E702E3342E84854597000000E78000F930
:10BDA000230085001763FFFF6700A3351763FFFFBC
:10BDB000E702E33241112317B100894597000000E3
:10BDC000E780C0F68347E1002300F5008347F100D8
:10BDD000A300F50041011763FFFF6700833217637B
:10BDE000FFFFE702C32F93D78500A2054111DD8D28
:10BDF0002317B100894597000000E78020F38347AF
:10BE0000E1002300F5008347F100A300F5004101A4
:10BE10001763FFFF6700E32E1763FFFFE702232C82
:10BE20001397850193D78501C166938606F0D98F54
:10BE300013D78500758FD98FA2053707FF00F98DBD
:10BE40004111DD8D2EC6914597000000E78000EE80
:10BE50006C00114697100100E78020D24101176362
:10BE6000FFFF6700032A1763FFFFE70243271C4118
:10BE7000854503C4070097000000E78080E622851F
:10BE80001763FFFF6700E3271763FFFFE702232520
:10BE90001C414111894503C7070083C717002307C9
:10BEA000E100A307F10097000000E78080E303555D
:10BEB000E10041011763FFFF6700A3241763FFFF41
:10BEC000E702E3211C414111894503C7070083C7ED
:10BED00017002307E100A307F10097000000E780A7
:10BEE00040E08357E100410113D58700A2075D8D33
:10BEF000420541811763FFFF6700A3201763FFFF1F
:10BF0000E702E31D0C4141112A8411466800971095
:10BF10000100E78080C69145228597000000E780F8
:10BF200040DCB247C166938606F01397870113D5AC
:10BF30008701598D13D78700758F598DA207370751
:10BF4000FF00F98F5D8D41011763FFFF6700631BE1
:10BF50001C45BE950CC18280AE87944391E6584142
:10BF600001EF0CC15CC1828003C757001367170043
:10BF7000A382E700B687D5B70CC3EDB7AA870841FF
:10BF800019CD1841D44398C36313D500D8C32A8769
:10BF9000034657009376160081E62320070082802F
:10BFA000944381CA8C4203A847008CC36393060163
:10BFB000CCC3799A14C3A302C7003687D1BF1C45EE
:10BFC000DC471D8DB777DBB6938777DB09853305B3
:10BFD000F502420541818280F147B385F50248456B
:10BFE0002E9582808347450085072302F5008280D5
:10BFF0001763FFFFE702A30E2A8409E41763FFFF1C
:10C000006700231083474400F5DBFD1793F7F70F14
:10C010002302F400E5F71C4403D72700050723910A
:10C02000E700DC4399C3228582974C4889CD83473A
:10C030005400898B99E71C4422859C479C439C476C
:10C040008297232A04000040232004007DB7176351
:10C05000FFFFE702C3088357250041112EC681EB7D
:10C060000144228541011763FFFF670083090357DD
:10C0700005008147F146E305F7FEB385D702404549
:10C0800085072E948345440008C4F5F5B247AA8479
:10C0900081E7232A040009A81C456C0022859C43E3
:10C0A0009C43829748C84DDD85472312F400B24770
:10C0B00023200400231804002319F4005C485CC406
:10C0C00083D72400FD172391F40061BF1763FFFF9E
:10C0D000E702E30097A7FF1F938747D388432326F0
:10C0E000050023240500410597F00000E780C0D932
:10C0F0001763FFFF6700E3001763FFFFE70223FEFC
:10C1000017A4FF1F130484D01C40411199CF9C47F2
:10C110002300B5002AC65CC197000000E78040FB01
:10C120001C40DC4399C33245829741011763FFFFEE
:10C13000670023FD0347450029E3584DAA877D5535
:10C140001DCF1763FFFFE70283F91CC3DC4797A6E7
:10C15000FF1F23ADE6CAF156130507012390D70050
:10C16000970500009385050297F00000E78060BF07
:10C1700001451763FFFF6700C3F87D558280828009
:10C180001763FFFFE702A3F501116146814528000F
:10C190009760FFFFE780A0F797A7FF1F938707C768
:10C1A0009C4328009305F00FDC473EC69700000033
:10C1B000E780C0F405611763FFFF670083F497A76A
:10C1C000FF1F9387A7C49C43D847A1679387C702E3
:10C1D000631EF70A397106DE22DC26DA80004AD8AF
:10C1E0004ED652D456D23285B28497000000E780F2
:10C1F000C0C7AA89268597000000E78020C92318B8
:10C20000A4FC268597000000E78040C82319A4FC01
:10C21000268597000000E78060C783D744000A8A1C
:10C22000231AA4FC858393F7F70F230EF4FC8607EB
:10C23000BD0793F7073F3301F1408A8A01498347DD
:10C24000C4FD6367F902CE85130584FC232C54FDDD
:10C2500097000000E78080EA5281130104FCF2504D
:10C260006254D2544259B259225A925A2161828060
:10C27000268597000000E78060C193171900D697C4
:10C2800005092390A7001379F90F55BF828097A75E
:10C29000FF1F9387A7B79C43D847A1679387A7023F
:10C2A000631AF70A397106DE22DC26DA80004AD8E2
:10C2B0004ED652D456D23285B28497000000E78021
:10C2C000C0BAAA89268597000000E78020BCFD57E8
:10C2D0002318A4FC26852319F4FC97000000E780AE
:10C2E000E0BA83D744000A8A231AA4FC858393F713
:10C2F000F70F230EF4FC8607BD0793F7073F3301C2
:10C30000F1408A8A01498347C4FD6367F902CE85FB
:10C31000130584FC232C54FD97000000E78000DE09
:10C320005281130104FCF2506254D2544259B25962
:10C33000225A925A21618280268597000000E78068
:10C34000E0B493171900D69705092390A700137935
:10C35000F90F55BF828097A7FF1F938727AB9C4398
:10C36000D847A16789076310F70A397106DE22DC16
:10C3700026DA80004AD84ED652D456D23285328937
:10C3800097000000E78060AEAA894A859700000008
:10C39000E780C0AF835749000A8A2318A4FC85832D
:10C3A00093F7F70F230CF4FC8607BD0793F7073FBD
:10C3B0003301F1408A8A8144834784FD63E7F402B4
:10C3C000CE85130584FC232A54FD97000000E780E6
:10C3D000E0D25281130104FCF2506254D25442590B
:10C3E000B259225A925A216182804A8597000000F0
:10C3F000E780C0A993971400D69785042390A700DF
:10C4000093F4F40F55BF828097A7FF1F938707A06F
:10C410009C43D847A1679387E704631EF70A3971E5
:10C4200006DE22DC26DA80004AD84ED652D456D216
:10C430003285B28497000000E78020A3AA89268570
:10C4400097000000E78080A42318A4FC26859700AD
:10C450000000E780A0A3231AA4FC26859700000013
:10C46000E780C0A283D744000A8A2319A4FC8583ED
:10C4700093F7F70F230EF4FC8607BD0793F7073FEA
:10C480003301F1408A8A01498347C4FD6367F90299
:10C49000CE85130584FC232C54FD97000000E78013
:10C4A000E0C55281130104FCF2506254D254425947
:10C4B000B259225A925A2161828026859700000043
:10C4C000E780C09C93171900D69705092390A70011
:10C4D0001379F90F55BF828097A7FF1F93870793A2
:10C4E0009C43D847A1679387C704631AF70A397139
:10C4F00006DE22DC26DA80004AD84ED652D456D246
:10C500003285B28497000000E7802096AA892685AC
:10C5100097000000E7808097FD572318A4FC26852C
:10C52000231AF4FC97000000E780409683D744006C
:10C530000A8A2319A4FC858393F7F70F230EF4FCD2
:10C540008607BD0793F7073F3301F1408A8A014907
:10C550008347C4FD6367F902CE85130584FC232C51
:10C5600054FD97000000E78060B95281130104FC7C
:10C57000F2506254D2544259B259225A925A21610D
:10C580008280268597000000E7804090931719006D
:10C59000D69705092390A7001379F90F55BF82801C
:10C5A00097A7FF1F938787869C43D847A167DD071E
:10C5B0006317F7041763FFFFE70263B279713285EF
:10C5C000328497000000E780408A2AC622859700BF
:10C5D0000000E780A08B2311A102228597000000B4
:10C5E000E780A088B2452300A10228089700000038
:10C5F000E780C0B045611763FFFF670083B08280AA
:10C6000097A7FF1F938787809C43D847A16793878D
:10C6100087046317F7041763FFFFE70243AC7971E0
:10C620003285328497000000E78020842AC6228564
:10C6300097000000E78080852311A10222859700E2
:10C640000000E7808082B2452300A10228089700FD
:10C650000000E780A0AA45611763FFFF670063AA97
:10C6600082809797FF1F9387677A9C43D847A1677B
:10C670009387A7046312F7021763FFFFE70223A65D
:10C6800001112800814597000000E78020A705617F
:10C690001763FFFF6700E3A682809797FF1F9387CA
:10C6A000E7769C43D847A167938757026319F7023F
:10C6B0001763FFFFE702A3A20111328597F0FFFF86
:10C6C000E780A07A2308A100814528009700000098
:10C6D000E780C0A205611763FFFF670083A2828025
:10C6E0009797FF1F938787729C43D847A1679387CB
:10C6F000E702631BF7041763FFFFE702439E011184
:10C700003285328497F0FFFFE7804078AA84228543
:10C7100097F0FFFFE7808077854709E9228597F04A
:10C72000FFFFE78080744205B337A00028008145F1
:10C73000231891003ECA97000000E780209C056105
:10C740001763FFFF6700E39B82809797FF1F938724
:10C75000E76B9C43D84799476313F7081763FFFFBC
:10C76000E702E39779713285328497F0FFFFE78023
:10C77000C06F2AC6228597F0FFFFE7802071231043
:10C78000A102228597F0FFFFE780206E2301A1021E
:10C79000228597F0FFFFE780406DA301A10222856B
:10C7A00097F0FFFFE780606C2302A102228597F0DB
:10C7B000FFFFE780806B2313A102228597F0FFFF24
:10C7C000E780A06AB2452314A10228089700000060
:10C7D000E780C09245611763FFFF67008392828004
:10C7E0009797FF1F938787629C43D847A1679387DA
:10C7F000C7036313F7081763FFFFE702438E7971DE
:10C800003285328497F0FFFFE78020662AC62285B2
:10C8100097F0FFFFE78080672310A102228597F041
:10C82000FFFFE780A0662311A102228597F0FFFF9A
:10C83000E780A0632302A102228597F0FFFFE78033
:10C84000C062A302A102228597F0FFFFE780E061AA
:10C850002303A102228597F0FFFFE7800061B24524
:10C86000A303A102280897000000E7802089456102
:10C870001763FFFF6700E38882801763FFFFE7020B
:10C88000038601112A8497F0FFFFE780005EAA84E7
:10C89000228597F0FFFFE780605F228597F0FFFF1A
:10C8A000E780C05E035744008D4763F7E7002285A9
:10C8B00097F0FFFFE780805D228597F0FFFFE7801C
:10C8C000E05C2800A68597000000E78020830561D2
:10C8D0001763FFFF6700E3829797FF1F9387075354
:10C8E0009C43D847A167FD07631FF7001753FFFF5D
:10C8F000E702E37E328597000000E78040F8176387
:10C90000FFFF6700038082809797FF1F9387075080
:10C910009C43D847A167E5076315F7081753FFFF46
:10C92000E702E37B79713285328497F0FFFFE7807D
:10C93000C0532AC6228597F0FFFFE7802055228545
:10C9400097F0FFFFE78080542310A102228597F023
:10C95000FFFFE780A053520551812311A1022285D8
:10C960002302010297F0FFFFE7802050A302A102FB
:10C97000228597F0FFFFE780404F2303A102228525
:10C9800097F0FFFFE780604EB245A303A10228089D
:10C9900097F0FFFFE780807645611753FFFF670040
:10C9A000437682809797FF1F938747469C43D847DB
:10C9B000A1679387E703631FF7001753FFFFE702A1
:10C9C0000372328597000000E78060EB1753FFFF8A
:10C9D0006700237382809797FF1F938727439C43A9
:10C9E000D847A16793874704631EF7021753FFFFD9
:10C9F000E702E36E79713285328497F0FFFFE780BA
:10CA0000C0462AC6228597F0FFFFE7802048B2453E
:10CA1000280897F0FFFFE780606E45611753FFFF1E
:10CA20006700236E82809797FF1F9387273E9C4362
:10CA3000D847A167938787026310F7041753FFFF56
:10CA4000E702E36979713285328497F0FFFFE7806E
:10CA5000C0412AC6228597F0FFFFE7800041B2451A
:10CA60002300A102280897F0FFFFE78020694561B5
:10CA70001753FFFF6700E36882801753FFFFE70249
:10CA80000366011197F0FFFFE780203EAA8528008A
:10CA900097F0FFFFE780806605611753FFFF67008F
:10CAA00043669797FF1F938767369C43D847A167D4
:10CAB000D107631FF7001753FFFFE7024362328578
:10CAC00097000000E780A0FB1753FFFF6700636338
:10CAD00082809797FF1F938767339C43D847A1674E
:10CAE000C507631FF7001753FFFFE702435F328557
:10CAF00097000000E780A0F81753FFFF670063600E
:10CB000082809797FF1F938767309C43D847A16720
:10CB1000B907631FF7001753FFFFE702435C328535
:10CB200097000000E780A0F51753FFFF6700635DE3
:10CB300082809797FF1F9387672D9C43D847A167F3
:10CB4000AD07631FF7001753FFFFE7024359328514
:10CB500097000000E780A0F21753FFFF6700635AB9
:10CB600082809797FF1F9387672A9C43D8478947FE
:10CB70006318F7021753FFFFE7026356011132856E
:10CB800032C897F0FFFFE780402EAA85280097F073
:10CB9000FFFFE780A05605611753FFFF670063564C
:10CBA00082809797FF1F938767269C43D847A1678A
:10CBB0008D076311F7041753FFFFE702435201117A
:10CBC0003285328497F0FFFFE780202A1306610048
:10CBD000AA844C00228597300000E780C0232800FB
:10CBE000A68597F0FFFFE780605105611753FFFFAF
:10CBF0006700235182809797FF1F938767219C438B
:10CC000081CFDC4391CB1753FFFFE702434D82975F
:10CC10001753FFFF6700E34E82801753FFFFE702C1
:10CC2000034C79713C08AE843ED2A165B7070A0077
:10CC30002A843ED448103C08DD053ED636C432C6B0
:10CC40003AC297D0FFFFE780E03412474810BA8518
:10CC500097F0FFFFE780C01332464810B28597F087
:10CC6000FFFFE780E014A2464810B68597F0FFFF6B
:10CC7000E7800012501001478146A685228597D093
:10CC8000FFFFE780805645611753FFFF670063474A
:10CC90001753FFFFE702A34401117C000329C501DC
:10CCA000AE843ECAA165B70707002A843ECC480877
:10CCB0007C00C5053ECE97D0FFFFE780A02D8345C1
:10CCC000D900480897F0FFFFE780800C5008014723
:10CCD0008146A685228597D0FFFFE7800051056138
:10CCE0001753FFFF6700E3411753FFFFE702233F9E
:10CCF00083C7950093F7F707A384F500970000001A
:10CD0000E78040F91753FFFF6700A33F1753FFFF6A
:10CD1000E702E33C79713C08AE843ED2A165B707D7
:10CD200009002A843ED448103C08938545043ED629
:10CD300032C636C497D0FFFFE780C025A246481010
:10CD4000B68597F0FFFFE780A00432464810B28511
:10CD500097F0FFFFE780C005501001478146A68588
:10CD6000228597D0FFFFE780404845611753FFFFBA
:10CD7000670023391753FFFFE702633683C7950027
:10CD800041112A8493F7F707A384F50032852EC654
:10CD900097F0FFFFE780800F85672AC46370F50274
:10CDA00097700000E78020E92246B24509ED11475F
:10CDB0008146228597000000E78060E64101175315
:10CDC000FFFF6700033401478346F501DDB71753C2
:10CDD000FFFFE702232F01113C003ECAB7070A00FC
:10CDE0003ECC3C003ECE83C79500AA89328593F79E
:10CDF000F707A384F5002E8497F0FFFFE780000972
:10CE00008567637DF504A165AA8493858504480838
:10CE100097D0FFFFE7800018268597700000E78015
:10CE200080E12A8929E19145480897F0FFFFE780D2
:10CE300020F6A685480897F0FFFFE78060F7CA85CF
:10CE4000480897F0FFFFE780A0F4014781465008AB
:10CE5000A2854E8597D0FFFFE780203905611753E3
:10CE6000FFFF670063298145480897F0FFFFE780CF
:10CE700020F20349090275BF1753FFFFE70283241D
:10CE800079711C103ECAB7070F003ECC404D1C10F4
:10CE9000AA84AE894808994532C636893ECE97D0D5
:10CEA000FFFFE780200F32464808B28597F0FFFF6A
:10CEB000E78000EE630C0902A545480897F0FFFFE4
:10CEC000E780C0E62546CA8597000100E780E0CAF2
:10CED000500801478146CE85268597D0FFFFE78021
:10CEE000C03045611753FFFF670003218355C4021B
:10CEF000480897F0FFFFE780A0EB0355E402814567
:10CF000005C5854785456301F502C167FD17930592
:10CF1000F00F630BF5007D1597700000E780208E01
:10CF20009305150093F5F50F480897F0FFFFE7808C
:10CF300020E683450403480897F0FFFFE78040E5BB
:10CF400083451403480897F0FFFFE78060E48355AA
:10CF50002403480897F0FFFFE78080E583554403EA
:10CF6000480897F0FFFFE780A0E49DB71753FFFF45
:10CF7000E702E31683C795008146014693F7F7075A
:10CF8000A384F50097000000E78040EF1753FFFFF0
:10CF9000670023171753FFFFE702631479713E847C
:10CFA0001C103ECA2E89B7070F00A1653ECCFD05B7
:10CFB0001C10AA84480842C03AC23ECE36C432C6CB
:10CFC00097D0FFFFE78000FD32464808B28597F012
:10CFD000FFFFE780E0DBA2464808B68597F0FFFF39
:10CFE000E78000DD12474808BA8597F0FFFFE78029
:10CFF00020DC0248630C08029145480897F0FFFFC7
:10D00000E780C0D21146A28597000100E780E0B614
:10D01000500801478146CA85268597D0FFFFE780E3
:10D02000C01C45611753FFFF6700A30D89454808E1
:10D0300097F0FFFFE78080CF834704002300F500CF
:10D0400083471400A300F500E1B71753FFFFE70281
:10D05000630783C7950001112A8A93F7F707A38412
:10D06000F5003285AE8432C697F0FFFFE78000E21C
:10D0700032462A89328597F0FFFFE78000DF856717
:10D080006373F902AA894A8597700000E780A0BA05
:10D090002A8419ED114781464A86A6855285970054
:10D0A0000000E780C0B705611753FFFF6700C304A6
:10D0B0009387E9FF93F7F70F0547E366F7FE83478A
:10D0C000F50195EB8947E380F9FE8346F40152852B
:10D0D00001474A86A68597000000E78040B4A16713
:10D0E000D90748083ECC230A010002CE9700000071
:10D0F000E780A0B04DBF639EE7008947639EF900BB
:10D1000093071020231FF50097700000E780C0B739
:10D110006DBF0947E39BE7FA8D47E398F9FA22854B
:10D1200097700000E78080DF9797FF1F938747ED98
:10D130009C4399E79797FF1F938747D69C4399C7CE
:10D1400003D5040097800000E780A0CE231F0400D1
:10D1500022855DBF1753FFFFE70263F801113C0012
:10D160003ECAB7070B003ECC3C003ECE83C79500BD
:10D170002A89328593F7F707A384F500AE8497F0E8
:10D18000FFFFE780A0D093170501C187635AF0061F
:10D19000A1652A849385E502480897D0FFFFE780C0
:10D1A00060DFA285480897F0FFFFE78060C097978F
:10D1B000FF1F9387A7CE9C43A9EB01449375F40FFF
:10D1C000480897F0FFFFE780A0BC9355844093F593
:10D1D000F50F480897F0FFFFE78080BB93550441A7
:10D1E00093F5F50F480897F0FFFFE78060BA014715
:10D1F00081465008A6854A8597D0FFFFE780E0FE6C
:10D2000005611753FFFF6700C3EF4165854605467B
:10D21000A2857D1597500000E78060BD59DD51055E
:10D2200097E00000E78040B61304400633448502CF
:10D2300071B71753FFFFE70283EA0111B707060032
:10D240003EC683C7950021642A8993F7F707A38414
:10D25000F500AE8428009305A4040AC40AC897D038
:10D26000FFFFE78020D3300001478146A6854A852D
:10D2700097D0FFFFE78060F797E0FFFFE78080151A
:10D2800013049404480822CC230A010002CE97001C
:10D290000000E780809605611753FFFF670063E693
:10D2A0001753FFFFE70203E2C1642A8901449799FB
:10D2B000FF1F938969D6130A8002FD1497E0FFFFD0
:10D2C000E78040C26347A40001451753FFFF670092
:10D2D000A3E2B307440303A7C90ABA9703D7070019
:10D2E0006306970083D72700638427010504F9B7F5
:10D2F0000545E1BF1753FFFFE702C3DC2A8A2E89E9
:10D3000099C123A0050081498144979AFF1F938A00
:10D310006AB0614B97E0FFFFE78000C363C7A400DA
:10D320004E851753FFFF670023DD3384640383A713
:10D330000A003E948357040099E763040900232000
:10D3400089008504C1BF4146D2851305440097007A
:10D350000100E780208075F5A289E5B71753FFFF2C
:10D36000E70243D639717C083ED4B7070A003ED69F
:10D370007C083ED883C795002A8A328593F7F70741
:10D38000A384F5002E8932C697F0FFFFE78000B036
:10D3900085676373F5083246AA84328597F0FFFFEC
:10D3A000E780A0AC8547AA8963E8A706A1659385B5
:10D3B0008504281097D0FFFFE780C0BD26859770B1
:10D3C0000000E78040872A8429ED9145281097F0D6
:10D3D000FFFFE780E09BA685281097F0FFFFE7801E
:10D3E000209DCE85281097F0FFFFE780609A0147C7
:10D3F00081463010CA85528597D0FFFFE780E0DE76
:10D40000A1679387770448183EDC230A010202DEF5
:10D4100097F0FFFFE780607E21611753FFFF6700F1
:10D42000A3CD8145281097F0FFFFE7806096A68581
:10D43000281097F0FFFFE780A0979797FF1F93872B
:10D4400027F09C4381CB22856389090097B00000B7
:10D45000E780004B8345040271B797B00000E78076
:10D460008049CDBF1753FFFFE702C3C583C79500AF
:10D470004111AA8993F7F707A384F5003285AE849A
:10D48000328A97F0FFFFE78060A08567637FF5022F
:10D490002A8997600000E780007A2A84914631C586
:10D4A0008347F50105476387E70291C70D47636628
:10D4B000F704AD461DA89305050303250A00414660
:10D4C00097F00000E78000690DE941011753FFFF65
:10D4D000670083C29305950803250A00414697F02B
:10D4E0000000E7802067814669F54A86A6854E855B
:10D4F00097000000E780C081C9BF83250A0013059B
:10D50000940897700000E780A02919C1C146F1BFB7
:10D510009797FF1F9387C7AE9C4399E79797FF1F85
:10D520009387C7979C4399C7228597800000E7801F
:10D53000208A69FD8547A30FF4002285979000009B
:10D54000E78020AB228597600000E780E0734E857E
:10D5500081464A86A68597F0FFFFE780607BA1673A
:10D560009387570448003EC42302010002C697F087
:10D57000FFFFE780806891BF1753FFFFE702A3B367
:10D5800083C795004111AA8993F7F707A384F50093
:10D5900032852E89B28A97F0FFFFE780208F85675A
:10D5A0006374F50EAA8497600000E780C0682A843F
:10D5B0000DED416B014A979BFF1F938BEBA5130C5D
:10D5C000400E7D1B19A833048A0383A70B0B3E94DE
:10D5D0008357C40163836705050A97E0FFFFE7806F
:10D5E000608FE342AAFE95460DA08357C50163965E
:10D5F00097029305050303A50A00414697F0000032
:10D60000E7804055994611E181462686CA854E85B8
:10D6100097F0FFFFE780C06F85A883A50A00130578
:10D62000040397700000E780A017C14679FD2285AA
:10D63000231E940097900000E780A09B22859760AE
:10D640000000E78060649797FF1F938767CF9C4334
:10D65000A9C323000402228597B00000E7800017C9
:10D660004E8581462686CA8597F0FFFFE780406A8F
:10D67000A1679387070448003EC42302010002C645
:10D6800097F0FFFFE780605741011753FFFF6700E6
:10D6900003A689472300F402E1B7397106DE22DCD4
:10D6A0004AD8800052D456D25AD026DA4ED65ECE10
:10D6B0002E8A32892A8B97D0FFFFE780A07E06054D
:10D6C000710541998A8A3301A140232224FC231445
:10D6D00004FC97D0FFFFE780E07C83479A000605B3
:10D6E000350593F7F7072315A4FCA304FA004A8530
:10D6F000232624FC97E0FFFFE7804079931705017C
:10D70000C1876340F0025681130104FCF250625459
:10D71000D2544259B259225A925A025BF24B2161B9
:10D720008280AA844A8597E0FFFFE7802076AA8955
:10D730004A8597E0FFFFE7806075A1659385C50284
:10D740002A89130544FC97D0FFFFE780A084268533
:10D7500097C0FFFFE780E078854511C94A86CE85EE
:10D7600097C0FFFFE7806072AA8B21E98945130506
:10D7700044FC97E0FFFFE780A061A685130544FC09
:10D7800097E0FFFFE780C062CE85130544FC97E079
:10D79000FFFFE780E061CA85130544FC97E0FFFFC7
:10D7A000E780006101478146130644FCD2855A8513
:10D7B00097D0FFFFE78060A3B9B78145130544FC0C
:10D7C00097E0FFFFE780C05CA685130544FC97E067
:10D7D000FFFFE780E05DCE85130544FC97E0FFFF87
:10D7E000E780005DCA85130544FC97E0FFFFE780F2
:10D7F000205C814497D0FFFFE780C06AE3D4A4FA9D
:10D8000083A70B0113971400BA9783D5070099C516
:10D81000130544FC97E0FFFFE78080598504D9BFDA
:10D82000797106D622D44AD000184ECE52CC56CAB0
:10D8300026D25AC8AE893289AA8A97D0FFFFE780DC
:10D8400060660605690541990A8A3301A140232AC9
:10D8500024FC231C04FC97D0FFFFE780A06483C74F
:10D86000990006052D0593F7F707231DA4FCA38453
:10D87000F9004A85232E24FC97E0FFFFE780006132
:10D8800093170501C187634FF0005281130104FD16
:10D89000B250225492540259F249624AD24A424B3F
:10D8A00045618280AA844A8597E0FFFFE780005E99
:10D8B000A1659385A5022A89130544FD97C0FFFF42
:10D8C000E780406D268597C0FFFFE7808061854532
:10D8D00009C9CA8597C0FFFFE780205E2A8B29E12E
:10D8E0008945130544FD97E0FFFFE780604AA68560
:10D8F000130544FD97E0FFFFE780804BCA851305C1
:10D9000044FD97E0FFFFE780A04A014781461306E8
:10D9100044FDCE85568597D0FFFFE780008DB5B7D3
:10D920008145130544FD97E0FFFFE7806046A6852B
:10D93000130544FD97E0FFFFE7808047CA85130584
:10D9400044FD97E0FFFFE780A046814497D0FFFFAA
:10D95000E7804055E3DBA4FA83270B0113971400FB
:10D96000BA9783D5070099C5130544FD97E0FFFFDB
:10D97000E78000448504D9BF1743FFFFE702237601
:10D9800083474500404DD5EFFD575DC48346940065
:10D9900009476363D70A0346B400854663EEC608A9
:10D9A0008306E40063CA06085C45F9562390D70055
:10D9B0009787FF1F83C7474699E3A304E40097872F
:10D9C000FF1F9387A74D9C4381E78947A306F40077
:10D9D0009797FF1F9387C7969C4381E78947230644
:10D9E000F4009705000093854506AA8413050401F9
:10D9F00097D00000E780E036FD57231AF4028147F4
:10DA00001CDC01489787FF1F23A487409787FF1FCF
:10DA100093874740232E040304C0804397D0FFFF21
:10DA2000E780805261463306C502814522859740D2
:10DA3000FFFFE780C06D81473E851743FFFF67000A
:10DA4000436CFD57D5BF1743FFFFE70243692A84A4
:10DA50000355450297600000E780E01D19E5231E8D
:10DA600004001743FFFF6700C3698357E401F5DB38
:10DA7000930504FF172501001305850797C00000D3
:10DA8000E780A03BF9BF1743FFFFE70243652E89FC
:10DA9000A16541119385E5032A8436C432C6BE844C
:10DAA0003AC297C0FFFFE780E04E12472285BA8551
:10DAB00097E0FFFFE780C02D32462285B28597E0D0
:10DAC000FFFFE780E02EA2462285B68597E0FFFFA4
:10DAD000E780002E630309029145228597E0FFFF4E
:10DAE000E780C0241146A68597F00000E780E00893
:10DAF00041011743FFFF6700C3608945228597E016
:10DB0000FFFFE780A02283C704002300F50083C73E
:10DB10001400A300F500E9BF1743FFFFE702235CF1
:10DB200083C79500444D054793F7F707A384F50095
:10DB30001C42411183C707006367F7062E842A89B8
:10DB4000B1C003C7D400630FF7021787FF1F130785
:10DB5000E734184305C3A386F40097800000E780EC
:10DB6000007183C7D40099E741657D159740000097
:10DB7000E780403083D72403918B89C797C000008A
:10DB8000E780803A4A85A28597F0FFFFE780801002
:10DB9000A167C10748003EC42302010002C697F0F6
:10DBA000FFFFE780800541011743FFFF67006355D2
:10DBB0001743FFFFE702A35203D745008D47AA840E
:10DBC00041112E8432892E8563E3E70297E0FFFF3F
:10DBD000E780C02BAA8523000900268597C0FFFF98
:10DBE000E780A02D41011743FFFF6700835197E0B5
:10DBF000FFFFE780A0292AC6228597E0FFFFE78084
:10DC0000E028B24585472A862300F900268597C07B
:10DC1000FFFFE7808027F9B7397106DE22DC26DABC
:10DC200080004ED652D456D24AD85AD05ECEAE8953
:10DC3000B284AA8A97D0FFFFE780C02506051305A6
:10DC4000250241990A8A3301A140232224FC23148E
:10DC500004FC97D0FFFFE780E02383C79900060507
:10DC60004D0593F7F7072315A4FCA384F900268537
:10DC7000232624FC97E0FFFFE7804021931705014E
:10DC8000C1876340F0025281130104FCF2506254D8
:10DC9000D2544259B259225A925A025BF24B216134
:10DCA0008280AA8B03AB040097C0FFFFE78060234C
:10DCB00051E583D7440001498544F11793B7170014
:10DCC000A301F4FC834734FCA165C9C79385E5042F
:10DCD000130544FC97C0FFFFE780C02BA685130502
:10DCE00044FC97E0FFFFE780A00ADE85130544FCB3
:10DCF00097E0FFFFE780C00B834734FC114691E3B8
:10DD00000946DA85130544FC97E0FFFFE7806005CC
:10DD10008144630A0900416B7D1B97D0FFFFE780B8
:10DD2000601763CCA40201478146130644FCCE85EC
:10DD3000568597C0FFFFE780404BB1B7A685130615
:10DD400034FC97000000E780E0E6933415002A8950
:10DD500086048DBF9385C504A5BF8327C90013978B
:10DD60001400BA9783D5070063886501130544FC46
:10DD700097E0FFFFE780C003850445B71743FFFF27
:10DD8000E702633379711C103EC4B7070F003EC62B
:10DD90001C103EC883C79500AA8A328593F7F707FF
:10DDA000A384F500AE89328497E0FFFFE780000E80
:10DDB00093170501C187635AF0062A8A228597E0E6
:10DDC000FFFFE780A00C2A895285032B040097C02F
:10DDD000FFFFE780001139ED83574400814405447B
:10DDE000F11793B71700A303F10083457100DA8799
:10DDF0002287CA865286280097000000E780E0C884
:10DE0000014781463000CE85568597C0FFFFE780E9
:10DE1000C03DA1679387D70348083ECC230A810001
:10DE200026CE97F0FFFFE78040DD45611743FFFFF7
:10DE30006700E32BA2851306710097000000E780BE
:10DE400060D7AA84094455D13544E30055FB4A857F
:10DE500097F0FFFFE78000450D4441D9014497D07A
:10DE6000FFFFE7802003634DA400C16B0144FD1B4D
:10DE700097D0FFFFE7800002634EA4001544B5B7BA
:10DE8000DC4413171400BA9783D707006383270372
:10DE90000504F1B7D84493171400BA9703D70700C5
:10DEA000631B770123902701268597800000E78078
:10DEB000400201441DBF050465BF1743FFFFE70291
:10DEC000632083C7950041112A8A93F7F707A3843B
:10DED000F50032852E89328497E0FFFFE78000FB52
:10DEE00093170501C1876353F006AA89228597E03D
:10DEF000FFFFE780A0F92311A1004E85832A0400CB
:10DF000097C0FFFFE780E0FD39E583574400854473
:10DF10000144F11793B71700A300F1000348110063
:10DF200003572100D6875285CE862686CA8597F06C
:10DF3000FFFFE7806006A167F10748003EC42302A7
:10DF4000910022C697F0FFFFE78020CB41011743E5
:10DF5000FFFF6700631AA2851306110097000000F7
:10DF6000E78040C52A84894455D983572100116729
:10DF70008544BA97C2071167C1831307F7EFE36FB0
:10DF8000F7F89787FF1F9387A7079C4381CB8545A9
:10DF90001305210097500000E7802075835521006C
:10DFA0002285814497C0FFFFE78040EA25D92310EE
:10DFB0000500228597800000E78000F485B71743AD
:10DFC000FFFFE702430F83C7950041112A8B93F7A8
:10DFD000F707A384F50032852E8A328497E0FFFF8D
:10DFE000E780C0EA93170501C1876351F006AA8A4A
:10DFF000228597E0FFFFE78060E92A895685832B19
:10E00000040097C0FFFFE780C0ED31E5835744006F
:10E0100081440544F11793B71700A301F1000348A9
:10E020003100DE875A854A87D6862286D28597F0C8
:10E03000FFFFE78060F6A167ED0748003EC42302BA
:10E04000810026C697F0FFFFE78020BB4101174300
:10E05000FFFF6700C309A285130631009700000087
:10E06000E78040B5AA8409445DD99167CA97C20781
:10E070001167C1831307F7EF0544E362F7FACA8516
:10E0800097C0FFFFE78080DC014451F9814997D0B8
:10E09000FFFFE78020E163DBA90098489397190010
:10E0A000BA9703D7070005EF2390270197D0FFFF0A
:10E0B000E78040DF1544E384A9F6268597800000B9
:10E0C000E78080E39787FF1F938787F39C43014492
:10E0D000B9D74A8597500000E780C05889B78509AD
:10E0E0007DB71743FFFFE702E3FD79713E847C08AB
:10E0F0003EC82E8AB7071400A1653ECAE5057C0814
:10E10000AA89080836C4428932C6BA8AC6843ECC77
:10E1100097C0FFFFE78000E8CA85080897E0FFFF87
:10E12000E78000C732460808B28597E0FFFFE78026
:10E1300020C8A246630A09049D45080897E0FFFF2E
:10E14000E780C0BE1D4681459740FFFFE78020FC69
:10E1500063890A089145080897E0FFFFE78000BD42
:10E160001146A68597F00000E78020A1100801471E
:10E170008146D2854E8597C0FFFFE7800007456145
:10E180001743FFFF670043F7B685080897E0FFFFD6
:10E19000E78000C21C400808D8439355C701858911
:10E1A00012075183B205D98D97E0FFFFE78040C089
:10E1B0001C40080883C5870097E0FFFFE78040BD4B
:10E1C0001C40080883C5A70097E0FFFFE78040BC1C
:10E1D0001C40080883C5970097E0FFFFE78040BB1D
:10E1E00085BF8945080897E0FFFFE78020B483C713
:10E1F00004002300F50083C71400A300F500BDB799
:10E200001743FFFFE70203EC83C795004111AA897A
:10E2100093F7F707A384F5003285AE84328497E044
:10E22000FFFFE780A0C693170501C187635DF00477
:10E230002A89032A040097C0FFFFE78080CA19E9F2
:10E24000835744000548F11793B71700A307F1005F
:10E25000814631A81306F100A28597000000E780EF
:10E2600060951DC51C459DC783D6470001480347DF
:10E27000F10093078500D2884A86A6854E859700CF
:10E280000000E78040E641011743FFFF6700C3E657
:10E2900009487DBF1D486DBF1743FFFFE70283E2BA
:10E2A00065715C083EC4B7077B013EC65C083EC88A
:10E2B00083C795002A8A328593F7F707A384F50070
:10E2C000AE8997E0FFFFE78040BA8357E100E1C7DE
:10E2D0008945280097C0FFFFE780C0CB8145280013
:10E2E00097E0FFFFE780C0AA97C0FFFFE780A0D1BB
:10E2F0009787FF1F9387C7049C431784FF1F03441E
:10E30000A4B1AA843334800099C31364240097878E
:10E31000FF1F9387A7B89C4399C313644400978752
:10E32000FF1F9387E7CD9C4399C31364840083D573
:10E3300004002800014997E0FFFFE78060A783D52C
:10E340002400280097E0FFFFE78080A683D54400E3
:10E35000280097E0FFFFE780A0A597D0FFFFE780A8
:10E3600060AF93150501C181280097E0FFFFE780AA
:10E3700020A4A285280097E0FFFFE78060A39C44CB
:10E380006360F902014781463000CE85528597C00F
:10E39000FFFFE78080E559611743FFFF6700C3D5A2
:10E3A000DC441314490028003E9497E0FFFFE78007
:10E3B0006096834744000347540089070607BA97CD
:10E3C0008607E36AF5FC835524002800814A97E01C
:10E3D000FFFFE780E09D83454400280097E0FFFFB2
:10E3E000E780009B83455400280097E0FFFFE7800B
:10E3F000209A8347440063C9FA00814A8347540046
:10E4000063C1FA020509A5BF1C4413975A002800EE
:10E41000BA9783D50700850A97E0FFFFE780409908
:10E42000C9BF032BC40093975A0028003E9B835515
:10E430002B00850A97E0FFFFE780809783550B004C
:10E44000280097E0FFFFE780A0964DBF1743FFFF2E
:10E45000E702E3C85C4993E717005CC997800000B6
:10E46000E780E0DC1743FFFF6700A3C91743FFFF06
:10E47000E702E3C62E84814597F0FFFFE780C0E7FF
:10E4800005C583570500FD172310F50009C4835700
:10E4900025002310F40097000000E78060FB014591
:10E4A0001743FFFF6700E3C531457DD82310040003
:10E4B000C5BF1743FFFFE702E3C083C795004111C3
:10E4C0002A8A93F7F707A384F50032852E893284D0
:10E4D00097E0FFFFE780809B93170501C187635694
:10E4E000F006AA89C145228597E0FFFFE780A0805A
:10E4F0002A8B4E85832A040097C0FFFFE780609E29
:10E5000031E983574400231101000544F11793B703
:10E510001700A300F10081440348110003572100B4
:10E52000D6875285CE862286CA8597F0FFFFE78080
:10E53000A0A6A1679387170248003EC4230281006A
:10E5400026C697E0FFFFE780406B41011743FFFFBE
:10E55000670083BA13061100A28597F0FFFFE780DA
:10E560006065AA8409E523110100094475B7930584
:10E5700021005A8597000000E78080EF8357210033
:10E580002A84D9DB9787FF1F938787A79C4381CB7A
:10E5900085451305210097500000E780001583553D
:10E5A00021002685314497C0FFFFE780208A2DD5C2
:10E5B00023100500268597800000E780E093014442
:10E5C000A1BF1743FFFFE70283B141112E896C0001
:10E5D000AA8402C697F0FFFFE78000D20DC103575F
:10E5E000050005072310E50097000000E78040E6DE
:10E5F00081473E8541011743FFFF670083B03247E3
:10E60000954765DBCA85268597300000E780400D79
:10E61000C147E34005FE3244854741462310F400DC
:10E6200083570900A685130544002311F40097E0E1
:10E630000000E7808054228545BF1743FFFFE702B3
:10E6400063A883C795004111AA8A93F7F707A384AB
:10E65000F5003285AE89328497E0FFFFE7800083C2
:10E6600093170501C1876356F0062A8AC1452285A2
:10E6700097D0FFFFE7802068AA845285032B04000F
:10E6800097C0FFFFE780E08531E9835744002311FD
:10E6900001008544F11793B71700A300F10001446E
:10E6A0000348110003572100DA875685D286268653
:10E6B000CE8597F0FFFFE780208EA1679387070242
:10E6C00048003EC42302910022C697E0FFFFE78086
:10E6D000C05241011743FFFF670003A2A285130642
:10E6E000110097F0FFFFE780E04C2A8409E5231131
:10E6F0000100894475B72685930521009700000025
:10E70000E78060ECAA8449FD83552100228597B0FB
:10E71000FFFFE780A07349F5014997C0FFFFE7803D
:10E720006078635DA900184893171900BA9703D75A
:10E7300007000DEF035721002390E70097C0FFFF6C
:10E74000E7804076630625039787FF1F9387478BF3
:10E750009C4399C70355210097500000E78080F043
:10E76000228597700000E78020791DBF050975B7E5
:10E7700095443DB705C19307F00F630FF500C547FA
:10E78000630CF5009307F5FF05453315F5004205C9
:10E79000418182800145828041657D158280B9E991
:10E7A0001743FFFFE702A393034506033284970054
:10E7B0000000E78060FC9305803EB305B502C2050A
:10E7C000C18181CD0357E402854763F8E700130553
:10E7D000040197C00000E780E0688357E4024167C6
:10E7E0007D176385E700FD172317F4021743FFFF2A
:10E7F0006700239182801743FFFFE702C38B00422B
:10E8000083C79500444D0349140093F7F707A38489
:10E81000F50083470400220911673369F900A167F5
:10E82000B347F90041112A8BAE8A63ECE70E8347A8
:10E8300024001307C00EB91793F7F70F6373F7108F
:10E8400003473400C14763EEE70E834744001307D4
:10E85000E00793C707086371F70C83498400834777
:10E860007400A209B3E9F900856763F7F90A034A5E
:10E870006400834754004E85220A336AFA00975099
:10E880000000E780403B61C123962403834B3400A2
:10E89000137AFA00239A34032388740323994403D8
:10E8A00093890401631C090023A60402239804022F
:10E8B0004E8597C00000E780205D3DA003492400FD
:10E8C0004A8597000000E78020EB2397A402834746
:10E8D00044004E85A388F402E38D0BFCE30B09FC96
:10E8E00097C00000E780E05597800000E780C0995E
:10E8F00081460146D6855A8597E0FFFFE78000589C
:10E90000A167938797033EC423020100480002C613
:10E9100097E0FFFFE780602E41011733FFFF67009C
:10E92000037D8544A2862686D6855A8597E0FFFF1B
:10E93000E780C054A167938797033EC423029100E8
:10E94000F1B7BD44C5B79144F1BF1733FFFFE702EC
:10E95000637701111C08404D3EC2B7070F003EC44B
:10E960001C083EC62A89AE8997C0FFFFE78060DB9E
:10E97000585C1C5C6346B70E6394E50063E2A70E27
:10E980003385A740B3B7A700B305B7401306803E51
:10E9900081469D8D97E00000E78040DE93140501DD
:10E9A000C180A1659385C503480097B0FFFFE7804C
:10E9B000605E8145480097D0FFFFE780603D83554A
:10E9C0000404480097D0FFFFE780803E835524046D
:10E9D000480097D0FFFFE780A03D814589CCC16703
:10E9E000FD179305F00F6388F4002685975000000B
:10E9F000E780E0E0AA85480097D0FFFFE780403934
:10EA000003554404814501CDC167FD179305F00FFF
:10EA10006307F50097500000E78060DEAA85480094
:10EA200097D0FFFFE780C03683456404480097D045
:10EA3000FFFFE780E03583457404480097D0FFFF6F
:10EA4000E7800035500001478146CE854A8597B062
:10EA5000FFFFE780807905611733FFFF6700C36917
:10EA6000814481B71733FFFFE702636783C79500CF
:10EA700093F7F707A384F50097000000E78020EDE7
:10EA80001733FFFF6700E3671733FFFFE702836376
:10EA900083C795004111404D93F7F707A384F50014
:10EAA0002A8A3285B284AE8997D0FFFFE780003E84
:10EAB0002A8B268597D0FFFFE780403D2A8926854F
:10EAC00097D0FFFFE780603A93170B0163CA0702F4
:10EAD000E177CA97C207C183116763E3E70293072F
:10EAE0000910C207C1831307B00F637BF7009317A8
:10EAF0000901C187AA8A634AF000C54763FE57012E
:10EB000041011733FFFF6700235F97B0FFFFE780E6
:10EB1000C02DE31725FFD5B763080B026306090272
:10EB2000814463890A02B7077F002310640523111B
:10EB300024057CC0568597000000E780E0C393045D
:10EB4000803EB304950239A0B7077F002320040458
:10EB50007CC081440355240497C00000E78060CA4C
:10EB6000A1C497C0FFFFE780C0BB269593D7F441AF
:10EB700033379500AE97BA9708DC5CDCCE855285BA
:10EB800097000000E780A0DC99E023220404A1673D
:10EB90009387B70348003EC42302010002C697E0F2
:10EBA000FFFFE7808005A9BF814701481CDC232EB9
:10EBB0000403E9B71733FFFFE702635297C0FFFF73
:10EBC000E7808038E1473305F50291459750000012
:10EBD000E78000C5E55711C59777FF1F23ACA72233
:10EBE00081473E851733FFFF6700A351854717779D
:10EBF000FF1F2303F72282801733FFFFE702234E14
:10EC00009777FF1F9387C72080433DC08357040435
:10EC10006390A70683572404639CB7043689B284A3
:10EC200097C0FFFFE780E0AF5C5C63C3B704639508
:10EC3000B7001C5C63EEA7028347640463F3F4002F
:10EC4000A6872303F4048347740463F39700A6871D
:10EC5000A303F4048357440441677D176385E700E9
:10EC600085072312F4043C4481C7CA852685829710
:10EC70001733FFFF6700E3489777FF1F9387471914
:10EC80009C43014599C303C5870082801733FFFF6A
:10EC9000E702E3440111B70707003EC683C79500AA
:10ECA000584D0AC493F7F7070AC8A384F5002A89C8
:10ECB000AE8411CB1C4283C707002304F700977072
:10ECC0000000E780C05A216493055402280097B0E1
:10ECD000FFFFE780202C97000000E78020FAAA853C
:10ECE000280097D0FFFFE780A00A30000147814647
:10ECF000A6854A8597B0FFFFE780204F13044402A2
:10ED0000480822CC230A010002CE97E0FFFFE780EB
:10ED1000C0EE05611733FFFF6700A33E1733FFFF07
:10ED2000E702E33B01117C003ECAB70707003ECC77
:10ED30007C003ECE83C795002E84AA8493F7F70704
:10ED4000A384F500A16593855502480897B0FFFF9D
:10ED5000E780402497000000E78040F2AA85480839
:10ED600097D0FFFFE780C002500801478146A28587
:10ED7000268597B0FFFFE780404705611733FFFF07
:10ED8000670023389777FF1F938787089C430945BF
:10ED900099C303C5970082809777FF1F9387470722
:10EDA0009C43094599C303C5D70082809777FF1F0D
:10EDB000938707069C43014599C303C5A70082803A
:10EDC0001733FFFFE70203300111B70708003EC603
:10EDD00083C79500404D0AC493F7F7070AC8A38478
:10EDE000F5002A89AE8429C41442854703C706006A
:10EDF00063E0E70A83479400094681496380C702BC
:10EE0000B307F740A304E400B339F00083C716004A
:10EE10002305F40097700000E78060450357240342
:10EE2000058B19C76386090097B00000E780C00F03
:10EE3000216493058402280097B0FFFFE7808015C6
:10EE400097000000E78040F4AA85280097D0FFFFD4
:10EE5000E78000F497000000E78080F5AA8528008D
:10EE600097D0FFFFE780C0F2014781463000A685BA
:10EE70004A8597B0FFFFE7804037130474024808C3
:10EE800022CC230A010002CE97E0FFFFE780E0D604
:10EE900005611733FFFF670023261733FFFFE702E3
:10EEA000032401117C003ECAB70708003ECC7C0059
:10EEB0003ECE83C795002E84AA8493F7F707A384D8
:10EEC000F500A16593858502480897B0FFFFE780AC
:10EED000600C97000000E78020EBAA85480897D0D7
:10EEE000FFFFE780E0EA97000000E78060ECAA857A
:10EEF000480897D0FFFFE780A0E950080147814606
:10EF0000A285268597B0FFFFE780202E0561173385
:10EF1000FFFF6700031F9777FF1F938767EF9C43EF
:10EF2000014599C303C5B70082801733FFFFE7028D
:10EF3000031B0111B70707003EC683C79500404D6C
:10EF40000AC493F7F7070AC8A384F5002A89AE8498
:10EF500005C81C42054783C707006368F7060347D7
:10EF6000B400630FF700A305F40097700000E7807A
:10EF700000308347B400B9CF97D0FFFFE78040BE91
:10EF800021649305B400280097B0FFFFE78080005C
:10EF900097000000E78060F8AA85280097D0FFFF5F
:10EFA000E78000DF014781463000A6854A8597B09B
:10EFB000FFFFE78080232904480822CC230A0100B0
:10EFC00002CE97E0FFFFE78040C305611733FFFFE4
:10EFD0006700231397D0FFFFE78020BF55B7173393
:10EFE000FFFFE702C30F01117C003ECAB70707000D
:10EFF0003ECC7C003ECE83C795002E84AA8493F736
:10F00000F707A384F500A165AD05480897B0FFFF99
:10F01000E78040F897000000E78020F0AA854808C4
:10F0200097D0FFFFE780C0D6500801478146A285F0
:10F03000268597B0FFFFE780401B05611733FFFF70
:10F040006700230C9777FF1F938787DC9C43094554
:10F0500099C303C5C70082801733FFFFE702230867
:10F0600001117C00AE843ECAA165B70707002A845F
:10F070003ECCD1057C0048083ECE97B0FFFFE7802C
:10F0800060F197000000E78020FCAA85480897D02F
:10F09000FFFFE780E0CF500801478146A685228523
:10F0A00097B0FFFFE780601405611733FFFF67002B
:10F0B00043051733FFFFE702830283C7950093F7E9
:10F0C000F707A384F50097000000E78020F91733C5
:10F0D000FFFF670003031733FFFFE702A3FE83C7A9
:10F0E00095000329C501411193F7F707A384F500A3
:10F0F0001C4283C90700854763E637079777FF1FE0
:10F10000938707249C432E84AA8485CF9700000010
:10F11000E78080F389476306F502630409028347A9
:10F12000C900638037032306390197700000E78028
:10F13000001483572903898B89C797B00000E780A3
:10F14000A0DE2685A28597000000E78020F1A16758
:10F15000CD0748003EC42302010002C697E0FFFF2E
:10F16000E780A0A941011733FFFF6700E3F8977715
:10F17000FF1F9387E7C99C431D4599C303C5E7005B
:10F1800082801733FFFFE70283F50111B7070700FD
:10F190003EC683C79500584D0AC493F7F7070AC8BF
:10F1A000A384F5002A89AE8415C71C4283C70700D3
:10F1B00093968701E18663C4060685466381D70678
:10F1C0008346E7006388F6002307F7009770000086
:10F1D000E780E00921649305E400280097B0FFFF71
:10F1E000E78040DB97000000E780A0F8AA852800B0
:10F1F00097D0FFFFE780C0B9014781463000A68560
:10F200004A8597B0FFFFE78040FE3504480822CCCE
:10F21000230A010002CE97E0FFFFE780009E056110
:10F220001733FFFF6700E3ED1733FFFFE70223EB20
:10F2300001117C003ECAB70707003ECC7C003ECEE1
:10F2400083C795002E84AA8493F7F707A384F5005B
:10F25000A165B905480897B0FFFFE780A0D39700E4
:10F260000000E78000F1AA85480897D0FFFFE780FB
:10F2700020B2500801478146A285268597B0FFFF3E
:10F28000E780A0F605611733FFFF670083E71733B8
:10F29000FFFFE70223E3AA8401441779FF1F130944
:10F2A00069B7E14997C0FFFFE78000CA6344A40043
:10F2B000014519A833053403832709003E95835778
:10F2C00025006397970011051733FFFF6700C3E21E
:10F2D0000504C9BF032E8500630A0E121773FF1FB2
:10F2E000130303D203230300631503002943639030
:10F2F000061203234E01631503001D436399071093
:10F300001733FFFFE70223DBC689428A3E89BA8AA8
:10F31000B684328BAE8B2A84B5E103554E0019E5D5
:10F3200001431A851733FFFF670063DCA167A98FCC
:10F33000116763FBE70097000000E78080F58145D7
:10F3400097F0FFFFE780C0120844B70700E058417C
:10F35000F98F18455CC1B707001FF98F1CC55C49C0
:10F3600091C7610597C00000E78000B2E38A09FAFF
:10F37000228597700000E78020ED5DB7328597A069
:10F380000000E780006A0D4349DD1C44116703D586
:10F390004700A167A98F63FBE70097000000E780A3
:10F3A00040EF814597F0FFFFE780800C0323840046
:10F3B00093164B01D1828347B300035663008588BF
:10F3C000FD8BA305F300FD777D8E558EFD76FD1632
:10F3D000B204F18E83274301C58E231273012313D8
:10F3E000D3002304530123052301A3044301BDDFFC
:10F3F000228597B0FFFFE78020D2AA850844B5D1C7
:10F40000610597C00000E780E0A58DB71D431A8510
:10F4100082801733FFFFE702E3CA0569AA84AE8939
:10F42000328A0144FD5A7D1997C0FFFFE78080A60C
:10F430006347A40001451733FFFF6700E3CBD844BF
:10F4400093171400BA9703D70700631F370323905D
:10F45000570163070A00268597700000E78060A7C0
:10F460009C449DC383D76700B3F72701639E370190
:10F47000D28801488147014781460146814526855A
:10F4800097000000E78040E5050479BF1733FFFFD0
:10F49000E70243C379711C103EC4B7070F003EC694
:10F4A0001C103EC883C79500AA8A328593F7F707D8
:10F4B000A384F5002E89328497D0FFFFE780009D5A
:10F4C00093170501C187635AF006AA89228597D050
:10F4D000FFFFE780A09B2A8A4E85032B040097B08C
:10F4E000FFFFE78000A039ED8357440081440544C5
:10F4F000F11793B71700A303F10083457100DA8772
:10F500002287D2864E86280097E0FFFFE780E057EB
:10F51000014781463000CA85568597B0FFFFE780D6
:10F52000C0CCA1679387F70348083ECC230A81002B
:10F5300026CE97D0FFFFE780406C45611733FFFF71
:10F54000670083BBA2851306710097E0FFFFE78089
:10F550006066AA84094455D1528597E0FFFFE78091
:10F5600060D40D4459D90546D28526859700000000
:10F57000E78060EA2A8451B71733FFFFE70223B61A
:10F58000835507000346270041112A842E8532C681
:10F590002EC497E0FFFFE780E0D001C93246A245C4
:10F5A000228597000000E78000E741011733FFFF45
:10F5B000670023B51733FFFFE702E3AF83C795006A
:10F5C0004111AA8A93F7F707A384F5003285AE8923
:10F5D000328497D0FFFFE780608B93170501C187C6
:10F5E0006357F00AC1452A8A228597C0FFFFE7804A
:10F5F00080702A8D228597D0FFFFE78020892A8995
:10F60000228597D0FFFFE7804086930705F893F7A0
:10F61000F70F1307E007AA8B637BF706228597D0C5
:10F62000FFFFE78080842A8C228597D0FFFFE78048
:10F63000C083AA8C5285032B040097B0FFFFE7809C
:10F64000408A39E983574400231101008144F117AE
:10F6500093B71700A300F100054403471100835638
:10F660002100938784005685DA8822885286CE85C9
:10F6700097F0FFFFE78020A7A167E90748003EC495
:10F680002302810026C697D0FFFFE7800057410183
:10F690001733FFFF6700A3A513061100A28597E0AB
:10F6A000FFFFE7802051AA8409E5231101000944E6
:10F6B0006DB7930521006A8597F0FFFFE780A0F002
:10F6C0002A8441FD835521009356C9001316490130
:10F6D00085486688E2875E87858A518226859700FD
:10F6E0000000E78060BF2A848DBF1733FFFFE70269
:10F6F000839C83C7950041112A8B93F7F707A38456
:10F70000F5003285AE89328497C0FFFFE78000782C
:10F7100093170501C1876352F00A2A8A228597C090
:10F72000FFFFE780A076AA8A228597C0FFFFE780C7
:10F73000E0752A89228597C0FFFFE7800073930751
:10F7400005F893F7F70F1307E0072A8C6377F7069E
:10F75000228597C0FFFFE7804071AA8C228597C061
:10F76000FFFFE78080702A8D5285832B040097A0CD
:10F77000FFFFE780007739E5835744008544014463
:10F78000F11793B71700A301F10003473100930766
:10F7900084005A85DE882688D6865286CE8597F0E4
:10F7A000FFFFE78040948D4748003EC4230291004C
:10F7B00022C697D0FFFFE780404441011733FFFF87
:10F7C0006700E392A2851306310097E0FFFFE78010
:10F7D000603E2A84894455D99356C90013164901BD
:10F7E00085486A88E6876287858A5182D685970030
:10F7F0000000E78060AEAA8449BF1733FFFFE7022D
:10F80000638C2A8981440144617A916A176BFF1FD6
:10F81000130B0B7F97B0FFFFE780C06863C7A4009E
:10F8200022851733FFFF6700238D832709009399F3
:10F830001400CE9703D507003307450142074183E3
:10F840006364570305C103270B0019C785453E852F
:10F8500097400000E78060E9832709000504CE9700
:10F860002390070085047DB797000000E78060A221
:10F87000832709000504CE972390070065D58145AD
:10F8800097F0FFFFE780C0BEF1BF1733FFFFE7022D
:10F89000638383C7950041112A8A93F7F707A384EE
:10F8A000F50032852E89328497C0FFFFE780005E25
:10F8B00093170501C187635AF004AA89832A0400BB
:10F8C00097A0FFFFE780E06131E58357440085445E
:10F8D0000144F11793B71700A301F1000348310069
:10F8E000D68752850147CE862686CA8597D0FFFFE8
:10F8F000E780806AA167F50748003EC423029100B3
:10F9000022C697D0FFFFE780402F41011723FFFF5A
:10F910006700837EA2851306310097E0FFFFE78032
:10F9200060292A8489445DD99767FF1F9387476DB3
:10F930009C4381CF044997B0FFFFE780A056AA857A
:10F94000268597400000E78040DA13050401970000
:10F950000000E780C0EA228597600000E780C05978
:10F960008144ADBF1723FFFFE702E37483C795000F
:10F970004111AA8A93F7F707A384F5003285AE896F
:10F9800032842311010097C0FFFFE78020509317B6
:10F990000501C1876354F0062A8AC145228597C0B4
:10F9A000FFFFE7804035AA8B5285032B040097A008
:10F9B000FFFFE780005321E9835744008544014459
:10F9C000F11793B71700A300F10003481100035784
:10F9D0002100DA875685D2862686CE8597D0FFFF0E
:10F9E000E780805BA1679387270248003EC423021B
:10F9F000910022C697D0FFFFE78020204101172306
:10FA0000FFFF6700C36EA2851306110097E0FFFF9A
:10FA1000E780401A2A8489444DD99767FF1F93874E
:10FA2000275E98433E8901CF044997B0FFFFE780E6
:10FA30006047AA85268597400000E78000CB130524
:10FA4000040197000000E78080DB97B0FFFFE780AC
:10FA5000604595443DD9930521005E8597F0FFFFF1
:10FA6000E78060B6AA8435F11C480357210022853F
:10FA70002390E70097600000E78000488327090093
:10FA8000A9D70355210097400000E780A0BD35BFEE
:10FA90001723FFFFE702236283C795004111AA8A5B
:10FAA00093F7F707A384F5003285AE89328497C0B7
:10FAB000FFFFE780A03D93170501C1876351F00662
:10FAC0002A8A228597C0FFFFE780403C2A89528519
:10FAD000032B040097A0FFFFE780A04031E5835788
:10FAE000440085440144F11793B71700A301F100C6
:10FAF00003483100DA8756854A87D2862686CE8526
:10FB000097D0FFFFE7804049A167F90748003EC44E
:10FB10002302910022C697D0FFFFE780000E41012B
:10FB20001723FFFF6700A35CA2851306310097E04F
:10FB3000FFFFE78020082A8489445DD99167CA972E
:10FB4000C2071167C1831307F7EF8544E362F7FA31
:10FB50009767FF1F9387C74A9843BE8B01CF04491D
:10FB600097B0FFFFE7800034AA8526859740000004
:10FB7000E780A0B71305040197000000E78020C8C4
:10FB800097B0FFFFE780003295443DD11C482285A5
:10FB900081442390270197600000E780E03583A728
:10FBA0000B00B9D74A8597400000E780A0AB89B722
:10FBB0001723FFFFE702A3522A844105B28497006E
:10FBC0000000E780C0C311C5228597600000E78070
:10FBD000A03281460146A685228597600000E78015
:10FBE00080751C4C89C7DC4799C3228582971723EF
:10FBF000FFFF670003519767FF1F938767219C43AF
:10FC0000014599C31385070182809767FF1F93877A
:10FC10002720884382801723FFFFE702434C931776
:10FC2000C600DD8DC2054111C1812A8432C697C04C
:10FC3000FFFFE780E0173246228511829375F60FA9
:10FC400097C0FFFFE780C01441011723FFFF670043
:10FC5000434B1723FFFFE702E34679713C083ED28E
:10FC6000B7070C003ED43C083ED683C79500AE844F
:10FC70002A8993F7F707A384F500A16593853504D6
:10FC8000481097A0FFFFE780E030C165FD150144F3
:10FC9000176AFF1F130A4A38930A400EAE892E8B4B
:10FCA0002EC697B0FFFFE780E022420593170401BC
:10FCB0004181C183B24563E9A702C167FD1763872C
:10FCC000F500481097C0FFFFE780800E50100147F5
:10FCD0008146A6854A8597A0FFFFE78000514561D0
:10FCE0001723FFFF670043413307540383270A0BA1
:10FCF000BA9703D6C701630A3601638A35014810F3
:10FD000097000000E78060F1DA85050451BFB285F5
:10FD1000EDBF1723FFFFE702033A79717C083EC865
:10FD2000B70711003ECA7C083ECC83C79500AA895C
:10FD3000328593F7F707A384F5002E8997C0FFFF5C
:10FD4000E780C01485676378F504A165AA848905F6
:10FD5000080897A0FFFFE780E02326859740000072
:10FD6000E78060ED133415000A04A285080897C0E7
:10FD7000FFFFE780E001A685080897C0FFFFE78046
:10FD8000200325CC014781461008CA854E8597A0DF
:10FD9000FFFFE780804545611723FFFF670023359C
:10FDA000B30754030327CA0ABA9703D70700631C93
:10FDB000970003D6270063806505080897000000B8
:10FDC000E780A0E5DE8505042EC697B0FFFFE7803B
:10FDD00060114205931704014181C183B245E3E1FB
:10FDE000A7FCC167FD17E38FF5F8080897C0FFFF70
:10FDF000E78000FC41BFB285F9B7C165FD1501443C
:10FE0000176AFF1F130A4A21930A80022E8BAE8BBA
:10FE100065BF1723FFFFE702832C184183471700B4
:10FE200083460700A207D58FD207D1832390F50020
:10FE300083472700034717008D45A207D98F918379
:10FE40002310F60097C0FFFFE780A0E91723FFFF0C
:10FE50006700232B1723FFFFE702C326C164014479
:10FE60001769FF1F1309491B93098002FD1497B0FE
:10FE7000FFFFE78020076347A40001451723FFFF2A
:10FE800067008327330534038327C90A3E958357C8
:10FE90000500E38597FE0504D9BF1723FFFFE7029E
:10FEA00063222A8AAE89B284B68A97400000E7802E
:10FEB00080D819E591473E851723FFFF6700C323CC
:10FEC0002A894E8597A00000E780A0B52A84638E1A
:10FED0000A048D476DD103570500C547E31D47FD53
:10FEE0000347F9018546AD47E317D7FC8347450033
:10FEF00081CF4146A6855D0597D00000E78080C58B
:10FF0000814755D9AD4745BF130965012302E50077
:10FF1000CA85268597100000E780606231C1A54739
:10FF2000E38B0AF82302040079B705C18357050063
:10FF3000E39247F94146A685190597D00000E7806E
:10FF400060C181472DD99947BDB74E859700000004
:10FF5000E78080F02A84954739DD130955004DBFAD
:10FF60004146A685231044012311340113051900CD
:10FF700097D00000E78060C0228597600000E7808E
:10FF8000601181470DBF1723FFFFE7024315797109
:10FF90007C003ECCB7070A003ECE7C003ED083C733
:10FFA0009500B2842E8493F7F707A384F500130617
:10FFB000A1002A892C00268597000000E780A0E593
:10FFC000A16528088D0597A0FFFFE780A0FC904061
:10FFD0008355A10003558100854697000000E78006
:10FFE00000ECAA84AA85280897C0FFFFE78040DAC2
:10FFF0000356A10083558100280897000000E78080
:020000040001F9
:10000000C0C1300801478146A2854A8597A0FFFFFD
:10001000E780A01D854748103ED42302910202D6F6
:1000200097D0FFFFE78060BD45611723FFFF6700A2
:10003000430D1723FFFFE702830A79717C003ECC52
:10004000B7070A003ECE7C003ED083C79500B2843D
:100050002E8493F7F707A384F5001306A1002A89DD
:100060002C00268597000000E780E0DAA1652808CB
:100070008D0597A0FFFFE780E0F190408355A10038
:1000800003558100814697000000E78040E1AA8483
:10009000AA85280897C0FFFFE78080CF0356A100FC
:1000A00083558100280897000000E78000B73008DA
:1000B00001478146A2854A8597A0FFFFE780E012AD
:1000C00048102302910202D402D697D0FFFFE780A6
:1000D000C0B245611723FFFF6700A3021723FFFF8C
:1000E000E702E3FF97000000E78060DB1723FFFFD4
:1000F000670023019767FF1F9387C7D188438280DA
:100100001723FFFFE702A3FD835725004111AE84AB
:100110002A842307B10017F5FFFF130525466C005D
:100120002316F10097A0FFFFE780E04991C42285E4
:1001300097600000E780A0FDFD572310F400130630
:1001400020028145130554009720FFFFE78020FC23
:1001500041011723FFFF6700C3FA1723FFFFE702E0
:1001600063F679717C003ECCB7070A003ECE7C0076
:100170003ED083C79500AA89AE8493F7F7073285EE
:10018000A384F5001306A1002C0097000000E7806F
:1001900080C803558100114497400000E780A0A962
:1001A00015C50355A100014497A00000E7806087B2
:1001B00011CD035705008357810045446318F700AC
:1001C000854597000000E780E0F30144216993052D
:1001D0003900280897A0FFFFE780C0DBA285280828
:1001E00097C0FFFFE780C0BA0356A1008355810086
:1001F000280897000000E78040A2300801478146A8
:10020000A6854E8597A0FFFFE78020FE48104AD4C0
:100210002302810202D697D0FFFFE780009E45614E
:100220001723FFFF670043ED1723FFFFE70283E972
:100230009767FF1F9387C7BD2A8488432E8915C5FA
:10024000035745038357C4016311F70223260502B0
:1002500023180502410597B00000E780E0C263065D
:10026000090097600000E780200281449769FF1F22
:10027000938989DA130A800297B0FFFFE78080C66E
:1002800063C4A4049767FF1F938747C19C4399C722
:100290000355C40197200000E780C0BD6307090033
:1002A000228597600000E78080C71306400E8145D5
:1002B00022859720FFFFE78080E5FD57231EF4008D
:1002C0001723FFFF670043E33385440383A7C90A6D
:1002D0003E95035705008357C4016317F700CA858D
:1002E00097000000E78000E2850479B71723FFFF3D
:1002F000E70243DD83C795004111AA8993F7F70709
:10030000A384F5003285AE8497C0FFFFE78000B874
:1003100085676378F5042A8997400000E780A091FB
:10032000014401CD83D7040031446388270185450A
:1003300097000000E78080EF01444E85A2864A8640
:10034000A68597D0FFFFE780A09CA167938717043D
:1003500048003EC42302810002C697D0FFFFE78019
:10036000C08941011723FFFF670003D91723FFFF4F
:10037000E70243D59767FF1F938787A9804329C466
:10038000014597A00000E780C04781470148C1644C
:100390001CDC232E0403232004041769FF1F130908
:1003A000A9C701449309400EFD1497B0FFFFE780F1
:1003B00060B2634FA400814517F5FFFF1305857FE9
:1003C00097A0FFFFE78020201723FFFF6700C3D21D
:1003D000330534038327090B3E958357C501638793
:1003E0009700854597000000E78040E4050475BF4D
:1003F0009357050113D78700A380F50093170501D4
:10040000C183A1832380E5002381F500A381A5009A
:1004100082801723FFFFE70283CC2300050083C7F8
:100420001500A300F50083C725002301F50083C74D
:100430003500A301F50083C745002302F50083C7FB
:100440005500A302F50083C7650093059500A3033B
:1004500005002303F5002304050032859700000002
:10046000E78040F91723FFFF6700A3C91723FFFFA9
:10047000E70243C54111E9540DCD85CD93F9C5FF80
:100480002E842A89AA84338AA900B7EA0400631853
:100490009A020D88854411CCB7E704009C5F8297CF
:1004A0002AC622866C003305390197C00000E78018
:1004B000C06C268541011723FFFF6700E3C383A7B4
:1004C0008A039104829793170501C183A183A38EA8
:1004D000F4FE93570501238FF4FEA183238EA4FE1F
:1004E000A38FF4FE6DB763E6D5021723FFFFE70283
:1004F00003BFB28741113686BE8536C697C000005D
:10050000E780A067B246410136851723FFFF6700E9
:1005100043BF814636858280838705001387F500B7
:100520003D05FD8793F77708834607007D1586060E
:10053000B58FA300F5006307B7007D178347170049
:100540009D83DDB782801723FFFFE70243B9B7E73A
:10055000040083A7070932872A863A8582971335D4
:1005600015001723FFFF6700C3B915C181478DC16F
:100570001723FFFFE702A3B6414697C00000E780BC
:10058000C05F85473E851723FFFF670083B781471C
:100590003E8582801DCD1723FFFFE70243B441460D
:1005A00081452A849720FFFFE78060B64146814558
:1005B000130504039720FFFFE78060B50147C1677B
:1005C0002322040438C87CC805451723FFFF6700B1
:1005D00043B30145828081473DCDB5CD1723FFFF51
:1005E000E702E3AFB2842E891306800581452A8491
:1005F0009720FFFFE780A0B1CA8524C42685970015
:100600000000E780C0F64146814522859720FFFF24
:10061000E780E0AF3044A285228597000000E780A4
:10062000C0F293040401A285268597000000E780AC
:10063000E0EEA6851305040297000000E78000EEB7
:10064000228597000000E78020F585473E85172327
:10065000FFFF670003AB3E8582801723FFFFE702A1
:1006600063A64111E9540DCD85CD93F9C5FF2E84C4
:100670002A89AA84338AA900B7EA0400639844034C
:100680000D88814411CCB7E704009C5F82972AC68D
:1006900022866C003305390197C00000E780E04DE9
:1006A000268541011723FFFF670003A583A78A035F
:1006B0009104829793170501C183A183A38EF4FE51
:1006C00093570501238FF4FEA183238EA4FEA38FED
:1006D000F4FE6DB765CD1723FFFFE702A39EB2843A
:1006E00011E605451723FFFF670003A12A842E8921
:1006F0000145EDD93C487848B3E6E700E5D6938656
:10070000F7FFB3B7F6007D17032A4404BA9734C83D
:100710007CC863050A06C14913050A03B389494128
:100720002295637D3601B2862E86A685970000004D
:10073000E780A0DB7C40BE9464C065B7CE862E8681
:10074000CE8597000000E78040DAC114D2944E991C
:1007500023220404A2879306040103C7070003C6EB
:1007600007038507318FA38FE7FEE398F6FE304439
:10077000A285228597000000E78020DD2699C149E7
:100780003306994063EC9900A9DCA686A68513057B
:10079000040397000000E78040D579BF8147B30686
:1007A000F4003307F6000347070083C506008507FA
:1007B0002D8F2380E600E39437FF3044A285228505
:1007C00097000000E78060D8C1145DBF01458280BA
:1007D0000DC11723FFFFE7028390130680058145B3
:1007E0009720FFFFE780A09205451723FFFF6700D2
:1007F000439101458280814749C5C1C51723FFFF49
:10080000E702E38DFC4141462E84AA846399C70424
:1008100013860501A2878146C14503C7070003C5AA
:1008200007038507298F3305D60003450500850694
:10083000298FA38FE7FEE392B6FE3044A28526857A
:1008400097000000E78060D0228597000000E780D5
:1008500060F885473E851723FFFF6700838A13856D
:1008600007031D8E814522959720FFFFE780208A90
:100870007C40130700F813060402A2972388E702BE
:1008800051BF3E8582801723FFFFE70243856D71CC
:100890002E84B284AA859010280036899700000023
:1008A000E780A0D309EDD55725A050400C40280083
:1008B00097000000E78040E27DD5FD142104F5F4A7
:1008C0002C004A8597000000E78020F3814761DD16
:1008D0003E8551611723FFFF6700A3821713FFFFB7
:1008E000E702E37F41112EC432C62C000546970073
:1008F0000000E78080F941011723FFFF6700638054
:100900001713FFFFE702A37D01112A842EC602C838
:1009100002CA02CC02CE97C00000E780804AB246ED
:100920002A86A285080897000000E78060FB1375FF
:10093000F50F05611713FFFF6700A37C1713FFFF77
:10094000E702E3797971B2872A8421462308B1004E
:1009500013051101BE853AC436C697C00000E78072
:10096000C021B24693059101368597000000E780CB
:1009700060A82285141035460C0897000000E78017
:1009800020F62A84224701E921460C103A8597C0B7
:100990000000E780801E228545611713FFFF670076
:1009A00043761713FFFFE70283737171AE84AA8544
:1009B0000A85328497000000E78060BB11C90A866F
:1009C000A685228597000000E78020B8814711E1C5
:1009D000C5473E854D611713FFFF670083721713EC
:1009E000FFFFE702C36C1D712A8AB289BE843546B7
:1009F0008547130511012E8CB68A3A8BC28C468D21
:100A00002308F10097C00000E780201710100C08A1
:100A10005285231F010097000000E780C0F82A8458
:100A20003DEDA1476313FD089307900591E0E5476D
:100A30003546E2851305110113990A012308F100D7
:100A40001359090197C00000E7802013135789004C
:100A500093978A00D98F90080C085285231FF100C4
:100A600097000000E78020F42A8415E9A1E4938729
:100A7000FA0091831379F9003EC6631309004149D6
:100A8000668B8144C14B854DB247639F970C6A8644
:100A90008C0033855C0197C00000E780000E228542
:100AA00025611713FFFF6700436493079004C9F0A3
:100AB000A547BDBF834701050947C14B2308F10086
:100AC00083471105A58FA308F10093872400814473
:100AD00063E1FB04014714083386E6008C08B38603
:100AE000E400BA95DA9683C6060083C505000507BB
:100AF000AD8E2300D600E390E7FE4147639CE704F8
:100B000090080C08528597000000E780C0E925D1C5
:100B100081A0B3069B00BA871008B305F6009008C1
:100B20003E9603C506000346060085078506298E06
:100B30002380C500E39277FF998F90080C085285B7
:100B4000BE9497000000E78000E68947014749D13D
:100B50002A84B1B790083E96034606001408BE9654
:100B60002380C600850759BFB24785046387971461
:100B700081471808B306F70098083E973386F900B6
:100B800003470700034606008507318F2380E600F0
:100B9000E39177FF90080C08528597000000E780EA
:100BA00080E05DF53546E285130511012308B101AA
:100BB00097C00000E78060FC13970401418393977E
:100BC00084002183D98F10180C085285231FF1004F
:100BD00097000000E78020DD25FD8147101833874E
:100BE000F9003E960347070003460600B306FB00E4
:100BF0008507318F2380E600E39277FF65A8180808
:100C0000B306F70098083E973386F90003470700BC
:100C1000034606008507318F2380E600E3E127FFC6
:100C2000CA87639E770990080C08528597000000D8
:100C3000E78060D711FD81479800B306F700900860
:100C400018103E973E9603470700034606008507A7
:100C5000318F2380E600E39177FF3546E285130567
:100C600011012308B10197C00000E78000F113973C
:100C700004014183939784002183D98F10180C08B5
:100C80005285231FF10097000000E780C0D1E311D7
:100C900005EC814710183387F9003E96034707009B
:100CA00003460600B306FB008507318F2380E6006C
:100CB000E3E227FFC109410BC1BB814785B7940817
:100CC000BE9683C6060018083E972300D700850706
:100CD00089BF638006321713FFFFE702433D597156
:100CE0002A84BE89B28B85473546130511022E8BA7
:100CF000468C4289BA8A368A2300F10297C00000E6
:100D0000E780A0E710180C10228523170102970036
:100D10000000E78040C963180512A147631FFC0665
:100D20009307900563930900E5473546DA85130577
:100D3000110293140A012300F102C18097C0000040
:100D4000E780A0E393178A0013D78400D98F900817
:100D50000C1022852317F10297000000E780A0C441
:100D60007DE1639209049307FA00BD88918391E0C5
:100D7000C144C207C183DE8C814A3EC6414DB247A1
:100D800063E2FA0E6286B3854B01881097C00000BB
:100D9000E78040DC4DC93D557DA093079004E39664
:100DA00009F8A54759B7834701050947C14C2300F6
:100DB000F10283471105B3C7F900A300F10293873D
:100DC0002900814963E1FC04814618103306D700ED
:100DD0008C083387D900B69556970347070083C51B
:100DE000050085062D8F2300E600E390D7FE4147DE
:100DF0006390E70690080C10228597000000E780BA
:100E000080BA35D189A0B3863A01BA871010B305EC
:100E1000F60090083E9603C50600034606008507C7
:100E20008506298E2380C500E39297FF3387EC4027
:100E300090080C102285BA9997000000E780A0B6B0
:100E40008947014741D165611713FFFF6700E32917
:100E500090083E96034606001410BE962380C600F6
:100E6000850779B7B247850A93990A01939D8A004D
:100E700093D909016391570F85473546DA851305E4
:100E800011022300F10293D9890097C00000E78086
:100E9000C0CEB3ED3D0190000C1022852317B103A5
:100EA00097000000E78020B059FD8147A68963EADA
:100EB000970626860C084A8597C00000E780E0CB9D
:100EC00081471810B306F700100898083E973E9621
:100ED00003470700034606008507318F2380E6009D
:100EE000E3E197FE639FA90590080C102285970007
:100EF0000000E78040AB21F981479810B306F70066
:100F0000900818183E973E960347070003460600D0
:100F10008507318F2380E600E391A7FF4109C10CCB
:100F2000B9BD18089000B306F7003E963387FC0061
:100F300003470700034606008507318F2380E6003C
:100F4000B5B798084E97034707001C10CE9723802B
:100F5000E700850941BF85473546DA85130511024B
:100F60002300F10293D9890097C00000E780E0C018
:100F7000B3ED3D0190000C1022852317B1039700BB
:100F80000000E78040A2E31005EC814718089000BC
:100F9000B306F7003E963387FC000347070003467D
:100FA00006008507318F2380E600E391A7FF4146C5
:100FB0000C084A8597C00000E78020BC81471810C4
:100FC000B306F700100898083E973E9603470700BF
:100FD000034606008507318F2380E600E391A7FFD3
:100FE00090080C10228597000000E780C09B1DD55B
:100FF00099BD7D5582801713FFFFE702430E011153
:101000002A842E8593055100328902C002C202C48F
:1010100002C69304740097F0FFFFE780A03D1D46D1
:10102000A6851305910097C00000E78000B5100861
:101030008A854A8597000000E780E09619ED9307BE
:101040001400180883C60700034607008507050734
:10105000B18EA38FD7FEE397F4FE05611713FFFF50
:101060006700230A1713FFFFE702C3052E848C4194
:101070004111AA89838715003289914463D30700FF
:10108000A1449757FF1F9387A72B9C43A1C7C1CAB1
:101090008D472310F10083C725004A852301F10005
:1010A00083C73500A301F10083C745002302F10087
:1010B00083C75500A302F10083C765009305910023
:1010C000A30301002303F1002304010097F0FFFFB5
:1010D000E78040320C404A860A8597F0FFFFE780A0
:1010E00080330328040083564400A6881D088147E6
:1010F0000147E51642868A854E8597000000E78005
:10110000408E2A8919E5A685228597B0FFFFE780E2
:10111000E0C14A8541011713FFFF6700E3FD4A86DE
:101120000A8597F0FFFFE780002F6DB71713FFFFC9
:10113000E70243F92E848C414111AA898387150067
:101140003289914463D30700A1449757FF1F9387C7
:10115000271F9C43A1C7C1C68D472310F10083C739
:1011600025004A852301F10083C73500A301F10062
:1011700083C745002302F10083C75500A302F10095
:1011800083C7650093059100A30301002303F100C9
:101190002304010097F0FFFFE780C0250C404A863A
:1011A0000A8597F0FFFFE780002783564400032855
:1011B00004008A85858EC2061D08C1822312D400D0
:1011C000A68881470147E51642864E8597000000B4
:1011D000E78060B041011713FFFF6700E3F14A8623
:1011E0000A8597F0FFFFE78000234DBF1713FFFF2D
:1011F000E702E3EEB335B000011185052A89131526
:10120000F601336515012308B100930511013684F9
:101210003AC632C03EC442C297F0FFFFE780801D4D
:10122000A2471248425593D68700230BF10093053D
:10123000910193578800A30AD100A30BF100230C5E
:10124000010197F0FFFFE780E01A324702460328CA
:101250000400B337E000835644009207914411C262
:10126000A1444A85A68842860C0897F0FFFFE780D4
:1012700040772A8919E5A685228597B0FFFFE78088
:10128000E0AA4A8505611713FFFF670083E717137C
:10129000FFFFE70223E301113EC68647B335B000E6
:1012A0008505AA891315F6015D8D2308B100930504
:1012B000110136843A89B28442C446C297F0FFFFD6
:1012C000E780401322489248164593578800A30AA6
:1012D000F1009305910193D78800230B0101A30B23
:1012E000F100230C110197F0FFFFE780A0103247B7
:1012F000104083564400B337E000920703280900EA
:10130000914891C0A1480C084E8597000000E780E5
:10131000809CAA8401E9835544004A8597B0FFFF69
:10132000E780C0A0268505611713FFFF6700C3DCB7
:10133000AA959307F00F17E700001307E77E6317DE
:10134000B50013C5F7FF1375F50F828005058346B9
:10135000F5FFB58FBA9783C70700D5B70357450088
:1013600014419307F00F17E600001306E67B36974B
:1013700042074183139506014181631BE500AD8F50
:10138000B29703C50700130515F3133515008280C6
:10139000850603C5F6FFA98FB29783C70700D9BF9B
:1013A0001713FFFFE702A3D3B28736842E86BA86CF
:1013B000AA853E85BA8497F0FFFFE7806052634FAD
:1013C0000500228597C00000E780A09F2A86A68698
:1013D000A285268597F0FFFFE78080501713FFFF57
:1013E000670023D21713FFFFE702C3CD5D712A8B7D
:1013F000AE8A17E500001305A5702C00B284368A6A
:10140000BA893E8997F0FFFFE780C04F2A845DE1EB
:1014100034104146DA85280097F0FFFFE780404C02
:101420002A8449E98547A303F100A6C29307710006
:101430002408BEC4A68685470D462C18281002DC59
:1014400002DED6C0BEC697F0FFFFE78000442A84C4
:1014500035E183477102A6860D4693F7F70723000F
:10146000FA00C1473EDE2C188947281026DCA3036A
:10147000F10097F0FFFFE78040412A8405ED4146E7
:10148000A6854E8597B00000E780206F8D47A68621
:101490000D462C182810A303F10097F0FFFFE780FA
:1014A000C03E2A8401E94146A6854A8597B00000DE
:1014B000E780A06C228561611713FFFF6700C3C33B
:1014C0001713FFFFE702A3C197D700009387C7C494
:1014D000984383C7470079712A89AE8417E50000D5
:1014E000130585620C083AC42306F10097F0FFFF4C
:1014F000E78040412A8405ED14104146CA8508085A
:1015000097F0FFFFE780C03D2A8415E114081546D7
:101510002C00081097F0FFFFE780803C2A8401E947
:1015200021462C08268597B00000E78000652285BB
:1015300045611713FFFF6700C3BC1713FFFFE702E6
:1015400003BA97D70000938727BD9C477971AA8477
:101550002E8417E500001305A55B0C083EC697F026
:10156000FFFFE780203A0DE914104146A6850808E0
:1015700097F0FFFFE780C03605E1140811466C00C4
:10158000081097F0FFFFE780A03519E58347F101C8
:1015900093F7F7032300F40045611713FFFF67007B
:1015A00043B61713FFFFE70283B33688A14881478C
:1015B0000147E54697F0FFFFE780A0421713FFFFC2
:1015C000670023B41713FFFFE70263B13688A14811
:1015D00081470147E54697F0FFFFE780C06F17138B
:1015E000FFFF670003B21713FFFFE70243AF0111CC
:1015F0002A842E850C0832C697F0FFFFE7808030E2
:1016000009ED324797E600009386064F1008C14562
:10161000228597000000E780E0D805611713FFFFDF
:10162000670023AE1713FFFFE70263AB4111C14709
:101630002EC032C48A8509463EC23EC697F0FFFFDF
:10164000E780A02441011713FFFF670083AB171346
:10165000FFFFE702C3A84111AE8613061009AA8551
:101660000A8502C002C202C402C697F0FFFFE780EB
:10167000202741011713FFFF6700A3A81713FFFFDF
:10168000E702E3A5328797E600009386E6482E86B8
:101690009305000297000000E780C0D01713FFFFFA
:1016A000670023A61713FFFFE70263A37971C14701
:1016B0002ACC2ED032D42C080D4628003ECE3ED265
:1016C0003ED602C402C602C802CA97F0FFFFE780F6
:1016D000C01B45611713FFFF6700A3A21713FFFF8D
:1016E000E702E39F0111AA842E8417E50000130589
:1016F00025438A8597F0FFFFE780C02015E5140891
:101700004146A6850A8597F0FFFFE780601D09ED39
:101710008347E1010347F101A207D98FCA07C983B3
:101720006177D98F2310F40005611713FFFF67005D
:10173000439D15CD1713FFFFE702639A9747FF1FDD
:101740009387C77190439745FF1F93856571174530
:10175000FF1F1305A56C97B00000E780C0EB17458D
:10176000FF1F1305A56B1713FFFF6700839917452C
:10177000FF1F1305A56A82808DCD1713FFFFE702B7
:1017800003969747FF1F9387676D944301112E843B
:101790000A869745FF1F9385A56C97B00000E780E8
:1017A00000ED0A850294014505611713FFFF6700EC
:1017B00043957D5582801713FFFFE702439297B050
:1017C0000000E78040F89747FF1F23A9A76817F597
:1017D000FFFF1305E5C997A00000E780809B171362
:1017E000FFFF670003921747FF1F130767699317EF
:1017F000150008433E95FD572310F500828017130E
:10180000FFFFE702C38D2A84084009E51713FFFF95
:101810006700238F1C4158401CC06313E5005CC067
:101820008347550023200500F99BA302F50097A0EC
:10183000FFFFE780207CC9BF1713FFFFE702838803
:101840009747FF1F9387C76598432A8411CB834727
:10185000350093F7070289C70355050089450297AC
:101860001305440197900000E7800062835504004F
:101870000355E40097300000E780A00C485819C5D4
:1018800097A0FFFFE7800077232A04021305840353
:1018900097000000E780E0F68144B1499790FFFF90
:1018A000E780806E63CBA4028347340023200404C6
:1018B00093F727FCA301F40000489790FFFFE7800F
:1018C000A06D13161500814522859710FFFFE78054
:1018D00000841713FFFF67002382B38734030329B3
:1018E000040385043E994A8597000000E78060F173
:1018F0002304090065B78347350093F7070299E38E
:10190000014582808357E500E39CB7FEC167FD1760
:101910006316F60005458280054599A81703FFFF69
:10192000E702E37B93170601C187B2842A84014949
:101930006359F002835705009DCB01456367F600AC
:10194000034584003E953325A6001375F50F0DA0C1
:101950001C4813171900BA9783D70700E38E97FA2C
:1019600005099790FFFFE7802063E343A9FE014547
:101970001703FFFF6700E3781703FFFFE702837495
:10198000AE89AA849790FFFFE780C0562A8497D03B
:10199000FFFFE780A02EAA86014713068401970562
:1019A0000000938585E41745FF1F1305A54D97900B
:1019B000FFFFE780401D2A8925C98C441304C50018
:1019C00022859E0593F5050897A0FFFFE780403C20
:1019D000CC4083877400E18163DD070493E505084B
:1019E000228597A0FFFFE780A03A0D46938544002B
:1019F000228597A0FFFFE780C03683D504002285AB
:101A000097A0FFFFE780E03D83D52400228597A0C3
:101A1000FFFFE780003D03D6490083A5090022852A
:101A200097A0FFFFE780E0334A851703FFFF6700B9
:101A3000A36C93F5F5076DB71703FFFFE702236A61
:101A400001112A84328532C697A0FFFFE780E02784
:101A50009780FFFFE7806039835704001747FF1F17
:101A60001307875B3246231BF100930700F8A30D91
:101A7000F1001C471843231AA1008983858BB30703
:101A8000F740B28548083ECE231C0100230D01001B
:101A900097000000E78080EE05611703FFFF6700F5
:101AA00043661703FFFFE702E361004101453DC4C0
:101AB0009304C40026853289AE8997A0FFFFE78092
:101AC000C02495452A8A2685035B040197A0FFFF61
:101AD000E7802021268597A0FFFFE780603E8D45A7
:101AE000AA8A268597A0FFFFE780A01F268597A0DA
:101AF000FFFFE780E03C5C48420A135A0A01D29794
:101B00005CC423186401814763983A0146054D81FE
:101B1000330625419337160013F5F70F1703FFFF20
:101B20006700835D1703FFFFE702E35889692A8B8B
:101B3000AE8B328AB68A81440144314CFD199790AC
:101B4000FFFFE780604463CDA4009790FFFFE7802C
:101B5000A046018D33B5AA001703FFFF6700235984
:101B60003389840383270B003E9963170A00834758
:101B7000890085043E94E1B703560A00DE854A8554
:101B800033F6C90097000000E780E0F16DD105450C
:101B9000E1B71703FFFFE702835401112A847C0099
:101BA0000355E5003ECAB70707003ECC7C003ECE99
:101BB00097200000E78020082A898545480897A0DB
:101BC000FFFFE78020399945480897A0FFFFE7808D
:101BD000E015AA844A8597200000E780A0082380AA
:101BE000A4009747FF1F938727439C434166130632
:101BF00006F09396870113D78701558F93D68700F8
:101C0000F18E558FA207B706FF00F58FD98F1146C9
:101C10002C00138514003EC497B00000E780E0F567
:101C20005008A38204008945228597000000E780C0
:101C3000E0E019C9AA851305840397A0FFFFE78098
:101C4000E0313C4085073CC005611703FFFF67009A
:101C5000434B1703FFFFE70283489790FFFFE7809E
:101C6000A0352A8405049790FFFFE780E033330511
:101C7000A402F14791453305F50297200000E78063
:101C800020BA11E565551703FFFF670083479747A3
:101C9000FF1F23AFA71E9790FFFFE780E0312A8444
:101CA00005049790FFFFE78020303305A4028945A3
:101CB000060597200000E780A0B669D59747FF1F6B
:101CC00023A0A71C9790FFFFE780002F2A8405041C
:101CD0009790FFFFE780402D3304A4029747FF1F32
:101CE0002392871A9790FFFFE780002D2A84979010
:101CF000FFFFE780602B930714003385A702974707
:101D0000FF1F2392A71897E70000938727A517477F
:101D1000FF1F232DF7160145BDB71703FFFFE7028D
:101D2000633AAA842E8901449749FF1F9389C92EDB
:101D3000130A80069790FFFFE78000276347A400FF
:101D400001451703FFFF6700233B3305440383A7C7
:101D500009024A86A6853E9597000000E780E0B913
:101D600019E10504C1BF0545E9BF1703FFFFE702FD
:101D70008334AA8A2E8BB28B368C3A8A81440144F2
:101D80008149974CFF1F938C2C29130D8006979047
:101D9000FFFFE780602163C9A40011E085494E85FB
:101DA0001703FFFF6700A3343389A40383A70C0242
:101DB0005E86D6853E994A8597000000E780E0B3AD
:101DC0001DC19790FFFFE780201F0544636D45010B
:101DD000D2866286DA851305090397000000E78042
:101DE000A0D411C1854985045DB71703FFFFE70241
:101DF000632DC16441112A8901449749FF1F9389CA
:101E0000A921130A8006FD1436C632C42EC297904B
:101E1000FFFFE780601992452246B2466348A4005E
:101E2000014541011703FFFF6700032D33054403FC
:101E300083A709023E9509C683473500C18B9DC71C
:101E400091C68347350093F707028DC36306990057
:101E50008357E500639C27010357050001CB63E727
:101E6000E50083478500BA97E3CDF5FA050469BF1D
:101E70001703FFFFE7020325C1642A89014497493C
:101E8000FF1F93896919130A8006FD149790FFFFBD
:101E9000E78080116346A4001703FFFF6700C32596
:101EA0003305440383A709023E958357E500638AFF
:101EB0009700630499006396270197000000E7806C
:101EC000E0970504E1B71703FFFFE702431E8969A6
:101ED0002A8AAE8A328BB68B8144174CFF1F130CB3
:101EE000AC13930C8006314DFD199790FFFFE780EE
:101EF000A00B63C6A4001703FFFF6700031F33890D
:101F0000940383270C028355CA015A863E994A8559
:101F100097000000E780609E31C1814D15A0338499
:101F2000AD038327090303D60B00D68533F6C9001A
:101F30003E94228597000000E780E0B609E9850D10
:101F40009790FFFFE7804004E3CBADFC01A822851A
:101F500097000000E780E08A23040400850471B73D
:101F60001703FFFFE70223154169AA8A014A174BAD
:101F7000FF1F130B6B0A7D19C14B054C9790FFFF98
:101F8000E78080026346AA001703FFFF670023165D
:101F900093098006B3073A0383290B02BE9983D7BE
:101FA000E900638E270163842A01639A570103A421
:101FB000890301E84E8597000000E780C0BD050A4F
:101FC00075BF83570401639977099304C40026857C
:101FD00097A0FFFFE78060D385452A8D2685835C27
:101FE000040197A0FFFFE780C0CF268597A0FFFFE1
:101FF000E780A0E762056185635905048D45268564
:1020000097A0FFFFE780E0CD8945268597A0FFFFD9
:10201000E78020CD8945268597A0FFFFE78060CC2B
:102020008545268597A0FFFFE780E0CC8347050024
:10203000094793F7F707639AE7009945268597A024
:10204000FFFFE78040CBA30285014848337D2D0187
:10205000231894016A9548C40040A1BF1703FFFFED
:10206000E702E30737E404008327041D82979747BC
:10207000FF1F83C767E71715FF1F1305254BA30035
:10208000F5008327441C82978327841C814613060E
:10209000F00F8145014582971703FFFF6700630634
:1020A0001747FF1F130747D418439745FF1F83C5E2
:1020B000A5E39747FF1F9387A7E18346870303465E
:1020C00097036397D5009747FF1F238FC7E0828050
:1020D00083C587010347A7036317B6009747FF1F10
:1020E0002384E7E0828003C687016317C700974710
:1020F000FF1F238BD7DE828083C687011307500220
:102100006319D700930760021747FF1F230EF7DC00
:10211000828083C68701130660026315D600930789
:102120007002DDB783C7870155BF9747FF1F9387AD
:1021300027DAD44B0947638DE6081703FFFFE70250
:1021400003FA1749FF1F1309E9D53E8483470900A5
:10215000918B9DCFB7E4040083A7041D829783A7CA
:10216000441C1745FF1F130565D4829783A7841C61
:1021700081461746FF1F034666D581450145829774
:1021800021C583470900ED9B1747FF1F230CF7D09C
:102190008347040093F7F70F85CB91471747FF1F3D
:1021A0002322F7D497000000E78080EB970000001F
:1021B000E78040EFB7E70400BC4F41469145174523
:1021C000FF1F034565D182971703FFFF670063F385
:1021D00082801703FFFFE70283F08D4741116306FA
:1021E000F504C5476308F50285476310F502974774
:1021F000FF1F238DA7CEB7E70400BC4B930500104B
:102200001745FF1F034545CD829741011703FFFF87
:10221000670023EF85471747FF1F2309F7CCB7E770
:102220000400BC4B93050020E1BF9747FF1F938735
:1022300027CAD44B1147638DE600B7E7040083A794
:10224000071D8297B7E70400BC4B930500044DBF00
:1022500005491747FF1F232727C983C7070032C631
:102260002E8493F7F70FD5D3B7E4040083A7041D9A
:102270007D141374F40F8297E37689FCB245994775
:1022800003C61500E3F0C7FCFC4409061745FF1F11
:10229000130505C68297BC48930500081745FF1F24
:1022A000034585C3829779BF1703FFFFE70223E346
:1022B0001747FF1F1307C7C14047184B1C409746DD
:1022C000FF1F23ADF6C06316E4001747FF1F232945
:1022D000F7C0130584FE9790FFFFE780C0AA03555F
:1022E00064FF9780FFFFE780407397A0FFFFE780C0
:1022F00060D01703FFFF6700C3E01703FFFFE7028B
:1023000003DE9747FF1F9387A7BCD84BDC4789C7DD
:1023100097000000E78080F985471747FF1F2323B8
:10232000F7BC9747FF1F938727AC9C439305000298
:102330001745FF1F034545BA83C787031747FF1F8C
:102340002304F7BAB7E70400BC4B82971703FFFFDB
:10235000670023DB9747FF1F23AEA7B682801703D2
:10236000FFFFE70223D637E404007C4CA145174564
:10237000FF1F034565B682977C48A1451745FF1F9F
:10238000034585B59744FF1F938484B48297DC444A
:1023900089EB97000000E78080D91703FFFF6700F3
:1023A000A3D503D567FF9780FFFFE7800067AA8961
:1023B0006DD1D84891476310F7027C4C9145174581
:1023C000FF1F034565B182977C4891451745FF1F64
:1023D000034585B0829703A9490103D409018947C0
:1023E000B7E904001747FF1F232EF7AE83A7091D87
:1023F00021044204829783C784011715FF1F130528
:10240000E51261191717FF1FA302F71283A7491CD2
:10241000418082979747FF1F238A07AC83A7C91C77
:10242000814609469375F40F4A85829711E99747CB
:10243000FF1F83C7E7BB89C79700FF1FE780807B2B
:10244000B7E70400BC4F2146A1451745FF1F0345D0
:10245000A5A8829799B71703FFFFE70243C893F730
:10246000052001112E8481CF97000000E78020E92C
:102470001345042005611703FFFF670083C893F726
:102480000510A9CF9744FF1F938484A4DC489700CC
:102490000000E78020C11747FF1F1307E794184388
:1024A00083C78401034787036318F700DC4489C7A7
:1024B00097000000E78080DF85471747FF1F232331
:1024C000F7A2B7E70400BC4B930500021745FF1FB6
:1024D000034585A082971345041069BF93F705084B
:1024E000BDC79747FF1F83C7B7A0E9171946974590
:1024F000FF1F938505A01305D10093F4F70F17492B
:10250000FF1F0349E99E97A00000E78000679397AB
:102510000401C1831747FF1F1307079E231DF10006
:10252000231CF1009747FF1F9387879A3ACE3ACA38
:10253000D8432306010009CBDC43931589015408D5
:102540000D46E185680082971345040825B793F787
:102550002500A5C39747FF1F93878797D84B8947C7
:102560006306F7029747FF1F83C7C79313F7270038
:1025700011EF918B99CFB7E70400BC4F1306000A07
:1025800089451745FF1F034525958297134524006C
:10259000D5B59747FF1F938727859C4383C787033C
:1025A0001747FF1F2302F79497000000E78060DBC6
:1025B000F1BF93F7050281CB97000000E78060DA56
:1025C0001345040245BD93F7850081CB97000000B9
:1025D000E780E0D21345840071BD93F7150081CBED
:1025E00097000000E780A0B41345140061B593F78D
:1025F000450081CB97000000E78060B3134544009D
:1026000095BD93F7050495C39747FF1F83C7478C74
:1026100091CB97000000E780A0A491471747FF1FC8
:102620002322F78C13450404B1B593F70501014546
:10263000E38207E49747FF1F93878789D84B914729
:102640006310F7049747FF1F9387C7859C4313D7F1
:1026500027008583D98F858B91E7B7E7040083A78F
:10266000071D8297B7E70400FC4F91451745FF1FF0
:1026700003458586829785471747FF1F2324F786E2
:1026800013450401C5BB9747FF1F2383A79682808C
:102690001703FFFFE702A3A49747FF1F23A00784A8
:1026A0009747FF1F23AE078285471734FF1F130488
:1026B000A4731747FF1F2327F7821C4083C7870394
:1026C0001747FF1F2302F7829790FFFFE7800094D0
:1026D00029C59717FF1F23AFA7E41C40170500006B
:1026E0001305A5D783C787031737FF1F230EF77E70
:1026F0001717FF1FA30CF7E29737FF1FA38A077C6A
:10270000B7E7040083A7070882979737FF1F238541
:10271000A77C1703FFFF6700C39EB7C7898E938707
:1027200067ED1717FF1F2327F7E045BF1737FF1F78
:102730000347077A795555E79737FF1F93874779FE
:1027400003C7170005079736FF1FA383E67803C763
:1027500017008D463377D7029736FF1FA38AE67698
:1027600083C617001737FF1F13070768184393F630
:10277000F60FA9EE834787031737FF1F2306F77667
:1027800085471737FF1F2305F7749737FF1F938778
:1027900067719C430145998BA9E71703FFFFE70287
:1027A000039437E404007C48C1451735FF1F0345F7
:1027B000A57282973C4885451735FF1F0345C571B3
:1027C000829701451703FFFF6700A39383C7170094
:1027D00085466395F6008347970379BF8347A70330
:1027E00061BF82809737FF1F83C7876EA1CF170312
:1027F000FFFFE702C38E37E404009737FF1F2389EA
:10280000076C7C4885451735FF1F0345E56C8297AB
:102810007C4C91451735FF1F0345056C82977C481A
:1028200091451735FF1F0345256B82973C48C145ED
:102830001735FF1F0345456A829701451703FFFFC0
:102840006700238C795582801703FFFFE7022389F5
:102850002A84035565FF9780FFFFE780001C9737A8
:10286000FF1F9387E766D847BE841DEF9790FFFF51
:10287000E78080779C48232004009DEB9737FF1F5B
:1028800023A087669737FF1F23AA8764B7E7040052
:10289000BC4B89451735FF1F0345056482970145E9
:1028A0001703FFFF6700E385630A8700184375BFBE
:1028B00080C39737FF1F23A58762C9BF7955CDB75E
:1028C0001703FFFFE702A3819737FF1F93878772E4
:1028D0008843232605002324050051059780000026
:1028E000E780805A1703FFFF6700A38117F3FEFFFD
:1028F000E702E37E1734FF1F1304C46F1C4041112D
:1029000099CF9C472302B5002AC61CC1970000003E
:10291000E78040FB1C409C4B99C3324582974101A4
:1029200017F3FEFF6700E37D17F3FEFFE702237B4B
:102930004111444D328532842EC69790FFFFE780C7
:10294000C0522AC422859790FFFFE780205403A835
:102950004400630C0800B2458357440018402246E7
:1029600083D54500AA8626850298410117F3FEFF0C
:102970006700237917F3FEFFE7026376404D1DC819
:1029800008C09705000093856503130544019780EF
:102990000000E780003D9737FF1F9387A7659C43A2
:1029A000014589E79737FF1F23A6876417F3FEFFCA
:1029B000670023757D55DDBF17F3FEFFE702237225
:1029C000011168009305F00F02C602C802CA02CCCA
:1029D00002CE97000000E780A0F1056117F3FEFF2B
:1029E000670023729737FF1F9387C7609C43D847C0
:1029F000A1679D076319F70217F3FEFFE702236E35
:102A0000011132859790FFFFE7802046230AA1003D
:102A10008145680097000000E78080ED056117F3AD
:102A2000FEFF6700036E82809737FF1F9387875CE6
:102A30009C43D847A167938777036319F70217F37D
:102A4000FEFFE702C369011132859790FFFFE7801F
:102A5000C041230AA1008145680097000000E7807B
:102A600020E9056117F3FEFF6700A36982809737AD
:102A7000FF1F938727589C43D84795476316F70451
:102A800017F3FEFFE702A3650111328532849790A8
:102A9000FFFFE780803D230AA10022859790FFFF7A
:102AA000E780C03E83574400231BA10081453ECCF4
:102AB0001C4068003ECE97000000E78060E305619F
:102AC00017F3FEFF6700E3638280930785FF8DC3E2
:102AD0008327C5FF91CFDC4B81CF17F3FEFFE702C1
:102AE0000360032585FF829717F3FEFF670063618C
:102AF000828017F3FEFFE702835E2A843285979077
:102B0000FFFFE7808036BD4763EBA700184493774B
:102B1000F5000345B70041995D8DA305A70017F3A4
:102B2000FEFF6700035E17F3FEFFE702435B011140
:102B30007C003ECAB70707003ECC7C003ECE5C4D11
:102B4000A9C72A8413858700AE8497800000E78098
:102B5000A023A1652A899D0548089770FFFFE7809B
:102B600060439305803EB345B902480893F5F50FDD
:102B70009790FFFFE780C021014781465008A68556
:102B800022859770FFFFE7804066056117F3FEFF1F
:102B90006700235717F3FEFFE70263549700000016
:102BA000E780A0F817F3FEFF6700A35517F3FEFFB9
:102BB000E702E35201117C00AE843ECAA165B7076B
:102BC00007002A843ECC48087C00938575033ECEDE
:102BD0009770FFFFE780003C1C44480883C5B7009E
:102BE000BD899790FFFFE780A01A500801478146F2
:102BF000A68522859770FFFFE780205F056117F3A8
